:020000040000FA
:100000000848040001000000E0FA0000E0FA0000E7
:10001000E0FA0000E0FA0000E0FA0000E0FA000078
:10002000E0FA0000E0FA0000E0FA0000E0FA000068
:10003000E0FA000030F20000E0FA0000E0FA000010
:10004000E0FA000056F200007CF20000E0FA000046
:10005000E0FA00002AF000007CF00000F823000025
:10006000E0FA0000E0FA0000B8E400003CE1000023
:10007000E0FA00008EFA000010F80000E0FA00003C
:10008000E0FA00007AF90000E0FA0000E0FA00006F
:10009000E0FA0000B2F20000D8F2000050F80000D0
:1000A000B4F0000006F10000E0FA0000E0FA000001
:1000B000E0FA0000E0FA0000E0FA0000E0FA0000D8
:1000C000E0FA0000E0FA0000E0FA0000E0FA0000C8
:1000D000E0FA0000E0FA0000B6FA0000E0FA0000E2
:1000E000E0FA0000E0FA0000E0FA000044E5000059
:1000F000D2E10000E0FA0000E0FA000066FA000039
:100100008CF80000E0FA0000E0FA0000E0FA0000DD
:10011000E0FA0000E0FA0000E0FA0000E0FA000077
:10012000E0FA0000E0FA0000E0FA0000E0FA000067
:10013000E0FA0000E0FA0000E0FA0000E0FA000057
:10014000E0FA0000E0FA000052FA0000E0FA0000D5
:10015000E0FA0000E0FA0000E0FA0000E0FA000037
:10016000E0FA0000E0FA0000E0FA0000E0FA000027
:10017000E0FA0000E0FA0000CCE5000068E20000D0
:1001800016EF0000E0FA0000E0FA0000E0FA0000DC
:10019000E0FA0000E0FA0000E0FA0000E2F30000FC
:1001A000E0FA0000E0FA0000E0FA0000E0FA0000E7
:1001B000E0FA0000E0FA0000E0FA0000E0FA0000D7
:1001C000E0FA0000E0FA0000E0FA0000E0FA0000C7
:1001D000E0FA0000E0FA0000E0FA0000E0FA0000B7
:1001E000E0FA0000E0FA0000E0FA0000E0FA0000A7
:1001F000E0FA0000E0FA0000E0FA0000E0FA000097
:100200000000000000000000E0FA0000E0FA00003A
:10021000E0FA0000E0FA0000E0FA0000E0FA000076
:10022000E0FA0000E0FA0000E0FA0000E0FA000066
:10023000E0FA000030F20000E0FA0000E0FA00000E
:10024000E0FA000056F200007CF20000E0FA000044
:10025000E0FA00002AF000007CF00000F823000023
:10026000E0FA0000E0FA0000B8E400003CE1000021
:10027000E0FA00008EFA000010F80000E0FA00003A
:10028000E0FA00007AF90000E0FA0000E0FA00006D
:10029000E0FA0000B2F20000D8F2000050F80000CE
:1002A000B4F0000006F10000E0FA0000E0FA0000FF
:1002B000E0FA0000E0FA0000E0FA0000E0FA0000D6
:1002C000E0FA0000E0FA0000E0FA0000E0FA0000C6
:1002D000E0FA0000E0FA0000B6FA0000E0FA0000E0
:1002E000E0FA0000E0FA0000E0FA000044E5000057
:1002F000D2E10000E0FA0000E0FA000066FA000037
:100300008CF80000E0FA0000E0FA0000E0FA0000DB
:10031000E0FA0000E0FA0000E0FA0000E0FA000075
:10032000E0FA0000E0FA0000E0FA0000E0FA000065
:10033000E0FA0000E0FA0000E0FA0000E0FA000055
:10034000E0FA0000E0FA000052FA0000E0FA0000D3
:10035000E0FA0000E0FA0000E0FA0000E0FA000035
:10036000E0FA0000E0FA0000E0FA0000E0FA000025
:10037000E0FA0000E0FA0000CCE5000068E20000CE
:100380009E480100E0FA0000E0FA0000E0FA0000F8
:10039000E0FA0000E0FA0000E0FA0000E2F30000FA
:1003A000E0FA0000E0FA0000E0FA0000E0FA0000E5
:1003B000E0FA0000E0FA0000E0FA0000E0FA0000D5
:1003C000E0FA0000E0FA0000E0FA0000E0FA0000C5
:1003D000E0FA0000E0FA0000E0FA0000E0FA0000B5
:1003E000E0FA0000E0FA0000E0FA0000E0FA0000A5
:1003F000E0FA0000E0FA0000E0FA0000E0FA000095
:1004000000480400010000004F472300607D2400E5
:1004100000018800000000000B000700005D2B00B9
:100420000100200010000700000020000000E00094
:100430000200320000000200000000006CBF020059
:10044000000000000000FE004440A90000AD2100B3
:100450000000E0000300320000002000A00188003E
:100460004440A80000000600F8FF2000591C2100AD
:1004700091018800800078000000EB001A0037002E
:100480008180E80032A0B4009101BA00E28040000F
:1004900032A0B4009102BA00E280400032A0B40061
:1004A0000002EB00472BDE00F507B200602CE100F4
:1004B00009003A00330007000700E00002003200A4
:1004C0000059EB00010037000201E8008301E90058
:1004D000F8FF3E00040037006128E100010032000F
:1004E0000082EB00040007001101BA000200E000E6
:1004F000E3FF3A0000000600220007000700E000CA
:10050000020032003159BA00020037008100E800D1
:100510000201E8008301E90017003200190007001A
:100520000700E000020032002159BA000200370043
:100530008100E9000201E8008301E9000D003200BA
:100540000400E00003003A00E280400032A0B40062
:10055000E9FF37000B0007000700E000020032004F
:1005600011D9BA00010037000201E8008301E90057
:10057000F5FF3A008100E800E180400032A0B400BD
:10058000000006000810E600020037000910E6002F
:10059000020037008083EB00000006008003EB00C0
:1005A000000006008A1F78008B1F780000000600FC
:1005B00091018800800478000000EB001A003700E9
:1005C000E284440032A0B4009905BA00E2844400F9
:1005D00032A0B4009906BA00E284440032A0B4000C
:1005E0000006EB00476FDE00FD07B200636CE10020
:1005F00003003A00EBFF07000000EB000A003700A1
:10060000606CE10004003A00005DEB008B05E9003E
:10061000FDFF3E00040037006168E1000100320088
:100620000086EB000B00070019C7BA001905BA00D5
:100630000E04E00003003A000A00E000E0FF3A0088
:1006400000000600FE07B2009E0188008A047800C0
:10065000F5FF3700395DBA008B05E9000C00320068
:10066000295DBA008B05E900080032000C00E000AB
:1006700003003A00E284440032A0B400F5FF3700E2
:1006800019DDBA008B05E900FAFF3A008904E80099
:10069000E184440032A0B40000000600D2FA040055
:1006A0000000000052D7040000000000009A04007F
:1006B000000000000EC10400000000001E9B0400AA
:1006C00000000000C6CD040000000000AEBE040023
:1006D00000000000E4BD040000000000FEBD0400B6
:1006E000000000004CBE04000000000032E90400DD
:1006F0000000000070E0040000000000CCF30400E3
:1007000000000000EAC1040000000000C2B10400C3
:1007100000000000FAB9040000000000F6B904006F
:100720000000000030BA040000000000FEB9040020
:100730000000000062BA040000000000A66404008B
:1007400000000000D86404000000000008650400F8
:10075000000000004A6504000000000092650400EB
:1007600000000000DA6504000000000020660400BC
:10077000000000009866040000000000E466040029
:1007800000000000306704000000000090670400D3
:1007900000000000FE670400000000007C68040008
:1007A00000000000CC68040000000000E8680400BD
:1007B000000000007069040000000000C869040027
:1007C00000000000046A040000000000406A040009
:1007D00000000000A66A040000000000D06B0400C6
:1007E00000000000026C040000000000266C040001
:1007F00000000000746C040000000000F26C0400B3
:1008000000000000406D0400000000008A6D04003C
:1008100000000000B86D040000000000EA6D040054
:10082000000000002C6E040000000000489C040042
:1008300000000000B69C0400000000007C9C040046
:1008400000000000F09C040000000000709D040007
:1008500000000000AE9D040000000000469E040061
:1008600000000000AA9E040000000000789E040022
:100870000000000076A0040000000000DC9E0400E0
:10088000000000003A9F040000000000D29F040016
:100890000000000008A004000000000024A00400E4
:1008A0000000000040A0040000000000A6A004001A
:1008B00000000000DCA0040000000000F8A004001C
:1008C0000000000060A104000000000090A10400EE
:1008D00000000000C0A1040000000000ECA1040022
:1008E000000000002A9D04000000000028BF040052
:1008F000000000006022B800060220000000D000C6
:100900008180D2000482D2008582D2000000A00043
:100910000202520083825A000300310002024200A8
:1009200083824A000000A1000603E900F3FF3A00B9
:1009300000000600020AB900001BB9000200B8005E
:10094000810042008100430000000600889FBE0035
:100950008A9FBE008C1F78000006EB00E00F50005D
:10096000E08F5800E00F5900E08F590007003D006C
:100970006044B8006055B8000000540081805C00FD
:1009800002015D0083815D001C002000E00F520029
:10099000E08F5A00E00F5B00E08F5B0007003D0036
:1009A0006044B8006055B8000402540085825C00C1
:1009B00006035D0087835D000C00A200170107009D
:1009C0000C00E000060032006022B8006033B8007E
:1009D0000000520081805A0002015B0083815B00AD
:1009E0004F0678004F05BE004F04BE000000060011
:1009F000889FBE008A9FBE0030044200B0844A0037
:100A000030054B0090854B006000B1000898BE0097
:100A10000A90BE00C10007000200310068004000DB
:100A20001008E8004F05BE004F04BE00000006009D
:100A3000889FBE008A9FBE003004BE002005BE0015
:100A40000418540005985C0006185D0007985D00C6
:100A500011002000B1000700010039008000EB0008
:100A6000108810004F05BE004F04BE0000000600B5
:100A70001200FA00889FBE008A9FBE008C9FBE00B5
:100A8000E0B79F00F1B79F0082BF9F0093BF9F0018
:100A90000605BE000404BE000000EB00D0B79F00B6
:100AA000C0B79F00B0B79F00A0B79F0090B79F004E
:100AB0000006EB005FB19700CFB0970082014100C4
:100AC0003FB097000200E00004003D0098000700DE
:100AD0007E805700C6FF0700030037009400070020
:100AE0007E805700D2FF0700DFB697000D00E000C0
:100AF0000C0035006FB29700FFB297000FBB970054
:100B00009FBB970010002000010020006011B8007A
:100B100000027200818272000203730083837300FB
:100B2000580007000C06E80001042000810F560061
:100B3000E0FF3A000D00E00004003D000802BE00A6
:100B40000A03BE007E805700A9FF07005FA8970038
:100B50000000E00005003A001FB29700AFB2970016
:100B60003FB39700CFB39700460007006FB09700E0
:100B7000FFB097000FB997009FB997004F06BE00CE
:100B80004F05BE004F04BE000080FA0000000600C2
:100B9000881F780018002000881F7800B4FF070025
:100BA0008F87E9004F04780000000600801FEB00EB
:100BB000AFFF07008F87E90000000600889FBE0096
:100BC0008A9FBE003D00070007003D00400007006F
:100BD000180020004500070008003D002B0007001A
:100BE0000004EB00050037000004EB003F000700A5
:100BF00002003D002500070018002000E4FF070068
:100C00000800E000010032003D0007004F05BE0073
:100C10004F04BE0000000600889FBE008A9FBE00F1
:100C20008C1F78002500070008003D002800070001
:100C30001C0020000820E10009A8E1000AB0E10042
:100C40000BB8E10007003D00050037000006EB008F
:100C50002600070003003D006044B8006055B8005E
:100C60000C000700D1FF07000C00E000010032007B
:100C7000230007004F0678004F05BE004F04BE005A
:100C80000000060008000700000006006044B800ED
:100C90006055B8000402540085825C0006035D00C4
:100CA00087835D0000000600A4B79F00B5B79F00D2
:100CB000C6B79F00D7B79F0000000600E00F5000A6
:100CC000E08F5800E00F5900E08F59000000060047
:100CD0006044B8006055B8000000540081805C009A
:100CE00002015D0083815D0000000600E00F5200FC
:100CF000E08F5A00E00F5B00E08F5B000000060011
:100D00006022B8006033B8000000520081805A00B1
:100D100002015B0083815B00000006000440E100EB
:100D200005C8E10006D0E10007D8E1000000060098
:100D30004F09DE0082817100B3B79F004F01DE00D2
:100D40008180400082807000A1B79F008FB0970023
:100D50004F09DE00000040000200700090B79F00C5
:100D60007FA897004F01DE008180400082807000E4
:100D700081B79F000D0007004F3ADE0000004000E1
:100D800004007000F0AF9F0008000700040242005A
:100D900085824A0006034B0087834B00C2FF070091
:100DA0000802BE000A03BE00000006002FB2970032
:100DB000BFB297004FB39700DFB397000000060063
:100DC000839F68000100E00002003D006000100009
:100DD000E08018000300E00002003D006001110007
:100DE000E0811900C3FE07004F00E00002003B0055
:100DF00060001000E080180000000600800178000C
:100E0000110009008280D8008001FD001100090056
:100E10004288D8008300780000000600889FBE004A
:100E20008A9FBE008C9FBE000404B8000506B8006F
:100E30008904460060854E000606B8000A05460093
:100E4000E0854E000706B8008B054600040EB8008A
:100E5000890446000A854E00E0854D00050EB80065
:100E60000A0546008B854E00060EB8008B0546002D
:100E70000416B8000A0546008B854E000516B8001A
:100E80008B054600041EB8008B0546000800BE0016
:100E90000A01BE004F06BE004F05BE004F04BE0053
:100EA000000006008001780002003700B159780088
:100EB0000201E9000200E000FCFF3A000000060029
:100EC0008001780002003700815978000201E900B2
:100ED0000200E000FCFF3A000000060080007800FD
:100EE0003104E000FEFF3A000080EA00008040008C
:100EF00000000600E68747008E1F7800D0BF9F00E5
:100F0000E1BF9F000E0037005FBA970014407800E1
:100F1000EFB99700934078000201E900814F50003B
:100F2000040032000080FB008180FB0001005000C3
:100F30000600370066875700041FE800030FE8002B
:100F40000200E000F0FF3A000000EB004F077800DD
:100F50006F00B100000006006D61000074680000C1
:100F60002E6300006F70000079000000636F0000C6
:100F70007069000065730000207300007263000058
:100F8000207400006F20000064650000737400008E
:100F9000206500006C6500006D6500006E74000047
:100FA0002062000079200000656C0000656D000083
:100FB000656E00007400000064650000737400003A
:100FC000007300007263000000000000AC870000A6
:100FD000B6870000FFFF0000DC870000FFFF000075
:100FE000E187000000000000000000006D610000CB
:100FF000746800002E660000696C00006C00000040
:10100000666900006C6C00007320000064650000DD
:1010100073740000207700006974000068200000ED
:10102000636F00006E730000746100006E74000056
:1010300020760000616C00007565000000760000FD
:10104000616C00007565000000000000F68700007C
:1010500000880000FFFF0000DC87000001000000A6
:101060001F88000000000000000000006D6100000B
:10107000746800002E610000646400007363000067
:10108000616C000061720000006100006464000097
:1010900020730000636100006C610000722000009A
:1010A000746F00002065000061630000682000008C
:1010B000656C0000656D0000656E00007420000026
:1010C0006F66000020730000726300002061000062
:1010D0006E64000020730000746F000072650000F1
:1010E0002072000065730000756C00007420000021
:1010F000746F00002064000065730000740000003D
:1011000073630000616C0000617200000000000069
:101110003688000045880000FFFF0000DC870000E3
:10112000FFFF0000E1870000010000008088000050
:1011300000000000000000006D6100007468000005
:101140002E6100006464000000610000646400001F
:101150007320000073720000633100002061000002
:101160006E640000207300007263000032200000F3
:10117000746F00002064000065730000742C000090
:10118000206500006C6500006D6500006E74000055
:101190002062000079200000656C0000656D000091
:1011A000656E00007400000073720000633100007F
:1011B0000073000072630000320000009C88000091
:1011C000A5880000FFFF0000DC870000FFFF000093
:1011D000D4880000FFFF0000D98800000000000054
:1011E000000000006D610000746800002E730000B4
:1011F00075620000007300007562000073740000E7
:1012000072610000637400007320000073720000BC
:101210006332000020660000726F00006D20000045
:101220007372000063310000207400006F20000022
:1012300064650000737400002C200000656C0000E1
:10124000656D0000656E000074200000627900008A
:10125000206500006C6500006D6500006E74000084
:1012600000000000F2880000FB880000FFFF000083
:10127000DC870000FFFF0000D4880000FFFF0000B3
:10128000D988000000000000000000006D6100002F
:10129000746800002E6D0000756C0000006D000089
:1012A000756C000074690000706C000069650000D6
:1012B00073200000737200006331000020610000A1
:1012C0006E64000020730000726300003220000092
:1012D000746F00002064000065730000742C00002F
:1012E000206500006C6500006D6500006E740000F4
:1012F0002062000079200000656C0000656D000030
:10130000656E000074000000468900004F890000EF
:10131000FFFF0000DC870000FFFF0000D488000012
:10132000FFFF0000D988000000000000000000005E
:101330006D610000746800002E6400006976000092
:1013400000640000697600006964000065730000B5
:1013500020730000726300003120000062790000F9
:10136000207300007263000032200000746F0000E0
:101370002064000065730000742C000020650000EC
:101380006C6500006D6500006E7400002062000056
:1013900079200000656C0000656D0000656E00003E
:1013A0007400000098890000A1890000FFFF000080
:1013B000DC870000FFFF0000D4880000FFFF000072
:1013C000D988000000000000000000006D610000EE
:1013D000746800002E6D0000696E00000077000048
:1013E00072690000746500007320000074680000DA
:1013F000652000006D6900006E6900006D750000D9
:101400006D2000006F660000207300007263000012
:1014100031200000616E0000642000007372000043
:1014200063320000207400006F200000646500003B
:10143000737400002C200000656C0000656D0000D6
:10144000656E0000742000006279000020650000D5
:101450006C6500006D6500006E7400000000000007
:10146000E6890000EF890000FFFF0000DC87000034
:10147000FFFF0000D4880000FFFF0000D9880000B3
:1014800000000000000000006D61000074680000B2
:101490002E6D000061780000007700007269000086
:1014A000746500007320000074680000652000006F
:1014B0006D610000786900006D7500006D2000000E
:1014C0006F6600002073000072630000312000008E
:1014D000616E00006420000073720000633200003F
:1014E000207400006F200000646500007374000029
:1014F0002C200000656C0000656D0000656E00002A
:101500007420000062790000206500006C65000016
:101510006D6500006E74000000000000448A000049
:101520004D8A0000FFFF0000DC870000FFFF000085
:10153000D4880000FFFF0000D988000000000000F0
:10154000000000006D610000746800002E63000060
:101550006C6100006D700000006300006C610000B1
:101560006D700000207300007263000020740000A2
:101570006F2000006C6F0000772F0000686900008A
:1015800067680000206200006F7500006E64000054
:1015900073200000696E0000746F0000206400007A
:1015A00065730000742C0000206500006C6500006D
:1015B0006D6500006E74000020620000792000005C
:1015C000656C0000656D0000656E00007400000031
:1015D0006C6F000077000000686900006768000019
:1015E00000000000A28A0000AD8A0000FFFF00009A
:1015F000DC870000FFFF0000E1870000FFFF000024
:10160000E88A0000FFFF0000EC8A000000000000F4
:10161000000000006D610000746800002E6400008E
:101620006F740000007700007269000074650000AC
:10163000732000007468000065200000646F0000E3
:1016400074200000707200006F6400007563000079
:10165000742000006F6600002073000072630000B9
:1016600031200000616E00006420000073720000F1
:1016700063320000207400006F20000064650000E9
:10168000737400002C200000616600007465000087
:10169000722000006120000073680000696600008D
:1016A00074000000736800006966000074000000A8
:1016B0000A8B0000138B000001000000DC87000093
:1016C000FFFF0000D4880000FFFF0000D988000061
:1016D00001000000528B000000000000000000002C
:1016E0006D610000746800002E73000074610000DA
:1016F0007400000070650000726600006F720000E8
:101700006D730000207300007461000074690000B4
:101710007374000069630000732000006F6E0000A6
:101720002073000072630000006D0000696E00000D
:10173000006D000061780000006D00006561000030
:101740006E000000708B00007A8B0000FFFF00002D
:10175000E187000001000000958B000001000000FF
:10176000998B0000010000009D8B0000000000002C
:10177000000000006D610000746800002E61000030
:1017800072670000626F0000756E000064730000F5
:1017900000670000657400002074000068650000A8
:1017A000206900006E64000069630000657300003A
:1017B0002028000061720000676D0000696E000063
:1017C0002C20000061720000676D0000617800004D
:1017D000292000006F66000020740000686500008A
:1017E000206C0000696D0000697400002076000024
:1017F000616C000075650000732000006F660000DA
:101800002073000072630000006100007267000036
:101810006D6900006E00000061720000676D0000DD
:101820006178000000000000BA8B0000C98B000046
:10183000FFFF0000E187000001000000058C0000B0
:10184000010000000C8C00000000000000000000FF
:101850006D610000746800002E7300006F7200005C
:1018600074000000736F00007274000020610000BB
:101870007272000061790000206900006E20000093
:10188000706C000061630000650000006172000080
:101890007261000079000000288C0000328C00008A
:1018A000FFFF0000468C0000000000000000000068
:1018B0006D610000746800002E6D0000756C000002
:1018C0006469000076000000706500007266000028
:1018D0006F7200006D7300002064000065730000EB
:1018E000742000003D200000286100002A620000F2
:1018F000292F000063200000696E000020330000E3
:10190000322000006269000074730000206500004E
:101910006C6500006D6500006E74000020620000C0
:1019200079200000656C0000656D0000656E0000A8
:10193000740000006100000062000000630000000D
:10194000588C0000648C0000FFFF0000DC87000062
:10195000FFFF00009A8C0000FFFF00009C8C00003D
:10196000FFFF00009E8C000000000000000000004F
:101970006D610000746800002E6100007461000059
:101980006E3200000070000065720000666F00009B
:10199000726D000073200000646500007374000025
:1019A000203D000020610000746100006E320000E4
:1019B000287900002C78000029200000656C0000C8
:1019C000656D0000656E0000742000006279000003
:1019D000206500006C6500006D6500006E740000FD
:1019E000007900000078000000000000B88C0000C2
:1019F000C38C0000FFFF0000DC870000FFFF000039
:101A0000F18C0000FFFF0000F38C000000000000DC
:101A1000000000006D610000746800002E7300007B
:101A2000696E00000070000065720000666F0000C3
:101A3000726D000073200000646500007374000084
:101A4000203D000020730000696E0000287800002F
:101A500029200000656C0000656D0000656E0000C7
:101A60007420000062790000206500006C650000B1
:101A70006D6500006E740000000000000A8D00001B
:101A8000138D0000FFFF0000DC870000FFFF000057
:101A9000F38C000000000000000000006D610000F9
:101AA000746800002E6300006F7300000070000077
:101AB00065720000666F0000726D00007320000008
:101AC0006465000073740000203D00002063000086
:101AD0006F7300002878000029200000656C00006A
:101AE000656D0000656E00007420000062790000E2
:101AF000206500006C6500006D6500006E740000DC
:101B0000000000004E8D0000578D0000FFFF000018
:101B1000DC870000FFFF0000F38C000000000000E5
:101B2000000000006D610000746800002E7200006B
:101B30006F74000032000000726F000074610000DA
:101B40007465000073200000762000006F660000BE
:101B5000206100006E6700006C65000020610000DD
:101B6000207400006F2000006465000073740000A2
:101B70000076000000000000928D00009C8D0000A7
:101B800002000000DC87000002000000B98D0000A8
:101B9000010000009A8C000000000000000000001E
:101BA0006D610000746800002E7300007172000007
:101BB0007400000070650000726600006F72000023
:101BC0006D73000020640000657300007420000045
:101BD0003D2000007371000072740000287800003E
:101BE00029200000656C0000656D0000656E000036
:101BF0007420000062790000206500006C65000020
:101C00006D6500006E74000000000000D08D0000C3
:101C1000DA8D0000FFFF0000DC870000FFFF0000FE
:101C2000F38C000000000000000000006D61000067
:101C3000746800002E6E00007A7300006571000069
:101C400000770000726900007465000020740000D5
:101C50006F200000646500007374000020740000B1
:101C600068650000206D000069640000646C00007D
:101C700065200000696E00006465000078200000A7
:101C80006F6600002074000068650000206C000092
:101C9000617200006765000073740000207300002B
:101CA00065710000756500006E630000652000002E
:101CB0006F660000206E00006F6E00002D7A00003D
:101CC000657200006F200000656C0000656D00000B
:101CD000656E00007473000020660000726F0000E3
:101CE0006D20000073720000632C0000202D0000A6
:101CF0003120000069660000206E00006F74000053
:101D0000206600006F7500006E640000206F000008
:101D10007220000069660000207300006D61000001
:101D20006C6C0000657200002074000068610000A7
:101D30006E2000006D6900006E4C0000656E0000B2
:101D400067740000680000006D6900006E4C0000C0
:101D5000656E00006774000068000000168E0000C9
:101D6000218E000001000000DC870000FFFF000062
:101D7000E187000001000000A48E000000000000C8
:101D8000000000006D610000746800002E72000009
:101D9000616E000064000000666900006C6C000069
:101DA000206100007272000061790000207700005D
:101DB0006974000068200000726100006E64000019
:101DC0006F6D000020760000616C000075650000FA
:101DD00073000000C28E0000CC8E0000FFFF0000E8
:101DE000DC870000000000000000000064650000C7
:101DF00071750000652E0000736900007A650000AF
:101E000000720000657000006F7200007420000016
:101E1000736900007A650000206F000066200000F2
:101E200064650000737400000064000065710000C8
:101E30007565000000730000697A0000650000000D
:101E4000F68E0000018F0000FFFF0000158F0000DC
:101E5000010000001B8F00000000000000000000D7
:101E60006465000071750000652E00006765000064
:101E700074000000666900006C6C000020640000C3
:101E80006573000074200000667200006F6D000032
:101E9000206400006571000075650000206100008D
:101EA00074200000696E0000646500007800000086
:101EB000696E00006465000078000000308F00004B
:101EC0003A8F0000FFFF0000158F0000FEFF0000AA
:101ED000DC87000001000000588F000000000000B7
:101EE000000000006465000071750000652E0000B0
:101EF0007365000074000000636F000070690000EB
:101F000065730000207300007263000020740000FD
:101F10006F200000646500007175000065200000FE
:101F200061740000206900006E64000065780000A4
:101F300000000000728F00007C8F0000FFFF000097
:101F4000158F0000FEFF0000E18700000100000087
:101F5000588F0000000000000000000064650000D1
:101F600071750000652E0000696E00007365000049
:101F7000727400000073000068690000667400005D
:101F8000206400006571000075650000206100009C
:101F900074200000696E0000646500007820000075
:101FA00062790000206C0000656E0000287300005C
:101FB0007263000029200000616E000064200000B0
:101FC000696E0000736500007274000020730000E9
:101FD0007263000000000000AE8F0000BB8F0000A5
:101FE000FFFF0000158F0000FEFF0000E1870000EA
:101FF00001000000588F00000000000000000000F9
:102000006465000071750000652E000065720000B7
:1020100061730000650000007368000069660000DD
:1020200074200000646500007175000065200000E8
:1020300061740000206900006E6400006578000093
:1020400020620000792000006C6500006E20000016
:10205000746F00002065000072610000736500006D
:10206000006C0000656E00000000000000900000A1
:102070000C900000FFFF0000158F00000100000021
:10208000588F0000010000003190000000000000A7
:10209000000000006465000071750000652E0000FE
:1020A00070750000736800005F660000726F0000CA
:1020B0006E740000006900006E730000657200001D
:1020C000742000007372000063200000626500004D
:1020D000666F0000726500002074000068650000F3
:1020E00020660000726F00006E740000206F000018
:1020F0006620000064650000717500006500000046
:102100004A9000005B900000FFFF0000158F000068
:10211000FEFF0000E187000000000000000000005A
:102120006465000071750000652E00007075000088
:10213000736800005F620000616300006B000000D4
:10214000696E000073650000727400002073000067
:102150007263000020610000667400006572000078
:1021600020740000686500002062000061630000C8
:102170006B2000006F6600002064000065710000A5
:10218000756500000000000090900000A090000025
:10219000FFFF0000158F0000FEFF0000E187000038
:1021A0000000000000000000646500007175000080
:1021B000652E0000706F0000705F00006672000006
:1021C0006F6E000074000000666900006C6C000017
:1021D0002064000065730000742000006672000037
:1021E0006F6D000020660000726F00006E740000CA
:1021F000206F00006620000064650000717500001B
:102200006520000074680000656E00002065000015
:102210007261000073650000206500006C650000BD
:102220006D6500006E74000073000000D490000023
:10223000E4900000FFFF0000158F0000FEFF00008B
:10224000DC87000000000000000000006465000062
:1022500071750000652E0000706F0000705F000057
:1022600062610000636B000000660000696C0000A2
:102270006C2000006465000073740000206600009C
:10228000726F00006D20000062610000636B00004F
:10229000206F00006620000064650000717500007A
:1022A0006520000074680000656E00002065000075
:1022B0007261000073650000206500006C6500001D
:1022C0006D6500006E740000730000002691000030
:1022D00035910000FFFF0000158F0000FEFF000099
:1022E000DC8700000000000000000000000000008B
:1022F0009301000024030000B7040000480600001A
:10230000DA0700006B090000FC0A00008C0C0000DA
:102310001C0E0000AB0F00003B110000C8120000B3
:1023200056140000E31500006E170000F9180000B5
:10233000831A00000C1C0000941D00001A1F0000EE
:10234000A020000024220000A7230000292500006F
:10235000A826000027280000A4290000202B000048
:10236000992C0000122E0000872F0000FC30000086
:102370006F320000DF3300004E350000BA36000037
:10238000253800008D390000F33A0000573C00006A
:10239000B93D0000173F000074400000CE4100002E
:1023A000264300007B440000CD4500001D4700008F
:1023B0006A480000B4490000FC4A0000404C00009C
:1023C000824D0000C04E0000FC4F00003451000060
:1023D000695200009B530000CA540000F6550000EB
:1023E0001E5700004358000064590000835A000043
:1023F0009D5B0000B45C0000C85D0000D75E00007B
:10240000E45F0000EC600000F1610000F262000097
:10241000EF630000E9640000DE650000D0660000A4
:10242000BD670000A76800008C6900006E6A0000AC
:102430004B6B0000246C0000F96C0000CA6D0000BA
:10244000976E00005F6F000023700000E3700000D3
:102450009E7100005572000008730000B673000002
:102460006074000005750000A5750000427600004C
:10247000D97600006C770000FB77000084780000BC
:10248000097900008A790000067A00007D7A000050
:10249000EF7A00005D7B0000C67B00002A7C000014
:1024A000897C0000E47C0000397D00008A7D00000A
:1024B000D77D00001D7E0000607E00009D7E000034
:1024C000D67E0000097F0000397F0000627F000097
:1024D000877F0000A77F0000C27F0000D87F000038
:1024E000EA7F0000F67F0000FE7F0000FF7F000013
:1024F0008C020000DF0200003003000080030000B7
:10250000D10300002204000073040000C204000094
:1025100014050000B305000054060000F106000099
:102520008F0700002D080000CA08000063090000A2
:10253000FC090000340B00005C0C0000820D000060
:10254000A40E0000BD0F0000D3100000E211000037
:10255000E7120000EF140000CC16000092180000F3
:10256000401A0000D61B0000531D0000B51E0000DD
:102570000B200000792200008D2400006F2600004F
:102580001428000090290000E02A0000112C00000F
:10259000252D0000052F000089300000D3310000F8
:1025A000EC320000DD330000AE340000673500007F
:1025B0000D36000020370000FB370000B238000065
:1025C0004A390000CC3900003B3A00009B3A000039
:1025D000F33A0000833B0000F43B0000513C000054
:1025E0009F3C0000E13C00001A3D00004B3D000014
:1025F000783D0000C03D0000F93D0000283E00008D
:102600004F3E0000703E00008D3E0000A53E0000E1
:10261000BC3E0000E03E0000FD3E0000143F000014
:10262000283F0000383F0000473F0000533F0000B4
:102630005E3F0000703F00007F3F00008A3F0000C7
:10264000943F00009C3F0000A43F0000AA3F000010
:10265000AF3F0000B83F0000C03F0000C53F000092
:10266000CB3F0000CE3F0000D23F0000D53F00002E
:10267000D83F0000DC3F0000E03F0000E33F0000E7
:10268000E53F0000E83F0000E93F0000EB3F0000AD
:10269000EC3F0000EE3F0000F13F0000F13F000082
:1026A000F33F0000F43F0000F53F0000F53F00005D
:1026B000F73F0000F73F0000F93F0000F83F00003F
:1026C000FA3F0000FA3F0000FA3F0000FB3F000025
:1026D000FB3F0000FC3F0000FC3F0000FC3F00000F
:1026E000FE3F0000FD3F0000FD3F0000FD3F0000F9
:1026F000FE3F0000FE3F0000FE3F0000FE3F0000E6
:10270000FE3F0000FE3F000000400000FF3F0000D1
:10271000FF3F0000FF3F0000FF3F0000FF3F0000C1
:10272000FF3F0000FF3F0000FF3F0000FF3F0000B1
:10273000FF3F0000FF3F000000400000004000009D
:102740000040000000400000004000000040000089
:102750000040000000400000004000000040000079
:102760000040000000400000004000000040000069
:1027700000400000416400006472000065730000C6
:10278000732000006F750000742000006F66000069
:102790002073000065740000746900006E6700001B
:1027A00073000000536C000065650000702000009D
:1027B0006D6F000064650000206E00006F74000003
:1027C0002073000075700000706F000072740000CC
:1027D0006564000000450000727200006F72000026
:1027E0003A2000006D6900006E2000003D3D0000B1
:1027F00020300000784600004646000046460000B3
:1028000046460000462000002100000045720000FE
:10281000726F0000723A0000205500006E610000E7
:10282000626C000065200000746F000020660000EC
:102830006C61000073680000206200007974000081
:10284000656300006F64000065200000283100000F
:10285000292000002100000045720000726F000076
:10286000723A0000205500006E610000626C0000AA
:1028700065200000746F0000206600006C6100009D
:102880007368000020620000797400006563000036
:102890006F6400006520000028320000292000003D
:1028A0002100000045720000726F0000723A0000C3
:1028B000205500006E610000626C00006520000081
:1028C000746F0000206600006C61000073680000F7
:1028D0002062000079740000656300006F640000EE
:1028E000652000002833000029200000210000009E
:1028F000466C000061730000686900006E670000AC
:10290000204F00004B000000564D00002041000009
:1029100053530000455200005420000021000000E5
:1029200074680000796D0000696F00002D49000097
:10293000490000005F690000640000006576000047
:10294000656E0000742E0000736F00007572000049
:102950006365000000650000766500006E7400008D
:102960002E61000072670000730000005F660000C7
:102970007776000065720000736900006F6E0000DA
:10298000005F0000707200006F640000756300005B
:102990007449000064000000627500007474000057
:1029A0006F6E0000732E00005F7200006177000000
:1029B0000062000075740000746F00006E2E00004D
:1029C00062610000636B00007761000072640000C8
:1029D0000062000075740000746F00006E2E00002D
:1029E0006C650000667400000062000075740000F1
:1029F000746F00006E2E0000636500006E740000AE
:102A0000657200000062000075740000746F0000C1
:102A10006E2E0000666F0000727700006172000089
:102A20006400000062750000747400006F6E0000A6
:102A30002E720000696700006874000000620000E8
:102A400075740000746F00006E7300002E5F00004C
:102A50006D650000616E000000620000757400008A
:102A6000746F00006E7300002E5F00006E6F000038
:102A70006973000065000000707200006F7800004C
:102A80002E6800006F720000697A00006F6E00000F
:102A9000746100006C000000707200006F7800002C
:102AA0002E6300006F6D00006D2E00007278000034
:102AB0002E5F000070610000796C00006F61000003
:102AC0006473000000700000726F0000782E000038
:102AD000636F00006D6D00002E720000782E000004
:102AE0005F6900006E740000656E0000736900008D
:102AF000746900006573000000700000726F0000D0
:102B0000782E0000636F00006D6D00002E720000D3
:102B100078000000707200006F7800002E630000E3
:102B20006F6D00006D2E00007478000000700000D2
:102B3000726F0000782E0000677200006F75000051
:102B40006E6400002E6100006D620000696100008B
:102B50006E74000000700000726F0000782E00009C
:102B6000677200006F7500006E6400002E72000036
:102B7000656600006C650000637400006564000019
:102B800000700000726F0000782E00006772000075
:102B90006F7500006E6400002E640000656C00001C
:102BA00074610000006D00006F7400006F7200001F
:102BB0002E6C000065660000742E00007461000039
:102BC0007267000065740000006D00006F74000003
:102BD0006F7200002E7200006967000068740000C8
:102BE0002E74000061720000676500007400000030
:102BF0005F76000062610000740000005F69000001
:102C00006D6F0000740000006D6F0000746F0000B5
:102C1000722E00006C650000667400002E730000C8
:102C20007065000065640000006D00006F740000B6
:102C30006F7200002E720000696700006874000067
:102C40002E7300007065000065640000006D0000D8
:102C50006F7400006F7200002E6C0000656600004B
:102C6000742E0000707700006D0000006D6F000092
:102C7000746F0000722E0000726900006768000027
:102C8000742E0000707700006D000000616300008A
:102C900063000000746500006D7000006572000044
:102CA000617400007572000065000000726300002E
:102CB000352E00006164000064720000657300003E
:102CC0007300000072630000352E0000636F000087
:102CD0006D6D0000616E0000640000006D69000011
:102CE000632E0000696E0000746500006E730000C2
:102CF00069740000790000006D690000632E000017
:102D00007468000072650000736800006F6C00005A
:102D1000640000006D690000632E00005F6D00001C
:102D2000656100006E000000746900006D650000C0
:102D3000722E000070650000726900006F64000070
:102D400000610000636300002E5F000074610000FA
:102D500070000000736400002E70000072650000B7
:102D6000736500006E740000000000009094000085
:102D7000010000009A940000010000009E940000F1
:102D800020000000AB94000002000000B694000098
:102D900001000000C194000005000000CC94000078
:102DA00001000000D994000001000000E994000037
:102DB00001000000F59400000100000003950000F0
:102DC0000100000012950000050000001F950000A2
:102DD000050000002D950000070000003C95000054
:102DE000070000004C9500000700000063950000FC
:102DF000010000007D950000010000008A950000A0
:102E0000020000009795000002000000AB95000052
:102E100002000000C195000001000000D3950000F1
:102E200001000000E595000002000000F895000098
:102E300002000000FE950000010000000496000062
:102E40000100000015960000010000002796000018
:102E500001000000369600000300000046960000C6
:102E6000010000004A960000010000005696000094
:102E70000100000062960000010000006E96000054
:102E8000010000007C960000010000008A9600000E
:102E9000020000009496000001000000A1960000CE
:102EA00001000000AA9600000000000000000000E1
:102EB000DE000000AD000000CA000000FE000000BF
:102EC000BE000000EF00000004000000020000004F
:102ED000F6B9000030BA0000FEB9000062BA000086
:102EE000A6640000D8640000086500004A65000080
:102EF00092650000DA650000206600009866000018
:102F0000E46600003067000090670000FE67000084
:102F10007C680000CC680000E86800007069000070
:102F2000C8690000046A0000406A0000A66A000048
:102F3000D06B0000026C0000266C0000746C000076
:102F4000F26C0000406D00008A6D0000B86D00005A
:102F5000EA6D00002C6E0000489C0000B69C00004A
:102F60007C9C0000F09C0000709D0000AE9D000065
:102F7000469E0000AA9E0000789E000076A00000F9
:102F8000DC9E00003A9F0000D29F000008A00000D5
:102F900024A0000040A00000A6A00000DCA00000CB
:102FA000F8A0000060A1000090A10000C0A10000F6
:102FB000ECA100002A9D000028BF00004261000033
:102FC000636B000077610000726400002062000003
:102FD00075740000746F00006E20000073740000B0
:102FE00061740000757300002063000068610000D8
:102FF0006E67000065640000004C0000656600001C
:103000007420000062750000747400006F6E000090
:1030100020730000746100007475000073200000CC
:1030200063680000616E00006765000064000000D6
:10303000436500006E7400006572000020620000AD
:1030400075740000746F00006E200000737400003F
:103050006174000075730000206300006861000067
:103060006E67000065640000004600006F7200009B
:103070007761000072640000206200007574000037
:10308000746F00006E200000737400006174000013
:103090007573000020630000686100006E67000027
:1030A0006564000000520000696700006874000059
:1030B0002062000075740000746F00006E20000034
:1030C00073740000617400007573000020630000D9
:1030D000686100006E670000656400000062000027
:1030E00075740000746F00006E73000000420000F1
:1030F00075740000746F00006E730000207600008D
:10310000616C0000756500007320000075700000A0
:1031100064610000746500006400000070720000CB
:103120006F78000000500000726F000078690000A6
:103130006D6900007479000020760000616C000069
:103140007565000073200000757000006461000068
:103150007465000064000000707200006F78000069
:103160002E6300006F6D00006D00000044610000E0
:103170007461000020720000656300006569000052
:1031800076650000642000006F6E0000207400006F
:103190006865000020700000726F00007869000010
:1031A0006D69000074790000206300006F6D0000FD
:1031B0006D7500006E6900006361000074690000B5
:1031C0006F6E00000074000061700000004100009C
:1031D000207400006170000020690000732000006E
:1031E000646500007465000063740000656400009D
:1031F0000041000063630000656C00006572000020
:103200006F6D00006574000065720000207600009C
:10321000616C00007565000073200000757000008F
:103220006461000074650000640000006D690000C6
:103230006300000046690000726500006420000021
:1032400077680000656E0000206D00006963000073
:10325000726F0000706800006F6E00006520000053
:10326000696E0000746500006E73000069740000F0
:10327000792000006973000020610000626F000087
:10328000766500002074000068720000657300001D
:10329000686F00006C640000007300006F75000030
:1032A0006E6400002E660000696E00006973000005
:1032B0006865000064000000466900007265000057
:1032C0006420000077680000656E00002074000034
:1032D00068650000207000006C61000079620000E9
:1032E000616300006B2000006F6600002061000039
:1032F000207500007365000072200000696E0000F8
:1033000069740000696100007465000064200000B9
:10331000736F0000756E0000642000006973000088
:1033200020660000696E0000697300006865000097
:1033300064000000546500006D70000065720000BC
:103340006174000075720000652000007661000065
:103350006C7500006520000075700000646100005D
:103360007465000064000000726300003500000016
:1033700052430000352000006D65000073730000AB
:103380006167000065200000726500006365000051
:103390006976000065640000006D00006F74000035
:1033A0006F720000004D00006F7400006F7200002B
:1033B00020740000696D0000657200000074000058
:1033C000696D000065720000300000005469000063
:1033D0006D6500007220000030000000746900007C
:1033E0006D6500007231000000540000696D00003E
:1033F000657200002031000000000000D994000038
:10340000DE970000E9940000FD970000F5940000AD
:1034100018980000039500003598000012950000F0
:10342000539800006F980000779800008E98000075
:1034300093980000AC980000B6980000E398000054
:10344000E798000046960000F998000016990000E1
:103450001A9900004D9900005C9900004A960000FE
:103460009A990000B4990000B8990000CD99000025
:10347000D3990000DF990000E6990000EE99000062
:10348000F599000000000000000000005F730000DC
:1034900079730000746500006D2E000072650000F5
:1034A000626F00006F74000000520000656200004F
:1034B0006F6F000074200000746800006520000039
:1034C0006D690000637200006F6300006F6E0000A2
:1034D000747200006F6C00006C65000072000000E8
:1034E0005F73000079730000746500006D2E0000AA
:1034F0007365000074740000696E0000677300005B
:103500002E7200006561000064000000526500003A
:1035100061640000206100002073000065740000F9
:10352000746900006E6700000061000064640000C0
:10353000726500007373000000760000616C00008B
:1035400075650000005F000073790000737400006F
:10355000656D00002E730000657400007469000042
:103560006E670000732E000077720000697400001F
:1035700065000000577200006974000065200000BB
:10358000612000007365000074740000696E000023
:10359000670000005F73000079730000746500002D
:1035A0006D2E00007365000074740000696E0000E9
:1035B000677300002E6600006C61000073680000F5
:1035C000005700007269000074650000207400005C
:1035D00068650000207300006574000074690000D5
:1035E0006E67000073200000696E0000746F0000B9
:1035F000206600006C61000073680000000000009D
:1036000045720000726F0000723A000020730000E3
:10361000616D0000706C000065730000206D00009B
:1036200075730000742000006265000020690000CE
:103630006E2000005B2D000031320000382C0000AD
:1036400031320000375D000020720000616E000022
:1036500067650000005F00006C6500006473000097
:103660002E730000657400000053000065740000B4
:103670002074000068650000206C00006564000094
:10368000006C0000656400000062000072690000C8
:1036900067680000746E000065730000730000002E
:1036A000736F0000756E0000642E000072650000EC
:1036B000636F00007264000000530000746100003A
:1036C0007274000020720000656300006F720000D9
:1036D000646900006E670000206F00006620000033
:1036E000724E00002E77000061760000004E000050
:1036F000007300006F7500006E6400002E70000003
:103700006C610000790000005374000061720000D9
:1037100074200000706C000061790000626100009C
:10372000636B0000206F000066200000704E0000F8
:103730002E77000061760000007300006F750000B6
:103740006E6400002E720000657000006C61000065
:1037500079000000537400006172000074200000C2
:10376000706C00006179000062610000636B000012
:10377000206F000066200000724E00002E770000CF
:1037800061760000007300006F7500006E64000039
:103790002E6400007572000061740000696F000003
:1037A0006E0000004769000076650000206400009C
:1037B0007572000061740000696F00006E200000E7
:1037C000696E0000203100002F31000030730000CE
:1037D000206F000066200000724E00002E7700006F
:1037E00061760000006400007572000061740000E2
:1037F000696F00006E000000736F0000756E0000BE
:10380000642E00007379000073740000656D000081
:10381000005300007461000072740000207000000A
:103820006C61000079620000616300006B200000A1
:103830006F6600002073000079730000746500005B
:103840006D200000736F0000756E000064200000A2
:103850004E0000006C650000647300002E630000E1
:1038600069720000636C0000650000005365000091
:10387000742000006369000072630000756C000032
:103880006172000020720000696E00006720000075
:103890006C65000064730000006C000030000000E4
:1038A0006C310000006C0000320000006C3300003E
:1038B000006C0000340000006C350000006C00005B
:1038C000360000006C370000006C000065640000EA
:1038D000732E0000746F000070000000536500003C
:1038E000742000005247000042200000746F000066
:1038F000702000006C65000064000000726500002C
:103900006400000067720000656500006E00000042
:10391000626C000075650000006C000065640000CA
:10392000732E0000626F0000747400006F6D000061
:103930002E720000696700006874000000530000E8
:103940006574000020520000474200002062000021
:103950006F7400006F6D0000207200006967000046
:1039600068740000206C000065640000006C0000BA
:1039700065640000732E0000626F00007474000024
:103980006F6D00002E6C0000656600007400000082
:1039900053650000742000005247000042200000E0
:1039A000626F0000746F00006D2000006C65000005
:1039B00066740000206C000065640000006C00006C
:1039C00065640000732E00006275000074740000CE
:1039D0006F6E00007300000053650000742000004B
:1039E00062750000747400006F6E000073200000A8
:1039F0006C65000064730000006C000065640000EA
:103A0000732E0000707200006F7800002E680000B6
:103A10000053000065740000206800006F72000011
:103A2000697A00006F6E0000746100006C20000075
:103A3000707200006F780000696D0000697400000A
:103A4000792000006C65000064730000006C0000C9
:103A500065640000732E0000707200006F78000033
:103A60002E760000005300006574000020760000F0
:103A70006572000074690000636100006C20000042
:103A8000707200006F780000696D000069740000BA
:103A9000792000006C65000064730000006C000079
:103AA00065640000732E0000726300000053000084
:103AB0006574000020720000632000006C65000047
:103AC000640000006C650000647300002E73000049
:103AD0006F7500006E640000005300006574000004
:103AE000207300006F7500006E640000206C000001
:103AF00065640000006C000065640000732E000027
:103B0000746500006D700000657200006174000053
:103B1000757200006500000053650000742000000D
:103B20006E740000632000006C65000064000000FB
:103B3000736F0000756E0000642E00006672000056
:103B400065710000005000006C61000079200000E9
:103B50006672000065710000756500006E6300000C
:103B600079000000487A0000006400007300000043
:103B7000736F0000756E0000642E00007761000016
:103B8000766500000053000065740000207400009A
:103B90006865000020700000726900006D6100001F
:103BA0007279000020770000617600006520000037
:103BB0006F6600002074000068650000207400003B
:103BC0006F6E000065200000676500006E650000F4
:103BD00072610000746F00007200000077610000E5
:103BE0007665000000700000726F0000782E000003
:103BF000636F00006D6D00002E6500006E610000B7
:103C0000626C000065000000456E0000616200000B
:103C10006C650000206F00007220000064690000E5
:103C200073610000626C0000652000007468000091
:103C300065200000707200006F780000696D000060
:103C40006974000079200000636F00006D6D000052
:103C5000756E00006963000061740000696F000008
:103C60006E000000737400006174000065000000C5
:103C7000736400002E6F0000706500006E0000008D
:103C80004F700000656E000020610000206600009B
:103C9000696C0000652000006F6E00002074000059
:103CA00068650000205300004420000063610000AC
:103CB00072640000006E0000756D00006265000017
:103CC00072000000737400006174000075730000DE
:103CD00000730000642E0000777200006974000019
:103CE0006500000057720000697400006520000044
:103CF0006461000074610000207400006F20000007
:103D000074680000652000006F700000656E0000A0
:103D10006564000020660000696C0000650000001A
:103D200064610000746100000077000072690000A7
:103D300074740000656E000000730000642E0000C3
:103D400072650000616400000052000065610000BF
:103D500064200000646100007461000020660000BF
:103D6000726F00006D200000746800006520000084
:103D70006F700000656E0000656400002066000042
:103D8000696C00006500000072650000616400005D
:103D900000730000642E000073650000656B000076
:103DA00000530000656500006B200000746800008F
:103DB000652000006F700000656E00006564000003
:103DC00020660000696C000065000000706F000054
:103DD00073690000746900006F6E0000005F0000EE
:103DE000726600002E6E00006F64000065690000BE
:103DF0006400000053650000742000005769000053
:103E0000726500006C65000073730000204E0000B6
:103E10006F6400006520000049440000006E00004F
:103E20006F6400006549000044000000733000002A
:103E30002E7700006176000000730000322E000033
:103E40007761000076000000733300002E770000D9
:103E50006176000000730000342E000077610000DE
:103E600076000000733500002E77000061760000B8
:103E700000730000362E000077610000760000001D
:103E8000733700002E77000061760000000000000C
:103E9000480D00000D000000301100000700000078
:103EA000EC130000070000000019000007000000EC
:103EB000781E000007000000000000000000000065
:103EC000781E00000D00000000190000070000002F
:103ED000EC13000007000000301100000700000094
:103EE000480D000007000000000000000000000076
:103EF0004C040000070000009808000007000000C4
:103F00000000000000000000E40C000007000000BA
:103F1000301100000D000000C8190000070000006B
:103F200000000000000000009C27000002000000CC
:103F3000AB220000010000009D1C000002000000F8
:103F4000FB180000020000002D32000001000000FC
:103F5000322D000001000000462800000200000091
:103F6000E826000001000000BF220000020000005F
:103F7000FB18000002000000FF32000001000000FA
:103F8000C620000001000000762F000002000000A3
:103F90002C2E000001000000CE2C000001000000CB
:103FA000FD390000020000000000000000000000D9
:103FB000C819000005000000BE0A0000040000004F
:103FC00000000000000000003011000007000000A9
:103FD0007C15000007000000000000000000000049
:103FE00030110000070000007C15000007000000F1
:103FF000C8190000070000000000000000000000D9
:10400000222A00002B2C00003A3B00003C3D00001F
:104010003E3F00005B5D00007C7F000000800000F0
:104020009A900000418E0000418F00008045000002
:104030004545000049490000498E00008F9000006E
:10404000929200004F9900004F5500005559000012
:10405000999A00009B9C00009D9E00009F410000DB
:10406000494F000055A50000A5A60000A7A8000024
:10407000A9AA0000ABAC000021AE0000AFB0000068
:10408000B1B20000B3B40000B5B60000B7B800008C
:10409000B9BA0000BBBC0000BDBE0000BFC000003C
:1040A000C1C20000C3C40000C5C60000C7C80000EC
:1040B000C9CA0000CBCC0000CDCE0000CFD000009C
:1040C000D1D20000D3D40000D5D60000D7D800004C
:1040D000D9DA0000DBDC0000DDDE0000DFE00000FC
:1040E000E1E20000E3E40000E5E60000E7E80000AC
:1040F000E9EA0000EBEC0000EDEE0000EFF000005C
:10410000F1F20000F3F40000F5F60000F7F800000B
:10411000F9FA0000FBFC0000FDFE0000FF000000BB
:104120002E2E00002F2E00002E2F00006D6F00009D
:104130006C6F00006C6500002F69000032630000A6
:104140002F690000326300005F7000007269000098
:10415000762E0000680000002E2E00002F2E00009A
:104160002E2F00006D6F00006C6F00006C6500006A
:104170002F690000326300002F6D000061730000A2
:1041800074650000725F0000707200006F740000C0
:104190006F6300006F6C00002E63000000000000E1
:1041A0002E2E00002F2E00002E2F00006D6F00001D
:1041B0006C6F00006C6500002F6900003263000026
:1041C0002F690000326300005F7000007269000018
:1041D000762E0000680000002E2E00002F2E00001A
:1041E0002E2F00006D6F00006C6F00006C650000EA
:1041F0002F690000326300002F6D00006173000022
:1042000074650000722E0000630000002E2E000076
:104210002F2E00002E2F00006D6F00006C6F00002D
:104220006C6500002F690000326300002F690000F8
:10423000326300005F70000072690000762E00009B
:10424000680000002E2E00002F2E00002E2F0000F0
:104250006D6F00006C6F00006C6500002F6900003E
:10426000326300002F7300006C610000766500006F
:104270002E630000000000002E2E00002F2E0000F4
:104280002E2F00006D6F00006C6F00006C65000049
:104290002F740000696D0000657200002F7400002B
:1042A000696D0000657200002E63000000000000D0
:1042B00001000000000000000800000000000000F5
:1042C00040000000000000000001000000000000AD
:1042D00052490000464600000000000000000000B7
:1042E0005741000056450000666D00007420000034
:1042F00010000000000000000100000001000000AC
:10430000841E000000000000841E00000000000069
:1043100001000000080000006461000074610000FA
:1043200000000000000000004172000067750000FE
:104330006D6500006E740000206100007272000064
:104340006179000020730000697A00006520000098
:1043500069730000207400006F6F0000206C000083
:104360006172000067650000202800003E330000F5
:1043700032290000000000005F4C00004F470000A1
:10438000445500004D5000002E2300004021000045
:10439000005F000054450000535400004D4F0000E2
:1043A000442E00002340000021000000564D000074
:1043B000434F0000444500002E410000424F0000E2
:1043C000000000002E2E00002F2E00002E2F0000D7
:1043D0006D6F00006C6F00006C6500002F660000C0
:1043E0006C610000736800002F6600006C610000C3
:1043F000736800002E630000000000002E2E0000F5
:104400002F2E00002E2F00006D6F00006C6F00003B
:104410006C6500002F690000326300002F69000006
:10442000326300005F70000072690000762E0000A9
:10443000680000005F540000455300005453000022
:10444000440000005F7000006F770000657200009C
:104450006F66000066000000506F00007765000086
:10446000726F000066660000000000002E2E000043
:104470002F2E00002E2F00006D6F00006C6F0000CB
:104480006C6500002F75000061720000742F000041
:1044900075610000727400002E63000000000000CF
:1044A0002E2E00002F6D00006D61000037360000D9
:1044B000363000002E630000000000005F42000064
:1044C0004C570000484C0000564C00002E440000A1
:1044D0004154000000000000101100001412000000
:1044E0001300000001160000170000000380000008
:1044F0000F0F00000F00000001017800833E200034
:10450000830F500003003C0083C12F00830F500035
:1045100001003D00030078000281B900481ADD0067
:104520004810DE000000720000000600EA87470025
:10453000889FBE008A9FBE008C9FBE008E1F7800A1
:10454000000578002B87200081BF9F00A2872000F4
:104550006D862000AE8620000006EB000FB89700A5
:104560003002780080BF9F001BA2B90013322000E8
:1045700011000900432AD800000278006A007E007A
:10458000000242006087200060007E00F6032000E9
:104590000683B9004FA0DE000602420087024800F1
:1045A00002003B00F403B0000580B000CA28DD0023
:1045B0004624DE000884700008007800638720002D
:1045C00088317E00631C210083014600A899980071
:1045D0008802780005F0A7008502EA008425200003
:1045E000848F5200010034001209E800B012B000BC
:1045F00064252000840F500001003E000009EB00FC
:10460000E086200060007E006A027E000002520008
:104610001D034200860E7800652C2100850F530093
:1046200001003400850E7800A5D32E009D8F120066
:1046300001003D00850E78000000E00008003A000F
:104640001E00E800000F780075022000850F500062
:104650000400340080022000000F780001003700C1
:10466000000FEB00800220009E0F100004003A00B3
:10467000800EEB00800DEB000002EB00060037001F
:104680006522B9001D0078003600200011000900E5
:104690000600D800040240001B0242002500200052
:1046A000110009000502D80000027800840D78008E
:1046B00010322000800F520001003400800D78007D
:1046C000F0CD2F009B0F100001003D00800D780001
:1046D00020002000920F10000E00340060C1B300D3
:1046E000D2B79F00E3B79F00EA98020000000000E5
:1046F000300020005FB19700000978001B007800AF
:1047000024002000110009000400D800800D78006A
:10471000EFB197003B007800E09998000C86E80024
:104720000281E8008D86E8000E87E800E40F56005D
:104730008AFF3A00904380008AD602000000000001
:10474000A0438000B0D60200000000004F077800B0
:104750004F06BE004F05BE004F04BE00AF00B100C3
:1047600000000600881F780000047800D1868100D0
:104770001800780060FF070070438800E186810020
:10478000180090005CFF0700804388004F04780009
:10479000000006006628EF006828EF008002200075
:1047A00050438800604388006E28EF007028EF00B7
:1047B00000000600110020008096200010884000B4
:1047C000E442A800000006000000EB000081EB00BE
:1047D0008196200091084100010032000080EB002A
:1047E0000000E00001003A00E442A90000000600D9
:1047F00021E3A90085A0A9000040060000000000F8
:1048000000000000000000000000000000000000A8
:104810000000000000000000000000000000000098
:104820000000000000000000000000000000000088
:104830000000000000000000000000000000000078
:1078000002003700315878000201E9000200E00070
:10781000FCFF3A0000000600020037000158780023
:107820000201E9000200E000FCFF3A00000006004F
:10783000889FBE008A9FBE008C9FBE008E1F78006E
:10784000000478000206BE0058159000E81590006C
:107850008000EB00820F5500838F5D0038003200FE
:10786000484090000004E00024003200EE022000B6
:107870000807470014C0B3000A01BE008E0078005C
:1078800018409000D8AA020000000000110020005B
:107890000000E0002A003A00404498005809900097
:1078A000E8099000780890008810900002004000DD
:1078B00083804800800F5500818F5D000F003100EC
:1078C000B84490000B00370058089000E80890007A
:1078D0000A0540008B85480014C0B3000A01BE00B1
:1078E0008E00780018409000D8AA02000000000026
:1078F0008944E900E1CF5400F3FF3E008000EB0033
:10790000E00F5600E08F5E000D003200E102200023
:107910008880400014C0B3000C01BE0018409000E5
:1079200068AA020000000000110020000000E00032
:1079300003003A005C1498006D1498008000EB007E
:10794000010078004F0778004F06BE004F05BE00CB
:107950004F04BE0000000600881F78000004780075
:10796000E10220008880400014C0B300184090005D
:1079700068AA0200000000008000780030C0B30058
:107980000100E00045003A00D0222000080040003D
:107990001081FB004811DD00C022200008004000DB
:1079A0001080FB000201700020C0B30051A52A0026
:1079B000810F510039003A0078E29000C822DD00C2
:1079C0000400200068E090008080FB0000002000A0
:1079D000000272008182720048E090000080FB008B
:1079E0008000EB00000272008182720058E090007B
:1079F0004800DD008000EB0000027200818272000E
:107A00000580FB0080007800040078000001BE00C3
:107A100064142400450520000040EB00840F510051
:107A2000858F59001D00320038439100C833DD00B6
:107A300006002000284091008080FB00000020000C
:107A40000003730081837300084091000080FB00F5
:107A50008000EB00000373008183730018409100E5
:107A60004800DD008000EB00000373008183730099
:107A70000781FB0082017800060178000200BE0049
:107A800004006800858068000080700000F0A70096
:107A90000000EA000000EA004F00DE004F0478001A
:107AA00000000600920020000000E0000C00320000
:107AB0001004E0000A003200B0019000818F5100F4
:107AC00007003A00104090005CAA0200000000008D
:107AD0000001EB000008A30001003200320020008A
:107AE0000200780000000600889FBE008A1F780010
:107AF000000478006011B800080078004CFF07000F
:107B0000800478000900E00060003A0030C0B30053
:107B1000984F100054003A00584090000004E000D4
:107B2000510032006000B8005014980061149800B1
:107B3000EA02200008054500022020008000EB003A
:107B40000A00780034FF0700C0222000080040002F
:107B500051C5B30001487800D02220000800400041
:107B6000A1CAB3000148780020C5B300606C98003A
:107B7000706C98006F4040000074980011C4B3000E
:107B800011749800232120008881410022C7B3008E
:107B900082497800332120008881410082497800A1
:107BA00042212000080141000149780051212000B4
:107BB0008880400080487800780090008808900015
:107BC0006221200008014100004978007221200054
:107BD00008014100C801DE0003497800822120002D
:107BE00008014100400ADE00050020000449780039
:107BF00092212000080141004808DE000049780079
:107C000058009000E8009000A221200008014100E7
:107C100000497800B221200008014100C801DE00BF
:107C200003497800C221200008014100400ADE001B
:107C30000500200004497800D221200008014100FD
:107C40004808DE000049780014C0B300180990000D
:107C5000A80990008A00780018409000D8AA020075
:107C600000000000594498000001EB008040EB0048
:107C70001840900072AB02000000000000F0A70066
:107C80000000EA008004EA00CF4CDE000900780022
:107C90004F0578004F04BE0000000600F88747003B
:107CA000889FBE008A9FBE008C9FBE008E1F7800FA
:107CB00002447800100178009201FB000303B10038
:107CC000E98F510008003E0092429000A4C3B30027
:107CD00084CF520004003A000288E800B40020007B
:107CE0000300E000DA013A00BE4A80008E08780006
:107CF000C40020000E00E000D50132001E04E000A8
:107D00000D0032001E4090005CAA0200000000003E
:107D10000080FB000008A30007003A000002EB000F
:107D20000804E000CA0132000028A300C8013200A4
:107D3000A4002000C6013700004FEB000040EB001C
:107D40001047980058A90200000000000080FB00C6
:107D5000340020000008A300BD013A000804E00040
:107D600003003200A40020000028A300B8013A005C
:107D70006011B8000E007800F7FE07006011B8002F
:107D8000C2B79F00D3B79F00E14F50001B003A00DD
:107D90000EF09300D40020000004E000AC0132009B
:107DA0007EF19300C811DD00020020006EF0930008
:107DB0008080FB00000020000001710081817100C3
:107DC0004EF093000080FB008000EB00000171008A
:107DD000818171005EF093004800DD008000EB00BF
:107DE0000002710081827100C4B79F00D5B79F0067
:107DF0000401BE000E007800D7FE0700140020002A
:107E0000E34F500092013200D40020000004E00053
:107E10008F013A00AE789000C808DD001E7890000F
:107E20000080FB008100700000202000808F500047
:107E300087013A005EC490004844DD004EC09000C7
:107E40000080FB00080470008004EB00E00F540089
:107E5000E08F5C0012003A005ED49000C844DD0060
:107E6000080020004ED090008080FB000000200021
:107E700000047400818474002ED090000080FB0008
:107E80008000EB0000047400818474003ED09000F8
:107E90004800DD008000EB00000474008184740061
:107EA000580F9800690F9800EE78900031479800BD
:107EB0000140E900D4002000E14F500064013E0081
:107EC000BE7B9000274798000704E0006001320065
:107ED0000780FB000001E900000061005C013A003E
:107EE0000EC390004833DD007E7890000080FB00D8
:107EF00006037000460798006F00630054013A00C3
:107F00002EC190004811DD001EC090000080FB00D3
:107F1000020070006105B800AAB79F00BBB79F00C0
:107F2000E00F5500E08F5D0014003A001ED0900075
:107F3000C802DD00040020000ED190008281FB0009
:107F40000200200002027200838272006EC990005B
:107F50000281FB008001EB0002027200838272004A
:107F60007EC990004811DD008001EB00020672001E
:107F700083867200ACB79F00BDB79F00DE7D900086
:107F8000C85DDD004E7890000080FB008B0570001E
:107F9000D40020002E0132000181FB008001EB00A3
:107FA0000800BE00F4B79F0086BF9F00E7B79F00A0
:107FB0009A040200000000000006BE006158B800EC
:107FC000E0AF9F00F1AF9F000FBB97004430DE0091
:107FD0006FA99700FFA9970002004000E0804900C8
:107FE0000005460081854E008AB79F009BB79F0021
:107FF0007FB29700EFB397002FB09700BFB0970004
:108000008A0F50008B8F5800110139000A00500070
:108010008B8058000781FB008001EB007A0402008E
:10802000000000007FB297000FBB9700E00F5000E8
:10803000E08F58000601320015C0B30053FF200046
:10804000830F5000E08F58000500360035C0B300A4
:10805000EB0F4000E08F580001003E0025C0B30048
:1080600062054000E08548003A0F98004B0F9800E9
:108070000FB097009FB097004FB19700DFB1970006
:108080000000410081804900301798004117980096
:108090006FA89700FFA89700020040008380480067
:1080A000A0B79F00B1B79F00700F9800011798000C
:1080B000E3CF52001C003A00D40020000600E0008C
:1080C000E3003A005ED99000C811DD0002002000F4
:1080D0004ED890008080FB0000002000000071005E
:1080E000818071002ED990000281FB008001EB009D
:1080F00002007000838070003ED990004811DD00BE
:108100008001EB000200700083807000101798005F
:10811000211798004258DD00CE50DE00810070002B
:108120004250DD001A003700D40020000600E000B5
:10813000C70032002FB19700BFB197000C0041007B
:108140008D8049001017980021179800E2CF520047
:1081500003003A000A0045008B804D000C003700F8
:1081600032002000030020000A00BE00E5B79F0097
:108170009A040200000000008100D1000080D300BA
:108180006105650000004500E0804800EFB29700FF
:10819000F01FB0000180B000C709DD004900DE001B
:1081A00000807100C908DE00D4002000800F540058
:1081B000818F5C00A60039000080EB008080EB001E
:1081C00070079800010F98006000B80050079800F1
:1081D00061079800E3CF520093003A000040EB00A3
:1081E000504798007ED990004811DD006ED890006D
:1081F0000080FB00020170004FB59700DFB59700CB
:108200000A014100E0814D00120F9800230F9800F1
:10821000E10220008E80400014C0B3001E40900098
:10822000E5B79F0068AA020000000000EFB29700C7
:108230000000E0007C003A00D02220000E00400048
:108240009080FB00C808DD00C02220000E00400026
:108250001080FB008100700050A52A00808F500024
:1082600071003A001E719000C811DD00020020006C
:108270000E7090008080FB00000020000001710063
:10828000818171006E6890000080FB008000EB002F
:1082900000017100818171007E6890004800DD005E
:1082A0008000EB0000017100818171002025250014
:1082B00011162400800F5100818F59005A003A0096
:1082C000502120000E0040001081FB008001EB00D7
:1082D000C811DD0002002000402120000E004000F7
:1082E0001080FB008000EB00C000DD0000002000DB
:1082F0000001710081817100202120000E004000EA
:108300001080FB008000EB00000171008181710092
:10831000302120000E0040001080FB004800DD00EE
:108320008000EB000001710081817100202727008F
:1083300011142600800F5100818F59003A003A0035
:10834000D02120000E0040001081FB008001EB00D6
:10835000C811DD0002002000C02120000E004000F6
:108360001080FB008000EB00C000DD00000020005A
:108370000000710081807100A22120000E014100E7
:108380001281FB008001EB0002007000838070000E
:10839000B22120000E0141001281FB004811DD00D6
:1083A0008001EB000200700083807000500798008D
:1083B00061079800902120000E0040001081FB0012
:1083C0008001EB00C811DD000200200080212000A8
:1083D0000E0040001080FB008000EB00C000DD00BC
:1083E00000002000000071008180710062212000E7
:1083F0000E0141001281FB008001EB0002007000C1
:1084000083807000722120000E0141001281FB0068
:108410004811DD008001EB000200700083807000D5
:1084200070079800010F9800054F78005809EC007C
:10843000C04A8800300798006000B80050179800C4
:10844000611798000040EB00404798000002EB00E5
:10845000040078004F0778004F06BE004F05BE00AD
:108460004F04BE008F01B10000000600000178003B
:10847000EB014100830F5100050032003282FB0006
:108480003180FB0000005200FAFF320000000600BD
:108490000000050080017800F1FF290051417800BB
:1084A0000200FB000204E00002003200830F5000D3
:1084B000FAFF3A0000000600E6874700889FBE00EA
:1084C0008A9FBE008C9FBE008E1F78000105780039
:1084D0009A007800810478008900780031417800A2
:1084E000F3C2B300834F5100FAFF3200C3C5B3009B
:1084F000834F5100F7FF320010047800B2002000D3
:108500000102200008007800C3FC07000901780080
:108510008006EB008000EB008E0020000046EB00A0
:1085200032407800804578008100E80003C2B30043
:10853000834F500034003600EFC14100834F50009C
:1085400031003200C3C5B300834F50002E0032000B
:10855000E3C2B300834F5000020032008E8F5600FA
:108560000A003900E80F570045003A00E3C2B300A3
:10857000834F500042003A00200020000066DD00DA
:108580008E067800BE002000E5FF37000004E00002
:1085900005003D003C40B3008085FB000B08B100A6
:1085A000F0002A00E0C57D000B80FB00F1B79F00C2
:1085B00082BF9F00B7FF0700FFB097000FB9970079
:1085C0000000E0002E003A00F0CBB30000C04500F0
:1085D000F94F500002003E000C14A00007003700C5
:1085E000F0C9B30000C04500F94F500003003E0041
:1085F0000C04A00000CEB30080C545000BF47E0043
:108600008D06E800C6FF3700018D44008040EB0076
:1086100002C2B300824F500001003E0041C0B300CF
:10862000600020000D00E0001600320050CEB300C4
:10863000984F100002003A0050C0B300004C780080
:10864000E80F570002003A00200020000066DD001D
:108650000C86FB0063006600E10F500001003A0049
:108660000144A0006C066600E40F560001003A00C9
:108670000134A000314C98000000EB0001003700ED
:10868000600020004F0778004F06BE004F05BE0077
:108690004F04BE006F00B10000000600881F780084
:1086A0000004780062005100E0805900380A900010
:1086B000C80A900062025200E0825A006011B800BD
:1086C000840F5000858F5800090031002841900028
:1086D0000281FB008001EB009A0402000000000010
:1086E00038119000C81190000001410081814900BB
:1086F0000200BE004F04780000000600889FBE0004
:108700008A9FBE008C9FBE008E1F780000047800F8
:108710000206BE001A0020000B002000E10F5100ED
:10872000E08F59007A00360038089000C8089000A1
:10873000800F5100818F590075003100184078007A
:10874000E24F50002F003200E34F5000450032004E
:108750000085EB008085EB00E14F50006C003A0093
:108760008204D100828444004949DE0078089000E8
:108770008810900000014100E08148000800780066
:108780002BFC07000085EB008085EB000000E0007B
:108790005F003A0009007800F01FB200E002B0006C
:1087A000684778008904E8004949DE0078089000AD
:1087B0008810900000014100E08148000800780026
:1087C0001BFC07000000E00051003A000E87FB0090
:1087D000F91FB200E902B00068C57C004855DD0011
:1087E0000A0577000C08A300020032004455DE00A1
:1087F00002003700FEFF20000E0565008005EB003B
:10880000430037004818DD004811DE000201700007
:10881000C819DE007808900088109000020140001E
:10882000838148000800780001FC07000085EB0008
:108830008085EB000000E00035003A000C064600A1
:10884000FC1FB200EC02B00068457E000A85FB0008
:108850000C0644001C4090004800DD000A05700032
:10886000E6FF37004918DD004711DE000201700005
:10887000C719DE00780890008810900002014000BF
:108880008381480008007800E9FB07000085EB00C1
:108890008085EB000000E0001D003A004266DD002C
:1088A000FC1FB200EC02B0000C004400204190001C
:1088B0000281FB008001EB00C012DD0004002000FB
:1088C00030419000C811DD0002002000020172005A
:1088D00083817200104090004800DD008000EB00B2
:1088E000000171008181710068407E000080FB0002
:1088F0008000EB000001710081817100F0FF200019
:108900000300600080007800020078000005BE00CF
:108910000A00BE004F0778004F06BE004F05BE009C
:108920004F04BE0000000600881F78000004780095
:108930000000EB002004980038019000C80190006E
:1089400020002000E10F5100E08F59003E0032006E
:1089500098007800310A9000C10A9000840F5100FD
:10896000858F590038003100E00F5100E08F590029
:1089700014003A0030C0B300914F100005003A00D7
:1089800011119000A1119000E00F5100E08F5900EB
:108990000C003A006011B80052049800630498007B
:1089A00041019000200020000200E000260032007B
:1089B00011119000A111900072049800030C98000E
:1089C00019003700214090000004E00010003A0038
:1089D0001800780049FF07000001BE00E10F4000C9
:1089E000E08F480015003200E10F5000E08F580082
:1089F0001400360018007800C0089000300890007D
:108A0000800F5100818F5900F1FF39000D003700B0
:108A10005204980063049800010078001FFF0700CB
:108A200070049800010C9800E302200018804100B7
:108A3000100C98000000EB0003003700100020002D
:108A400001003700200020004F04780000000600DD
:108A50000800FA00889FBE008A9FBE008C9FBE005F
:108A6000000478000205BE000406BE0020002000BD
:108A7000E10F5100E08F5900A50036003809900041
:108A8000C8099000820F5500838F5D00A00031005F
:108A900098407800E2CF500040003200E3CF500011
:108AA00052003200E1CF500097003A008A04D10012
:108AB0008A8444004949DE007808900088109000BC
:108AC00000014100E08148000800780058FB0700E1
:108AD0000000E0008C003A0089007800F11FB2002D
:108AE0006105650008003200E0022000010040003E
:108AF000684178006F4161000C80FB004400DD009C
:108B000000407100010037000C40780081004400F3
:108B1000E06898008904E80010C0B3004044980061
:108B20004949DE007808900088109000000141005B
:108B3000E0814800080078003DFB07000000E000ED
:108B400071003A00F91FB2000A00E000050032008F
:108B5000CC68DD004466DE000C867000C46EDE006A
:108B60000B003700E10220008980400068C17800D6
:108B700001CFB300814061004869DD004866DE0036
:108B80000C067100C86EDE006F4666000CC67000F1
:108B900089044400EC6C98005B003700485BDD0002
:108BA0004851DE0002017300C859DE0078089000C9
:108BB000881090000201400083814800080078007E
:108BC0001BFB07000000E0004F003A000A054500CB
:108BD000FA1FB2008A004400EC6898000105780092
:108BE0004866DE007C6D980047003700C95BDD00F9
:108BF0004751DE0002817300C759DE0078089000FB
:108C0000881090000201400083814800080078002D
:108C100007FB07000000E0003B003A004255DD0082
:108C2000FA1FB200E90220008A844400890044004F
:108C3000638240008182E8001581FB008001EB0027
:108C4000C013DD0006002000E6B79F00F7B79F00C5
:108C50001481FB008001EB00C813DD00060020003A
:108C600086BF9F0097BF9F006FB19700FFB197002D
:108C70000601710087817100E2B79F00F3B79F0082
:108C80005183FB004833DD006131B80082BF9F0093
:108C900093BF9F006FB39700FFB397000203730069
:108CA00083837300E6B79F00F7B79F0068C17C001D
:108CB0000283FB008003EB006FB19700FFB19700C8
:108CC000060371008783710002002F000701610015
:108CD0008001EB00C011DD00020020000C067100D5
:108CE0008D8671000A0544006C6D98004861DE00B5
:108CF000824878004069DE0003002000824A780044
:108D0000486EDE000C4A780011C0B3004144980060
:108D10004F06BE004F05BE004F04BE000080FA00A3
:108D2000000006000400FA00889FBE008A9FBE0073
:108D30008C1F7800000678000204BE00E00F51008E
:108D4000E08F59000B003A005C029000EC029000AA
:108D5000E00F5200E08F5A00120032003C089000F1
:108D6000CC089000800F5200818F5A000D00310016
:108D70000E0037000C00780060FE0700E10F500085
:108D8000E08F5800510036003C099000CC0990005B
:108D9000820F5000838F5800520039000802BE0035
:108DA0000200370014002000050020000405BE006A
:108DB00061054500E0854D003C089000CC0890001E
:108DC000800F5500818F5D0005003900E10F5200D2
:108DD000E08F5A00400036002A0020000B002000DF
:108DE0000A01BE000C00780094BF9F00A5BF9F0041
:108DF00042FE07001FBA9700AFBA9700E00F50007D
:108E0000E08F58000A003200E10F4000E08F480078
:108E100034003200E10F5000E08F58003100320082
:108E2000840F5500858F5D00E1FF3A002A0037006E
:108E3000F4FF2F00F5FF20000A01BE000C007800AF
:108E400003FF0700000178000200E00018003A006C
:108E5000E00F5400E08F5C00070032000A02BE0001
:108E60000801BE000C007800F9FE07000001780040
:108E70000200E0000E003A005A0698006B069800C7
:108E80007C0090008C089000E10F4000E08F4800CB
:108E90001300320061005000E08058007006980016
:108EA000010E980010C0B300504698000C00370027
:108EB0001000200001002000E10F510009003A00DD
:108EC0000080EB008080EB000600370010002000DF
:108ED00001002000030037006000B80001003700E7
:108EE0000A00BE004F0678004F05BE004F04BE00CA
:108EF0000080FA0000000600889FBE008A9FBE0026
:108F00008C9FBE008E1F78000004780081067800D8
:108F1000A80490008904E8004E0020007B00320085
:108F20007800900088089000E00F5000E08F580013
:108F3000760032006F8664006B003A0061004000EA
:108F4000E080480070049800010C980058019000DF
:108F5000E801900018007800E00F5100E08F590000
:108F600004003A0040009000808F54005E003900F9
:108F700066003700A04090008180FB008100E9007E
:108F8000444ADE008480600057003A00DBFD0700A1
:108F90000005BE002E002000E10F5000E08F5800B9
:108FA0005A0036001E002000E10F4000E08F48000C
:108FB000560032001800780030099000C009900077
:108FC000820F5500838F5D00400039004E00200065
:108FD0000D00E0004D00320058019000E8019000C3
:108FE00050FF07000005BE007E002000E00F50008B
:108FF000E08F5800450032002E002000E10F5000A5
:10900000E08F5800410032001E002000E10F4000B8
:10901000E08F48003D0032006011B8001800780071
:1090200003FA07000000E00038003A00E1022000E7
:1090300018804000022020008000EB00F6F90700B5
:10904000980678000A01BE000D00780093FD070025
:10905000D0169800E11698008046EB000F0037000C
:1090600011C0B300414098006011B80018007800AA
:10907000EFF907000000E00023003A001800780034
:1090800050119000E011900061014100E081490021
:1090900052109800631098008D46E8001800780080
:1090A000A040900081CF5600EDFF39000D81FB00FC
:1090B0008001EB0050129000E0129000020152007B
:1090C00083815A0052109800631098005A04980047
:1090D0006B0498000A01BE00180078006FFD0700BD
:1090E00070049800010C980029049800E102200007
:1090F000188040004566DD000C0640001C0C9800FE
:109100000007EB00010037001E0020000E00780071
:109110004F0778004F06BE004F05BE004F04BE004B
:1091200000000600889FBE00000478000800780058
:10913000FDFD0700800478000900E00016003A00F9
:10914000780190008809900018007800B8F90700AD
:10915000800478000900E0000F003A001808900031
:109160001004E0000B003200B04890000138A3006A
:1091700004003A00A8089000BCFC07000000E000D2
:10918000050032008000EB00080078005AFF07005D
:10919000E8FF370049002000090078004F04BE00B6
:1091A000000006000200FA00881F78000004780022
:1091B000E1BF9F0011407800F2C2B300824F50001F
:1091C00003003200C2C5B300824F500002003A00D3
:1091D0008100E800E1BF9F006000B8003004980003
:1091E000410498006FB89700F1C1B30090CF100010
:1091F00005003E0008007800CBFD07008000EB0072
:10920000110C98002A00370074004400E4805700D5
:10921000A9FC07000000E00025003A0008007800E3
:10922000C0FF0700A8089000B14890000000E000CF
:1092300005003200E40F50001D003A000128A30091
:109240001A0032001A0037000128A30018003A0063
:1092500018089000B04890000148A30013003200A5
:10926000505290004822DD00C05090008180FB00E9
:10927000048270008002EB00C022DD0004002000A8
:10928000305990004811DD00205890000080FB000C
:10929000020170008001EB00020072008380720006
:1092A0003004980041049800D7FF37005000200098
:1092B0004F0478000080FA0000000600889FBE007E
:1092C0008A1F7800000478000800780096FD0700E7
:1092D000800478000900E0001D003A007801900049
:1092E000880990001800780051F907008004780080
:1092F0000900E00016003A001808900010407800BD
:10930000FB4F4000160032000004E0001400320061
:109310001100200008007800F7FE0700ECFF37007E
:10932000180D9000020220008000EB000A00780077
:1093300039F90700B2002000A80890000A00780060
:109340002FF907001800780011C0B30041409800C1
:10935000090078004F0578004F04BE0000000600A9
:1093600078019000880990001800780030F9070013
:10937000800478000900E000F5FF3A00E8FF3700BC
:10938000881F78008A9FBE008C9FBE000004780072
:109390000205BE0020002000E10F5100E08F5900BF
:1093A0002F00360038099000C8099000820F550040
:1093B000838F5D0020003900290037000A01BE00BC
:1093C00008007800CDFC07000006BE00E00F50004A
:1093D000E08F58001D003200E10F5000E08F580070
:1093E0001C003200E10F4000E08F48001B003200FB
:1093F0006022B8000A01BE000800780094FD070052
:109400000000E00016003A00780090008808900004
:10941000E10F4000E08F480006003200610040008C
:10942000E080480070049800010C980010C0B30060
:10943000504498000C05BE0038089000C808900001
:10944000800F5500818F5D00DCFF39000000EB00CC
:10945000030037002000200001003700100020002A
:109460004F06BE004F05BE004F0478000000060006
:10947000B20020000004E00009003A00B04A800079
:109480000000E000010032000048EB000100E000B5
:10949000010032008048EB00B14A88000001EB0077
:1094A00002007800000006002800FA00889FBE0035
:1094B0008A1F78008C9FBE008004780081BF9F00C7
:1094C000800CEB007F4561007E416100A1FD2F0013
:1094D0008F80400070805700F0F90700E1FC2F00FA
:1094E0008F804000F1B79F000000E00004003A00C8
:1094F0008FB89700A0FD2F000F00400029FF070044
:109500006FB497000000E00003003A000800E0009C
:1095100001003A00600020008A80FB007C8160002E
:10952000550032000000E0000A003200E40F500055
:1095300003003A00A0FD2F000F0040005FFF07006E
:109540006FB497000000E00092003A000A34A000D7
:109550000700370038499000710161007000200059
:109560008C003A00800020000128A30089003A0006
:109570000A38A3004C0032000EB2020000000000C6
:10958000604C98004801DE00724C98004009DE00F3
:1095900003002000025498004808DE001054980090
:1095A0000040EB00304C9800405C9800505C980004
:1095B000605C9800705C980075004400F400440002
:1095C0007B014400FA0144001086FB004866DD0080
:1095D0001182FB000C0672008006EB00C066DD0005
:1095E0000C0020001282FB004822DD009382FB0069
:1095F000048272008002EB00040676008586760005
:109600008049EB000049EB008048EB000048EB008C
:109610005FA8970011C0B30041409800E00F5600CA
:10962000E08F5E002000320050129000E0129000A7
:109630000C01BE0094BF9F00A5BF9F0050FF070014
:109640001FBA9700AFBA97000000E00051003A003F
:109650005FA8970061065600E0865E005C009800F7
:109660006D0098000401BE0071F807000000E000E2
:109670000D003200470037000000E00045003A00CE
:10968000384990000281FB00400020000248A300FE
:1096900040003A000118A3000300320070002000CF
:1096A0000208A3003B003A000A38A3000100320080
:1096B0000A54A0005FA8970050119000E01190009C
:1096C000D20C9800E30C9800F80C9800CA4498005B
:1096D000585190004811DD00C85090008180FB0077
:1096E000028170008001EB00C011DD00020020004B
:1096F000385A90004822DD00A85890008180FB0075
:10970000048270008002EB00040171008581710009
:10971000F2049800830C9800785990000281FB00B5
:109720008001EB00C812DD000400200068599000A1
:109730008281FB000200200002017200838172001E
:10974000485A90000482FB008002EB000401710083
:1097500085817100585A90004822DD008002EB009C
:109760000401710085817100D2049800E30498001F
:109770006011B800B2049800C3049800B20C9800BD
:10978000C30C9800800C7800300090009004980082
:109790000000EB004F06BE004F0578004F04BE00EE
:1097A0000080FA0000000600E6874700889FBE00A0
:1097B0008A9FBE008C9FBE008E1F78000004780038
:1097C0000107780082047800F3B79F000300780057
:1097D0000008EB009800900018007800B1F807002E
:1097E0000000E000AF003A00C840900020002000D8
:1097F0000104E000AB003500700020000108A30068
:10980000A800320058019000E80190003800900054
:10981000C800900000005100818059006149B800E3
:10982000800F5100818F59009B0036008004780022
:109830009900370038019000C801900002007800BC
:10984000F01FB2007A003A0018007800C91BDE0051
:10985000C718DD004913DE00068370002042900027
:109860000442E9000642620013003A00E00F510092
:10987000E08F590003003A007800900088089000BB
:109880000500370018099000A809900084BF9F00C8
:109890009AFB07000FBA9700E10F5000E08F5800C5
:1098A0000F003600E10F4000E08F48005900320001
:1098B000100C9800210C9800980578001809900069
:1098C000A80990000B00780084BF9F0073FB07007D
:1098D0000FBA9700E00F5000E08F580005003A00E3
:1098E000484090000074A0004044980020002000F0
:1098F0006C0037000486FB008006EB000006460083
:1099000081864E00494DDE00220032002B4090003F
:109910000482FB00840045000080FB00808F500023
:1099200001003600040550000A4278000C01BE0018
:109930008E0078001B40900068AA02000000000022
:10994000C84090000000E00023003A000168A30036
:109950000E00320038089000C80890000C06500035
:109960008D8658006150B800800F5600818F5E00D0
:109970000600310001022000888040004960DD00BF
:1099800000004700022020009DF707004955DD0038
:109990003700370038099000C80990008C0F51003B
:1099A0008D8F590020003200484090000068A300CD
:1099B0000E003200010220008880400014C0B30075
:1099C0001B409000D8AA020000000000C840900090
:1099D0000000E000030032000174A0004144980040
:1099E0000F0037000164A1004144980001022000EB
:1099F000888040001800780014C0B3000C01BE003D
:109A00001040900068AA0200000000000000E00082
:109A100005003200484090000074A00040449800C7
:109A2000100020001F0037003C0C98004D0C9800DF
:109A300038009000C800900080007800F11FB2004C
:109A4000002020000100500009057800808F54009C
:109A500001003600000578000002200008004000E8
:109A6000810040000A0178000E00780064F70700CA
:109A70000A07470038009000C80090000000450029
:109A8000E080480030049800410498007FB09700BF
:109A9000100845008A8454000900E00065FF3A0080
:109AA0000000EB004F0778004F06BE004F05BE00D8
:109AB0004F04BE006F00B10000000600E6874700BB
:109AC000889FBE008A9FBE008C9FBE008E1F7800BC
:109AD000000478000107780082047800F3B79F0043
:109AE000030078000008EB00980090001800780050
:109AF000ECF707000000E000D0003A00C8409000FA
:109B0000200020000104E000CC003500700020009F
:109B10000118A300C900320058009000E80090002E
:109B200000814400E0814800800F5100818F59007E
:109B3000B30031008004EB00B10037003801900021
:109B4000C801900002007800F01FB20090003A00B7
:109B500098007800C91ADE004718DD004912DE00BF
:109B600004027000214090000040E90004406000C1
:109B700080F79F0020003A00E00F5100E08F59006D
:109B80000C003A007801900088099000E00F510025
:109B9000E08F59000F003A006011B8000100780012
:109BA00060FC07000001BE0070049800010C9800E2
:109BB0000500370018099000A809900001007800FE
:109BC00058FC07000001BE00E00F5100E08F590073
:109BD0008D00320048409000E10F5100E08F5900A5
:109BE00022003200E10F4100E08F490062003200A4
:109BF000120C9800230C9800484090000068A300C5
:109C00001100320001022000888040001800780016
:109C100014C0B30038099000C809900010409000AB
:109C2000D8AA020000000000C84090000000E00038
:109C3000030032000174A000414498005000370036
:109C40000164A1004144980098057800180990002B
:109C5000A80990000B00780090FA0700E00F500070
:109C6000E08F580005003A00484090000074A000C2
:109C70004044980020002000700037000FF197004A
:109C80000286FB008006EB000006460081864E003F
:109C9000494DDE0022003200AB4090000280FB0004
:109CA000000145008180FB00810F5100010036005A
:109CB000008550000A4278000C01BE008E0078003A
:109CC0001B409000D8AA0200000000000000E00045
:109CD00028003A0038089000C80890000C06500090
:109CE0008D8658006150B800800F5600818F5E004D
:109CF00009003100C960DD0081004700000220003A
:109D00000800400002202000BDF6070048409000F7
:109D10000064A100404498004955DD002E00370042
:109D200038089000C80890008C0F50008D8F5800A4
:109D30001500320038019000C801900058009000D2
:109D4000E8009000800F5100818F59000E00310013
:109D5000010220008880400014C0B3000C01BE0046
:109D60001B40900068AA0200000000000000E00014
:109D700005003200484090000074A0004044980064
:109D8000100020002D0037003C0C98004D0C98006E
:109D900038009000C8009000F01FB20001202000A1
:109DA0008080500009057800818F54000100360042
:109DB00001057800010220008880400000804000FA
:109DC0000A0178008E0078008DF607004840900068
:109DD0000064A000404498000A0747003800900043
:109DE000C800900000004500E08048003004980062
:109DF000410498007FB09700100845008A84540001
:109E00000900E0004DFF3A0038009000C8009000C3
:109E100058019000E8019000820F5000838F580095
:109E200002003600500498006104980048409000F9
:109E30000054A000404498000000EB004F07780059
:109E40004F06BE004F05BE004F04BE006F00B100BC
:109E500000000600889FBE00000478009800900073
:109E6000180078000FF707000000E00041003A00FA
:109E7000C84090008180FB000158A3003D003200E3
:109E80000168A30010003200010220008880400019
:109E90001800780014C0B30038099000C809900079
:109EA00010409000D8AA0200000000008000780056
:109EB000100020000100E0002E003A004840900011
:109EC0000064A1004044980058099000E8099000FF
:109ED0001800780056F607000000E00025003A0060
:109EE000F80C90006B8044001054A00028489000AB
:109EF000C05C980038489000D05C980048489000BA
:109F0000E05C980058489000F05C98006848900029
:109F1000A05C980078489000B05C980008509000D1
:109F2000C054980018509000D05498000EB202000F
:109F300000000000E05498004801DE00F254980050
:109F40004009DE0003002000825C98004808DE0023
:109F5000905C9800484090000054A1004044980054
:109F60001800780011C0B300414098001800780034
:109F7000DDF607004F04BE0000000600881F7800D1
:109F80000004780008007800B2FF07000000E0003D
:109F900001003A00000C78004F0478000000060031
:109FA000EA874700889FBE008A9FBE008C9FBE0044
:109FB0008E1F7800000778000202BE009E0090000D
:109FC0001E007800F2B79F0085BF9F00B5F607001E
:109FD000D0B79F007FB297008FBA97000000E000D3
:109FE000F0003A004E4190000204E000EB00350022
:109FF0005E009000EE009000800F5200818F5A00AA
:10A00000030036000218A30001003A000002BE005F
:10A010003E009000CE0090006011B800320798001A
:10A02000430798006044B800E00F5200E08F5A00E8
:10A03000A00032001E037800264190000281FB0040
:10A040008001EB00491DDD00C715DE008B057500A2
:10A050004915DD00E00F5000E08F5800230032006A
:10A0600061045000E084580061005200E0805A0012
:10A070000A01BE00F4B79F0085BF9F00E6B79F00AE
:10A080007A040200000000000006BE000A01BE00C3
:10A090000800BE007A040200000000007FB29700B2
:10A0A0008FBA97006FB39700800F5600818F5E00C4
:10A0B0000E00390060001500E0801D000003640000
:10A0C0000181640082017800060178000200BE0070
:10A0D00030079800410798000002520081825A0020
:10A0E0001E099000AE099000170037007E01900015
:10A0F0008E099000E00F5100E08F590010003A00E7
:10A100006011B80006007800F4B79F0085BF9F007B
:10A1100004FB07000001BE007FB297008FBA9700D2
:10A12000E10F5000E08F580058003200E10F40006E
:10A13000E08F48008400320070079800010F9800FB
:10A14000120F9800230F98006044B800E00F5100F0
:10A15000E08F590057003200340037004E40900025
:10A160000018A3000B0032001E007800F4B79F0017
:10A1700085BF9F00EBFA07000001BE007FB2970089
:10A180008FBA9700E00F5000E08F580008003A00A7
:10A190002A0037001E007800F4B79F0085BF9F009B
:10A1A00056F907000001BE008FBA97007FB29700F2
:10A1B000E10F4100E08F490004003A004E4090005A
:10A1C0000074A0004047980051003700E10F510093
:10A1D000E08F5900060036001E007800C00890008D
:10A1E00030089000800F5100818F59000500390020
:10A1F0004E4090000074A0004047980022002000CC
:10A2000055003700120F9800230F98003E00900071
:10A21000CE0090000000450081804D00300798007E
:10A22000410798000A0252008B825A008A0F52009E
:10A230008B8F5A00C9FF3E00010037000A02BE00A2
:10A240003E009000CE0090000000420081804A0055
:10A25000300798004107980004007800F01FB20012
:10A260006044B800130032001E007800F4B79F006D
:10A2700085BF9F0009F907007FB297008FBA97004A
:10A28000E00F5000E08F580004003A004E4090006C
:10A290000074A0004047980040003700C92CDE0041
:10A2A0004729DD004924DE00080471000004440051
:10A2B00081844C003E009000F01FB2002A00320062
:10A2C0003E099000CE099000820F5400838F5C00FD
:10A2D000250032004E4090000068A30010003200BC
:10A2E000010220008E8040001E00780014C0B300E0
:10A2F00010409000D8AA020000000000CE4090005C
:10A300000000E000040032000174A0004147980002
:10A3100010002000220037000164A100414798008E
:10A32000010220008E8040001E00780014C0B3009F
:10A330000801BE001040900068AA02000000000062
:10A340000000E000060032004E4090000074A000C3
:10A350004047980012002000D2B79F00110037003C
:10A36000380F9800490F98003E009000CE009000F2
:10A370005E019000EE019000820F5000838F580024
:10A380000800360050079800610798004E40900082
:10A390000054A00040479800020037002000200031
:10A3A000D0B79F005FB097004F0778004F06BE0000
:10A3B0004F05BE004F04BE00AF00B1000000060014
:10A3C000FF4F500002003E0080407800060037003A
:10A3D0008040EB00F2C3B300824F500002003E0009
:10A3E00001C4B30080C050000140780000000600A6
:10A3F000889FBE008A1F7800800478005A48EC00CD
:10A400005AE8B70001C6B300814F50000100360082
:10A410005A68EF005AC8BF00804C780009047800E1
:10A4200002C2B30082404000016C780002C6B30053
:10A4300082CF50000100360002CC50000985E800B0
:10A440000044B000004D780001C6B300814F5000B9
:10A4500001003600014D500019407800D8FF070078
:10A46000804C780018407800D5FF0700004C780039
:10A470001A407800D2FF0700004D78004F057800A1
:10A480004F04BE0000000600800078000000EB00D2
:10A49000E48F50000A003200E88F500008003200BC
:10A4A000100020000100E00005003A00704280002A
:10A4B00000F0A7000000EA000000EA004F00DE0004
:10A4C00000000600889FBE000004BE00090444008E
:10A4D0000100370069045400E80F5400FDFF3C0000
:10A4E00001003700690444000800E000FDFF35006A
:10A4F00008007800E4FF07000000E000F3FF3200EE
:10A50000080078004F04BE00000006008000EB0049
:10A51000E80F5000E08F58002B003E000060010063
:10A5200008003700090037000B0037000E00370025
:10A5300011003700130037001500370018003700EE
:10A540001C0037000041EB000C0037000041EB001D
:10A5500001C2B300140037000041EB0001C2B30098
:10A5600001407800110037000041EB008240780084
:10A5700000C2B3000D00370002C2B3008240780071
:10A58000F7FF370002C2B3008040EB00F4FF370052
:10A5900002C2B300824078000040EB0003003700A5
:10A5A00002C2B3008040EB00024078000AC70400FA
:10A5B0000000000052C0B300F1C0B30000C2B300FD
:10A5C0000AC702000000000000000600889FBE00CD
:10A5D0000004780008007800CCFF07008004EB003E
:10A5E000E80F5400E08F5C003D003E000860010071
:10A5F0000800370009003700360037000D0037002B
:10A6000034003700170037001F0037002F003700D5
:10A6100030003700000021002F00370040002000EC
:10A620006C740200000000007EB102000000000017
:10A630002B003700001020006C74020000000000A6
:10A64000400020006C740200000000000041EB009C
:10A6500082407800F0C0B3000AC70200000000008A
:10A660001F003700400020006C7402000000000052
:10A67000000120006C74020000000000600F200048
:10A68000A094880016003700E0252A00B6B4020026
:10A69000000000000000E0000E003A002100200051
:10A6A000408D200044B50200000000002100200081
:10A6B000608D200044B50200000000000000EB00A7
:10A6C000B6B4020000000000020037005228EF007C
:10A6D0005428EF00400020006C74020000000000CD
:10A6E0004F04BE00000006000400FA00889FBE0070
:10A6F000000478000001EB006000B800AEC7020063
:10A70000000000008043EB00074378008742780098
:10A710000742780087417800074178008740780039
:10A7200007407800BAC60200000000008040EB003D
:10A7300000C1B300DAC50200000000008040EB0059
:10A7400010C1B300DAC50200000000008040EB0039
:10A7500040C1B300DAC50200000000008040EB00F9
:10A7600050C1B300DAC50200000000008040EB00D9
:10A7700020C1B300DAC50200000000008040EB00F9
:10A7800030C1B300DAC50200000000008040EB00D9
:10A7900060C1B300DAC50200000000008040EB0099
:10A7A00070C1B300DAC50200000000008040EB0079
:10A7B00001407800DAC50200000000008040EB0094
:10A7C00010C0B300DAC50200000000008004EB00F6
:10A7D000E80F5400E08F5C0054003E000860010068
:10A7E00008003700090037000E0037000A00370064
:10A7F0004B0037000F0037002200370044003700BD
:10A8000047003700000021004600370088B10200F1
:10A8100000000000030037000010200084740200D4
:10A8200000000000400020008474020000000000CE
:10A830000F00370040002000847402000000000078
:10A840000001200084740200000000008040EB0042
:10A85000E0C1B300DAC50200000000004029210079
:10A860000008EB00F1BF2F0020932000108860004B
:10A87000202721000008EB000080E8000008EB0022
:10A880002A003700E0252A00B6B4020000000000CC
:10A890000000E0001E003A00C0BF9F00D0BF9F0034
:10A8A000210020006880570044B50200000000002D
:10A8B000210020006680570044B50200000000001F
:10A8C0004FB89700D408E30003003A005FB8970040
:10A8D000D608E3000B0032006000B80004B50200A7
:10A8E0000000000021002000408D20008AB50200F9
:10A8F0000000000021002000608D20008AB50200C9
:10A90000000000000000EB00B6B4020000000000F0
:10A91000202721000008EB000080E8000008EB0081
:10A920004000200084740200000000004F04BE00BC
:10A930000080FA00000006006448EC0080407800C7
:10A9400042862000014978000100FB000104E0007C
:10A950000700340082C2B30082CF500008003400E8
:10A9600001C8B300428620000149780000000600BB
:10A9700042002000110009000200D8000000EA0097
:10A98000000006000400FA00889FBE008A9FBE00F7
:10A99000C8918000812321000005EB0010002000F9
:10A9A00051017800880F5100020034000005780042
:10A9B000020478000000E800E50F5000F8FF3A00BC
:10A9C000C446800062051500220020001100090025
:10A9D0000202D8008000FD0001D5B900C9DA2000CC
:10A9E000890F54000A00340001FA2000810F54003E
:10A9F00005003C0088845400110009008204D8003E
:10AA0000800478000F0037008404EA000D0037004E
:10AA100071BB2000810F540000013C00813EB10059
:10AA2000810F54000900340089C12F00888444003C
:10AA300092FF2F00110009008204D80080047800E2
:10AA4000C912B000848F54000100340084047800DF
:10AA50008400EA00818F540001003D0081047800E9
:10AA6000311F2000810F54000A003C005848E200CA
:10AA70000300320094938800A493880009003700F3
:10AA8000202721000008EB000080E8000008EB0010
:10AA900004003700402721000A8844000080E900B4
:10AAA0000A8854005848E200140034005948E20073
:10AAB000120032006C8057004DFE07006FF19700C6
:10AAC000DFF097004FF097000AC702000000000077
:10AAD0005FF19700CFF097006FF0970042C7020038
:10AAE000000000004FF19700EFF097005FF0970033
:10AAF00026C7020000000000060037008EFF070096
:10AB00000001EB00800078000000EB00AEC70200FF
:10AB1000000000005848E2001600320057C8BF008D
:10AB2000DA48B40057E8B700FE4F50000200360084
:10AB3000DAE8EF00040037000004E00002003A0009
:10AB400010C0B300DAE8B7007585200095427800A0
:10AB50008580FB004309DE00C408DE0081437800E5
:10AB60000243780004C2B300854178000040EB0046
:10AB7000080037008043EB000743780005C2B300AC
:10AB800005427800854178000741780087407800C9
:10AB900007407800BAC602000000000030FC220026
:10ABA0009080FB008100EA00CF08DE000000EB008F
:10ABB0000104E000040032009AC8BF000080FB00DE
:10ABC0000000E9004F00DE00A28920000149780062
:10ABD0000000E00007003200C14680002103B00001
:10ABE000C1468800401F2000808F500001003400C3
:10ABF000C046880000FC22009080FB008100EA0033
:10AC0000CF08DE000000EB000104E0000400320089
:10AC100099C8BF000080FB000000E9004F00DE0083
:10AC200092892000014978000000E000070032000E
:10AC3000C14680002103B100C146880040ED2F00CD
:10AC4000808F500001003D00C046880011C0B30055
:10AC5000401F2000800F540003003C008040EB00A8
:10AC60000000EB000400370098C8BF000080FB0024
:10AC70000000E9004F00DE008289200001497800D1
:10AC80000000E000030032006000200000E102004C
:10AC9000000000000A00E0000D003A000900E0009A
:10ACA00060003A005948E2005E003A00401F200070
:10ACB000800F54005B00340010C0B30059E8B700A7
:10ACC0007000200000E102000000000001003700D9
:10ACD0005968EF001008200071938000808F5000A9
:10ACE0000300340081938000808F50000A003C00F4
:10ACF000202721000008EB000080E8000008EB009E
:10AD000001C2B30080C0B300DAC502000000000039
:10AD100001C2B300050037008040EB0080C0B300E3
:10AD2000DAC50200000000008040EB00B0C0B300B4
:10AD3000DAC502000000000058C8BF00020032005F
:10AD40000040E90058E8B70032E9AB0039003200B2
:10AD5000F1F72F0020932000108860005868EF0062
:10AD600042252100A19280000009EB000004EB00C5
:10AD700010002000D2017800818F510002003400C1
:10AD800000047800830078000009EB000000E80070
:10AD9000E70F5000F7FF3A0080BB2000808F500083
:10ADA0002400340028938800202621001000E900A8
:10ADB000E20F50001F003E00080078000010A200C3
:10ADC00000F0A7000000EA000000E9004F00DE00EC
:10ADD0008000EB000004E0000500320071892000D3
:10ADE000914078008180FB008100E900CF08DE00FF
:10ADF00097E8B7000100E000030032007000200077
:10AE000000E1020000000000E20F540009003A00D7
:10AE100060C0B30058E8B700060037008004EB00BC
:10AE200008FF3700301F2000800F5400A8FF3400B7
:10AE3000A8FF37004F05BE004F04BE000080FA0097
:10AE4000000006000C00FA00889FBE008A9FBE002A
:10AE50008C9FBE0078805700030009000018EB00AB
:10AE6000B5FE07000041EB00804078000AC70200F1
:10AE7000000000005BC8EC005BE8B7008080FB00CE
:10AE8000C508DE0002C2B300F881570082F17800E5
:10AE90007F4060008101E900E781610000415100CD
:10AEA00002437800F882570086F279008100E800BA
:10AEB000E78060000041780082F27800FFEB9700A5
:10AEC0006FEB9700DFEA97004FEA9700BFE9970022
:10AED0002FE997009FE897000FE89700BAC6020095
:10AEE0000000000030FC22009080FB008100EA009E
:10AEF000CF08DE000000EB000104E0000400320097
:10AF00009CC8BF000080FB000000E9004F00DE008D
:10AF1000C3892000814978000000E000070032006A
:10AF2000E14680002103B000E1468800401F200078
:10AF3000808F500001003400E046880000FC2200B1
:10AF40009080FB008100EA00CF08DE000000EB00EB
:10AF50000104E000040032009BC8BF000080FB0039
:10AF60000000E9004F00DE00B5892000814A78002A
:10AF70000000E00007003200E14680002103B1003C
:10AF8000E146880040ED2F00808F500001003D0019
:10AF9000E0468800E84680000800E00055003500E3
:10AFA000C3918000D1918000F091800002928000D6
:10AFB000611AB9004F93DE000402410085024B0084
:10AFC000018640004FE3DE000402460085024B008C
:10AFD000EC9180006366B9004FE3DE000406460092
:10AFE00085064B0000024000CFA2DE000C064200A6
:10AFF0008D864A00D6FF2F00068BB900C1FF2F00B7
:10B00000019AB900CFA2DE00CFB0DE0004024300F7
:10B01000858248006300B900CF81DE000400400053
:10B02000858049004212DD004FA3DE00000242008D
:10B0300081024B000400460085804E006145B90046
:10B040000A01BE0084BF9F0095BF9F009A040200C2
:10B05000000000000001BE00097D20001100090071
:10B060004919D800800078002027210001085400E9
:10B070000FBA97009FBA97000400560085805E00C3
:10B080000A01BE009A040200000000000001BE0098
:10B09000110009004919D8008004780009045400FF
:10B0A000A893880080DA2F0091938000808F500051
:10B0B00001003D0090938800800F540002003D0085
:10B0C00080DA2F00A09388008025200091938000D3
:10B0D000808F50000100340090938800802520006C
:10B0E000A1938000808F500011003400A09388004D
:10B0F0000F003700209280000882B90042ED2F0037
:10B1000011000900422AD800800078002027210081
:10B1100008884000109280000882B90011000900E0
:10B12000422AD80000017800402721000808410089
:10B130001008200071938000808F500003003400BD
:10B1400081938000808F50000A003C00202721005E
:10B150000008EB000080E8000008EB0001C2B3002B
:10B1600080C0B300DAC502000000000001C2B300D5
:10B17000050037008040EB0080C0B300DAC5020054
:10B18000000000008040EB00B0C0B300DAC5020050
:10B19000000000004F06BE004F05BE004F04BE0079
:10B1A0000080FA0000000600889FBE008A9FBE0053
:10B1B000F046800080004000808040003094800095
:10B1C00000F0A7000000EA0080804000409480006A
:10B1D00000F0A7000000EA000080400051948000C9
:10B1E00001F0A7008100EA00010040004200DE00FB
:10B1F000F046880018002000ED0F500001003600D6
:10B200000004EB0011C0B300EE0F500003003E003D
:10B210008040EB000000EB00040037009FC8BF0037
:10B220000080FB000000E9004F00DE00F2892000F2
:10B23000014978000000E000050032000041EB0009
:10B2400082407800F0C0B3000AC70200000000008E
:10B25000F0468000ED0F500011003E005C08EC004D
:10B26000E0428800E50F500007003400EA0F50006C
:10B2700001003A005C28EF000041EB0082407800BA
:10B2800000C2B300030037000041EB0082407800A9
:10B29000024078000AC702000000000005003700E5
:10B2A000A5FD07000001EB008000EB00AEC7020027
:10B2B00000000000E09480000000E0000500320083
:10B2C000C02921000008EB005000200000E102002E
:10B2D00000000000DA918000803E2000800F5500C1
:10B2E00019003400E2918000800F510016003400F4
:10B2F000F2918000800F5100130034001292800000
:10B30000800F510003003C0022928000800F51000A
:10B310000D0034002008200072938000800F51003F
:10B320000900340082938000800F51000600340031
:10B33000202721000008EB000080E8000008EB0057
:10B34000180020004E003700C5918000803E20008C
:10B35000F4918000808F52000A003C00800F55005D
:10B3600008003C00E2918000800F510005003C0085
:10B37000800F520003003C0002928000800F5100B9
:10B380002D0034000B9280004300200011000900C2
:10B390000305D80080047800520020001100090045
:10B3A0008202D8000003780086844400E691800081
:10B3B000110009000303D8008003780007834400CC
:10B3C000110009000302D8008003780087014300C0
:10B3D000110009008205D8008003780087814100B0
:10B3E000110009000205D800000578006700200060
:10B3F000110009008702D80080027800050145008D
:10B40000A6FF2F00110009008605D80000014100A9
:10B41000B6FF2F00110009000602D800000241000B
:10B4200084804100202721000108EA000080E80014
:10B43000030852001200370013928000249280000B
:10B44000808F510002003C00800F52000800340041
:10B4500042002000110009008201D800909388006A
:10B46000110009000202D800A093880004003700F0
:10B47000202721000008EB000080E8000008EB0016
:10B480001008200071938000808F5000030034006A
:10B4900081938000808F50000D003C002027210008
:10B4A0000008EB000080E8000008EB000041EB0022
:10B4B0008240780000C2B30026C7020000000000EE
:10B4C0000041EB008240780000C2B3000800370062
:10B4D0000041EB00824078000240780026C702005D
:10B4E000000000000041EB0082407800024078003C
:10B4F00042C702000000000080DA2F009193800014
:10B50000808F500001003D009093880080DA2F006A
:10B51000A1938000808F500001003D00A09388001F
:10B520008025200091938000808F5000010034001E
:10B530009093880080252000A1938000808F500088
:10B5400001003400A0938800884078000000EB00E0
:10B550000804E000040032009EC8BF000080FB0029
:10B560000000E9004F00DE00E28920000149780078
:10B570000000E000030032004000200004E102006F
:10B58000000000000804A2000000EB000804E00036
:10B59000040032009DC8BF000080FB000000E900ED
:10B5A0004F00DE00D1892000884878000000E000CC
:10B5B000030032000080EB0000E102000000000008
:10B5C0004F05BE004F04BE00000006000400FA0054
:10B5D0003349AB0041003200F1BF2F00209320001F
:10B5E0001088600011862000914078000104E0007E
:10B5F0000C003A006268EF0010C0B30061E8B700C9
:10B600008043EB00074378008742780007427800C8
:10B610008741780007417800874078007F404000EC
:10B620001400370062C8BF00E1CF500014003A0098
:10B63000E24F500029003400FD4F500027003C002D
:10B6400021C0B30012862000014978000040E800C4
:10B650005EE8B70007C2B3000043EB008642780003
:10B6600006427800864178000641780087407800DD
:10B6700007407800BAC6020000000000170037003B
:10B68000E2CF500015003A005E48E30013003D0091
:10B6900071C2B300814F500010003C0030C0B300B5
:10B6A00061E8B70007C2B300074378008042EB00AF
:10B6B000054278008541780007417800874078008E
:10B6C00007407800BAC602000000000070002000A9
:10B6D00000E10200000000006068EF0062C8BF00E7
:10B6E00031C6B300814F500002003C000040E8002A
:10B6F00062E8B70020C3B3006248E3000B003400E7
:10B700006168EF008043EB000743780087427800D0
:10B710000742780087417800074178008740780029
:10B7200007407800BAC602000000000062C8BF00EF
:10B73000E54F500015003A005FC8BF00E14F5000D0
:10B7400009003A0061C8BF00E14F50000F003A0005
:10B7500020C0B3005FE8B700000520009093880088
:10B7600000FB2F0008003700E24F500007003A00AE
:10B7700061C8BF00E14F500004003A005FE8B70025
:10B780000005200090938800A093880062C8BF0045
:10B79000FE4F500012003A0061C8BF005F48E2004F
:10B7A00008003A00E24F500006003A0010C0B30013
:10B7B0005FE8B7000005200090938800A093880000
:10B7C00007003700E24F500005003A005F68EF00C5
:10B7D000202721000008EB000080E8000008EB00B3
:10B7E00080C2B3006248E3000A003A0061C8BF00AB
:10B7F000E34F500007003A0010C0B3005FE8B70005
:10B800000105200091938800412721008008EB006A
:10B8100060E8B7001008200071938000808F50000E
:10B820000300340081938000808F50000D003C00A5
:10B83000202721000008EB000080E8000008EB0052
:10B840000041EB008240780000C2B30026C702002E
:10B85000000000000041EB008240780000C2B3000D
:10B86000080037000041EB00824078000240780079
:10B8700026C70200000000000041EB008240780073
:10B880000240780042C70200000000006048E20069
:10B890002200320064805700D5FA07006FF9970044
:10B8A000DFF897004FF897000AC702000000000079
:10B8B0005FF99700CFF897006FF8970042C7020032
:10B8C000000000004FF99700EFF897005FF897002D
:10B8D00026C70200000000006048EC0060E8B700E6
:10B8E000F1C7B300814F500012003A006068EF00CA
:10B8F0000041EB00824078000240780042C702001D
:10B90000000000000041EB00824078000240780017
:10B9100026C70200000000000600370006FC0700F2
:10B92000004178008040EB00014078000AC7020027
:10B93000000000000080FA0000000600FEFB070087
:10B9400000417800804078000040EB000AC7020008
:10B95000000000000040EB0001FC22001104E000A8
:10B960000D003200E38040001104E0000A003200C4
:10B97000E02621008080E8009100780010804000DF
:10B9800022002000110009000200D8006009B00068
:10B99000A046880010C0B30011FC22001104E00092
:10B9A00013003200E38040001104E0001000320078
:10B9B000E02621008080E80091007800108040009F
:10B9C00022002000110009000200D800B0468800C3
:10B9D00051092000810F500002003E00800C200021
:10B9E000B0468800A0F62F00D628B4000200370029
:10B9F0000004E0000F0032008043EB0007437800B2
:10BA00008742780007427800874178000741780034
:10BA10008740780007407800BAC6020000000000A6
:10BA2000202721000008EB000080E8000008EB0060
:10BA30000000060071938000A2468000828F5000B3
:10BA400002003100204723000048EB00B046800090
:10BA5000808F50000300360013C0B300214723003D
:10BA60008348780081938000828F5000020031006B
:10BA7000324723000049EB00808F5000030036005E
:10BA800011C0B3003047230001487800204723004D
:10BA900010407800314723000004E00004003A0021
:10BAA0001104E00006003A006368EF001700370059
:10BAB000E14F500002003A001104E0001200320091
:10BAC0003147230012C0B300914F110004003A0027
:10BAD0000004E00002003A0063E8EF000B003700CA
:10BAE00063C8BF004240A9000200340020C0B30078
:10BAF000050037000004E00002003200E0CFB30090
:10BB000001003700A0C0B30063E8B70063C8BF00FE
:10BB10000C003A00C012200090938800A093880087
:10BB20008043EB00074378008742780004C2B300EB
:10BB3000874178000741780087407800044078000A
:10BB400036003700E14F50000D003A00C0122000CF
:10BB500090938800402721000008EB008043EB0011
:10BB600007437800874278000742780003C2B30099
:10BB700007417800834078000740780027003700AD
:10BB8000E14F400009003A00202721000008EB00A7
:10BB9000C0122000A093880007C2B3000043EB004E
:10BBA00087427800064278000A003700E24F4000E2
:10BBB0000C003A0040ED2F0090938800C012200046
:10BBC000A09388008043EB0006C2B3008742780050
:10BBD000074278008441780004417800844078006E
:10BBE0000D003700E24F50000E003A00C012200056
:10BBF0009093880040ED2F00A09388008043EB00D5
:10BC00000743780087427800074278008741780030
:10BC100002C2B3008740780001407800BAC6040031
:10BC200000000000EA4F500004003A00C01220005B
:10BC30009093880040ED2F00A0938800000006003C
:10BC40003DFB0700004178008040EB000AC702007E
:10BC50000000000010FC22009080FB008100EA0040
:10BC6000CF08DE000000EB000104E0000400320019
:10BC7000A5C8BF000080FB000000E9004F00DE0007
:10BC8000528A2000014978000000E00002003200E2
:10BC9000A0F62F00A042880040FC22009080FB000C
:10BCA0008100EA00CF08DE000000EB000104E000A4
:10BCB00004003200A4C8BF000080FB000000E900BF
:10BCC0004F00DE00428A2000014978000000E000B9
:10BCD0000200320060092000A042880000FC22001F
:10BCE0009080FB008100EA00CF08DE000000EB003E
:10BCF0000104E00004003200A3C8BF000080FB0084
:10BD00000000E9004F00DE00328A2000014978007F
:10BD10000000E000060032005408E2000200320099
:10BD20005428EF0002003700A0F62F005228B4007C
:10BD300030FC22009080FB008100EA00CF08DE008A
:10BD40000000EB000104E00004003200A2C8BF00C4
:10BD50000080FB000000E9004F00DE00228A200086
:10BD6000014978000000E000060032005408E200BB
:10BD7000020032005428EF00020037006009200062
:10BD80005228B4008000EB0000FC22001004E00008
:10BD900004003200630040009080FB008100EA0054
:10BDA000CF08DE000000EB000104E00004003200D8
:10BDB000A1C8BF000080FB000000E9004F00DE00CA
:10BDC000128A2000014978000000E00001003200E2
:10BDD0005228EF008000EB0040FC22001004E0003D
:10BDE00004003200630050009080FB008100EA00F4
:10BDF000CF08DE000000EB000104E0000400320088
:10BE0000A0C8BF000080FB000000E9004F00DE007A
:10BE1000028A2000014978000000E00001003200A1
:10BE20005428EF00809480000000E00047003200BA
:10BE300001022000810F50003000320014003C004D
:10BE4000E60F50003A00320006003C00E40F5000BC
:10BE50002E00320039003C00E20F500039003A0059
:10BE600026003700ED0F50003400320003003C0084
:10BE7000E80F500033003A0026003700F00F500062
:10BE80002B003200F10F50002E003A001F00370047
:10BE900001052000810F50001800320008003C000E
:10BEA000E3805000810F5000180032008100E8004C
:10BEB000810F50001E0032001102200005003700E3
:10BEC00051052000810F50001000320004003C009A
:10BED000E4805000810F50001A003A000D00370036
:10BEE00061052000810F5000110032008100E80040
:10BEF000810F500013003A00100037006009200045
:10BF00005408E2000800320005003700A0F62F00B8
:10BF100008003700A0F62F005408E20002003200AB
:10BF20005428EF00070037005228B40005003700FE
:10BF300060092000A0428800020037005428EF006A
:10BF40005228EF00002921000008EB008025200086
:10BF50005208E300010034009042880080DA2F008C
:10BF60005208E30001003D00904288008025200037
:10BF70005408E30001003400A042880080DA2F005A
:10BF80005408E30001003D00A04288009142800077
:10BF9000A042800022272100010940000281E80020
:10BFA0000089500000000600001020006C740200A0
:10BFB00000000000002020006C740200000000005F
:10BFC000000120006C74020000000000400020000E
:10BFD0006C74020000000000100020006C7402006D
:10BFE00000000000000120006C740400000000004C
:10BFF0005648EC0056E8B70041C6B300814F5000E8
:10C000002100360050C6B30056E8B70020FC2200DD
:10C010009080FB008100EA00CF08DE000000EB000A
:10C020000104E0000400320096C8BF000080FB005D
:10C030000000E9004F00DE0062892000014978001D
:10C040000000E0001000320060428000A6F9070006
:10C05000804280000000E00002003A000040210021
:10C06000140037004C08E30004003A000000EB0025
:10C0700056F907004C28EF000300370053F907007A
:10C080005008F8004C08F900C2F40200000000005B
:10C090000000E00004003A006CC302000000000051
:10C0A0000048A30006003200604280008EF90700BD
:10C0B000004020008474020000000000BAFF370036
:10C0C000604280008000EB00E70F5000E08F5800D6
:10C0D0005D003E000060010007003700540037009B
:10C0E0005400370054003700570037005300370022
:10C0F000530037005300370000FC22009080FB0003
:10C100008100EA00CF08DE000000EB000104E0003F
:10C110000400320095C8BF000080FB000000E90069
:10C120004F00DE0052892000014978000000E00045
:10C13000040032008080EB0080428000E1F80700BC
:10C140008042880010FC22009080FB008100EA0001
:10C15000CF08DE000000EB000104E0000400320024
:10C1600094C8BF000080FB000000E9004F00DE0023
:10C1700042892000014978000000E00004003200FC
:10C180008080EB0080428000CEF80700804288006B
:10C1900030FC22009080FB008100EA00CF08DE0026
:10C1A0000000EB000104E0000400320093C8BF006F
:10C1B0000080FB000000E9004F00DE003289200013
:10C1C000014978000000E000040032001100200066
:10C1D00080428000BBF807008042880040FC2200BB
:10C1E0009080FB008100EA00CF08DE000000EB0039
:10C1F0000104E0000400320092C8BF000080FB0090
:10C200000000E9004F00DE0022892000014978008B
:10C210000000E00004003200110020008042800095
:10C22000A8F807008042880080428000B7F83700F5
:10C23000D4F9370003FB3700DBFB3700E3FC3700A2
:10C24000BEFD37007EFE0700000006007042880039
:10C250000000EB00DDF807004E08E20002003200AB
:10C260005028EF00030037001000200080428800B3
:10C27000A6F80700B04620006C740400000000001F
:10C28000004020007C740200000000008000780064
:10C290000080EB000100E0000100320060428000FD
:10C2A0000000060090089000E0019000018140002D
:10C2B000630179008100E90011089800020078000C
:10C2C0000000060023002000730098007001400069
:10C2D000610029001CD3040000000000889FBE00FC
:10C2E0008A9FBE008C1F7800000678004C039000E7
:10C2F0008203E80087834300E6837B008582E900B0
:10C30000020441000803430016831100860F520007
:10C3100003003E00818540000003EB000F00370062
:10C320000C007800E7FF07000E0037004C04900077
:10C330008384430086844400110009008584D8006A
:10C3400081047800890441008984E80089844400DC
:10C35000E9357C000603E8008B85E800840F530074
:10C36000F2FF39004F0678004F05BE004F04BE00B3
:10C3700000000600889FBE008A9FBE008C1F7800C8
:10C380008005780001067800130037001B03780051
:10C390000C84E800110009008281D8008103780034
:10C3A000888343008784430085834100110009008E
:10C3B0008283D80081037800888343008783430009
:10C3C000E7347B000500E00002003D008301E90046
:10C3D000010037008301E8000500E00003003D0094
:10C3E000848F5100E9FF310002003700848F510033
:10C3F000E6FF36004F0678004F05BE004F04BE0032
:10C4000000000600889FBE008A9FBE008C9FBE0071
:10C410008E1F7800800478000304780049009000A3
:10C420000187400060057F008106E8008D86460098
:10C43000E0817E0002005500800F540003003600AA
:10C44000090078009FFF07001D0037008485E90080
:10C450000A00D1008802EA00800F51000D0031006F
:10C46000088641000201E90008014100688044009B
:10C470000C027800830141000B017800BDFF07002A
:10C4800049019000110009000B86D80001B17E001F
:10C49000080037000502E9000A02420068804400F3
:10C4A0008802780003024200828141000B0178007B
:10C4B000B0FF0700490090000804550008307F00D5
:10C4C0004F0778004F06BE004F05BE004F04BE0068
:10C4D00000000600E6874700889FBE008A9FBE00D6
:10C4E0008C9FBE008E1F78000006780081057800C2
:10C4F000F2B79F008306780005047800CC00900016
:10C500000B80450080BF9F00610778000B00E800AA
:10C510000000400000814000920478000485E9009A
:10C520008E005500810F5400030036000C00780087
:10C5300064FF0700330037008E00D100818F560062
:10C54000110031000900E00002003A0088045500A3
:10C5500006003700888454008A84440011000900D2
:10C560008A84D8008000FD008004780009097800E2
:10C570000D82E90068004600880278000802420047
:10C5800089017800070037000D0244008801470048
:10C590008301E900680046008802EA0009024200BF
:10C5A000898141000A0178008B00780071FF070043
:10C5B000FFB09700018140008002EB000B003700C4
:10C5C0008D81440085814100110009008A81D800D5
:10C5D00081017800838145008381E80083814100E7
:10C5E000E2317B008502E8000281E8004C03900004
:10C5F000888F5200F2FF39000E0444008FB8970074
:10C6000008B378004F0778004F06BE004F05BE0004
:10C610004F04BE006F00B100000006000200FA00E7
:10C62000889FBE0080047800010478000900E000C3
:10C6300003003A00000028000000640056003700A4
:10C64000000024000800E0005000320008017800DB
:10C6500002F0A7000201EA000900780000F0A7003C
:10C660000000EA006102B900E681570011000900EC
:10C6700042AAD80081097800000378005FBA9700C9
:10C680008002EB00C022DD00040020001100090040
:10C6900042AAD800000178008600780002007800E5
:10C6A0000681CF000200E0000300320003022000F8
:10C6B00002815100040037000081CF000200E00039
:10C6C00001003200700111006C03510009003B00B1
:10C6D000C2282000030020009A040200000000008D
:10C6E000440ADD004C01DE00020172000200780005
:10C6F000220037001400200005002000820178008D
:10C700008301E900030033000402420085824A00ED
:10C71000FBFF37000400500085805800680151007D
:10C720000201E900030033008180D1000080D300C2
:10C73000FBFF3700FF0160004580DE004333DD0072
:10C7400086004000018040008427290064007800B2
:10C7500002022000030351000683B9008100E800B3
:10C7600081804000648078000380B90000034300AA
:10C7700081834B0011000900423BD8000800E00013
:10C7800002003D0001002800008050000900E00088
:10C7900001003C000000EA004F04BE000080FA00E7
:10C7A000000006000000E0000C003D0002002C002C
:10C7B000820F500003003D000100280001004000EE
:10C7C0000400370011002800820F500023003200BF
:10C7D0000000EA00120020000A00370002002400D6
:10C7E000820F500003003400010028000080500038
:10C7F00003003700F1FF2700820F500017003200BE
:10C800000001EB00C780DE0000027800F407B200F0
:10C810000100E80000004000631729006300780071
:10C820000483B9008180400000082000040050000B
:10C830006382780000A0B9000600400087804800AD
:10C84000C909DD004702DE0004827100840078001F
:10C850000200E000010032008100EA0001007800DF
:10C86000000006000100240001004000CDFF370059
:10C870000100240001003700C288DE00808F5000D4
:10C88000FDFF3C00000178000000EB0007003700CE
:10C89000808140000080D100830F510002003500EC
:10C8A0000301510001004000C288DE000100E000E9
:10C8B000F7FF3A0000000600889FBE008A9FBE0076
:10C8C0000005BE000B0178008001EB001800370066
:10C8D000430020000311B80054002000110009009B
:10C8E0004499D800000178000A0378008202E90028
:10C8F0008582420085024500020278008001EB003B
:10C9000009003700B6037800550478008884530086
:10C910004240A9000300340078BB9F00870A7800DA
:10C92000130020000402E8008B0F5200F5FF3900CD
:10C93000E10F5100E6FF3E000300E000EAFF3A008D
:10C940004F05BE004F04BE0000000600889FBE00D9
:10C950008A1F7800000478000800780051FE070064
:10C9600000057800080078004EFE0700800478007B
:10C97000080078004BFE07000A0545008984440042
:10C980008000EB0005003700480190006935790010
:10C990008100E8000A85E8008984E800808F500063
:10C9A000F9FF39004F0578004F04BE000000060073
:10C9B000889FBE008A1F7800000478000800780075
:10C9C00038FE0700800478000800780035FE070074
:10C9D000000578000800780032FE07000A054500CF
:10C9E000898444008000EB00040037004801900077
:10C9F000EA3479008100E8008984E800808F5000E3
:10CA0000FAFF39004F0578004F04BE000000060011
:10CA1000889FBE008A9FBE0000047800080078004E
:10CA200020FE070000057800080078001DFE0700C2
:10CA300080047800080078001AFE0700800578005E
:10CA40000800780017FE0700C80090008B8545009D
:10CA5000E1817D000A054500898444008000EB00E7
:10CA6000070037004801900062827C000302420008
:10CA700004317D008100E8000A85E8008984E8002F
:10CA8000808F5000F7FF39004F05BE004F04BE00F5
:10CA900000000600889FBE008A9FBE000004780048
:10CAA00008007800FFFD0700800578000800780086
:10CAB000FCFD07000005780008007800F9FD07007C
:10CAC0008004780008007800F6FD07008000EB0085
:10CAD0000001EB000E003700C80190000B824500FA
:10CAE00001024200048241008982440081824200A6
:10CAF000858241000A03450001034300868141000D
:10CB000095027800138A42000201E8008180E80063
:10CB1000800F5100F0FF39004F05BE004F04BE00EA
:10CB200000000600889FBE008A9FBE0000047800B7
:10CB300008007800DBFD0700800578000800780019
:10CB4000D8FD07000005780008007800D5FD070033
:10CB50008004780008007800D2FD07008000EB0018
:10CB60000001EB000E003700C80190000B82450069
:10CB700001024200048241008A0245008182420093
:10CB800085824100098344000103430086814100FE
:10CB900095027800138A52000201E8008180E800C3
:10CBA000800F5100F0FF39004F05BE004F04BE005A
:10CBB00000000600889FBE008A9FBE000004780027
:10CBC00008007800B7FD07008005780008007800AD
:10CBD000B4FD07000005780008007800B1FD0700EB
:10CBE0008004780008007800AEFD07008000EB00AC
:10CBF0000001EB000D003700C80190000B824500DA
:10CC00000102420009834400010343008A024500F7
:10CC10008182420063037B00E3827A0005B3B9009E
:10CC200086317A000201E8008180E800800F51001F
:10CC3000F1FF39004F05BE004F04BE0000000600A2
:10CC4000E4874700889FBE008A9FBE008C9FBE007D
:10CC50008E1F7800000478000800780091FD07001E
:10CC600080067800080078008EFD07000006780036
:10CC7000080078008BFD0700800578000800780028
:10CC800088FD0700000278008004EB000005EB003F
:10CC90001F003700C80090000C004600090040004B
:10CCA000610078000B8145000901410061017900B4
:10CCB000CF91DE00E00F5100E08F59000C003200F0
:10CCC0000D874600090747000E874000CF80DE0031
:10CCD00084BF9F00E006020000000000000F780003
:10CCE0000A05E8008984E8000FBA970008003700B9
:10CCF0002300200073049800700144007100290093
:10CD0000080078001CD30200000000000200370079
:10CD1000840F5500DFFF39004F0778004F06BE0033
:10CD20004F05BE004F04BE004F00B10000000600DA
:10CD3000889FBE008A9FBE0000047800080078002B
:10CD400058FD0700800578000800780055FD0700B1
:10CD5000000578000800780052FD07008004780084
:10CD6000080078004FFD07008000EB000001EB0099
:10CD700010003700C80190008B824500818242007C
:10CD80008582410009834400010343000A024500F3
:10CD90000102420063027A00E3017B00848F5100AC
:10CDA0000100340084017800830A78000201E80061
:10CDB0008180E800800F5100EEFF39004F05BE0072
:10CDC0004F04BE0000000600889FBE008A9FBE0080
:10CDD000000478000800780032FD07008005780024
:10CDE000080078002FFD0700000578000800780093
:10CDF0002CFD0700800478000800780029FD07005A
:10CE00008000EB000001EB0010003700C80190002B
:10CE10008B82450081824200858241000983440063
:10CE2000010343000A0245000102420063027A0046
:10CE3000E3017B00848F510001003D0084017800F4
:10CE4000830A78000201E8008180E800800F510029
:10CE5000EEFF39004F05BE004F04BE000000060083
:10CE6000889FBE008A9FBE008C1F78000004780057
:10CE7000080078000BFD0700000678000800780025
:10CE800008FD0700800578000800780005FD070010
:10CE9000000578000800780002FD07008004780093
:10CEA00008007800FFFC07008000EB000002EB00A8
:10CEB00015003700480190008B81450081814100B9
:10CEC000E28279008A014500818141006283790014
:10CED0008981440081814100E2817900838F520081
:10CEE00004003C0086017800858F510001003D0060
:10CEF000850178008C0246008182420003B17A00ED
:10CF00000402E8008180E800800F5200E9FF390048
:10CF10004F0678004F05BE004F04BE00000006001B
:10CF2000889FBE008A9FBE008C1F78000004780096
:10CF300008007800DBFC0700800478000800780017
:10CF4000D8FC07008005780008007800D5FC0700B1
:10CF5000000678004805900008007800D1FC070022
:10CF6000000040006A05780008007800CDFC07004A
:10CF700001022000810F550005003C000C06460010
:10CF80008B8545000002EB006011B8000D003700F2
:10CF9000480090008984440089044000800CEB0024
:10CFA00012003700E1827D0061037E0006ABB9000C
:10CFB0000201430083814B000402E8000C86E80074
:10CFC0008B85E800C8009000800F5200F5FF390003
:10CFD000898444000A05E900030033008381D100FD
:10CFE0000281D300FBFF370082B07C004F0678003F
:10CFF0004F05BE004F04BE00000006000200FA000C
:10D00000889FBE008A9FBE00000178000200780061
:10D01000B2BF9F00A3FC0700800478003FB89700D0
:10D02000A0FC0700800578003FB897009DFC070032
:10D03000000478003FB897009AFC070000057800CC
:10D040003FB8970097FC0700800278003FB997002F
:10D050000500E000240032004202900009804400F4
:10D06000E40178006118B9008B85450003B27D00AA
:10D07000080444004202900003327C0014002000A7
:10D08000100037008901420083814100E681790068
:10D090000B034300968F510001003D00030B780005
:10D0A0004203900008034300968F510001003400B2
:10D0B000030B78004F9BDE000080410081004B0095
:10D0C0000402E80042039000850F5200EDFF390092
:10D0D0000A0545000A0443006129B800E006020081
:10D0E00000000000000C78004F05BE004F04BE0099
:10D0F0000080FA0000000600889FBE008A9FBE00E4
:10D10000000478000800780066FC070080047800BE
:10D110000800780063FC07008005780008007800AC
:10D1200060FC070000057800080078005DFC07003F
:10D130000000E000150032008B8545000A0545001F
:10D14000898444008000EB0004002800F3FF2700DE
:10D15000C802900065817C00830F510002003D00F1
:10D1600081B27D0082017800840F510003003400F9
:10D170004802900001327D00020278008100E80040
:10D180008984E800808F5000F1FF39004F05BE0010
:10D190004F04BE0000000600889FBE000004780017
:10D1A000080078003FFC0700800478000800780041
:10D1B0003CFC07008000780089844400480090000F
:10D1C00009004000BCFD07004F04BE00000006003F
:10D1D000E6874700889FBE008A9FBE008C9FBE00E6
:10D1E0008E1F780000047800080078002DFC0700EE
:10D1F00000077800080078002AFC07008006780005
:10D200000800780027FC0700000678000800780076
:10D2100024FC0700800578000800780021FC070046
:10D22000800278008004EB000005EB00240037004A
:10D23000C80090000D80460009004000610378009E
:10D240000C00460009004000610078000B81450099
:10D250000901410061017900CF91DE00E00F51002A
:10D26000E08F59000E0032000E0247000902420012
:10D270000482400000B0B90084BF9F00F5B79F0052
:10D28000E0060200000000000FBA9700000A7800D4
:10D290000A05E8008984E800FFB29700080037001B
:10D2A00023002000730498007001440071002900DD
:10D2B000080078001CD302000000000002003700C4
:10D2C000850F5500DAFF39004F0778004F06BE0082
:10D2D0004F05BE004F04BE006F00B1000000060005
:10D2E000E4874700889FBE008A9FBE008C9FBE00D7
:10D2F0008E1F78008004780009007800E9FB0700A1
:10D300000007780009007800E6FB07008006780037
:10D3100009007800E3FB07000006780009007800A8
:10D32000E0FB0700000178000004EB000005EB00C3
:10D330000F003700C90590008C004600888040002F
:10D340000D80460008004000EB8078006B007800FC
:10D3500082BF9F00B1FC07008E004700888040001C
:10D3600080B578000A05E8000884E8000FB9970046
:10D37000820F5500EFFF39004F0778004F06BE00BF
:10D380004F05BE004F04BE004F00B1000000060074
:10D39000889FBE008A9FBE008C9FBE0080047800DC
:10D3A00009007800BFFB07008006780009007800BC
:10D3B000BCFB07000005780009007800B9FB0700F6
:10D3C000000678000A0545000004EB00080037005D
:10D3D000C90590006B007D00F2FC07008D00440041
:10D3E0008180400080B578000804E8000A85E800E4
:10D3F0008C0F5400F6FF39004F06BE004F05BE00EB
:10D400004F04BE0000000600889FBE008A9FBE0039
:10D410008C9FBE008004780009007800A1FB070003
:10D4200080067800090078009EFB07000005780060
:10D43000090078009BFB0700000678000A054500FC
:10D440000004EB0008003700C90590006B007D0068
:10D4500004FD07008D0044008180400080B5780005
:10D460000804E8000A85E8008C0F5400F6FF390034
:10D470004F06BE004F05BE004F04BE000000060070
:10D48000889FBE008A9FBE008C9FBE008E1F7800C2
:10D49000000478000800780082FB0700000578008F
:10D4A000080078007FFB07008005780008007800FE
:10D4B0007CFB0700C80490008B804500E98678005B
:10D4C0008B05E8008B854500E9857D000000400064
:10D4D000690778000E007800E2FC0700000678007B
:10D4E0000E007800AFFC07008A0045000DE2B9008D
:10D4F0000B81B9000202520083825A00412BDD00E9
:10D500004F21DE000201730082B478000A05E800B2
:10D51000C80090000A0545000D81B9000BE6B9006E
:10D520000206460083864E004168DD004F61DE0042
:10D530000201700082307D004F0778004F06BE0068
:10D540004F05BE004F04BE0000000600889FBE00CD
:10D550008A9FBE008C9FBE0080047800090078007E
:10D5600050FB070080067800090078004DFB07009B
:10D5700000057800090078004AFB070000067800E3
:10D580000A0545000004EB0008003700C9059000BB
:10D590006B007D00B6FC07008D00440081804000D8
:10D5A00080B578000804E8000A85E8008C0F540074
:10D5B000F6FF39004F06BE004F05BE004F04BE0007
:10D5C00000000600889FBE008A9FBE008C9FBE00A0
:10D5D000800478000900780032FB0700000478001E
:10D5E000090078002FFB070000057800090078008B
:10D5F0002CFB0700800578000900780029FB070054
:10D6000000017800C90690008B854500ED837D0000
:10D610008A01E90003824100048246000006EB0013
:10D62000070037000C06E800820F560004003600A1
:10D6300008044400888046008008EB004B00370057
:10D640005400E000F7FF3A000C0278008C814100A2
:10D6500083814100838146000B0037000C06E800FF
:10D66000820F560008003600080444000400E00061
:10D67000360032000400E900870F50003300390003
:10D680000000D100380037005300E000F3FF320003
:10D690000003EB008002EB008001EB000302780046
:10D6A000030037000402E800820F52000900310035
:10D6B0008C044200110009008284D80081047800A3
:10D6C0008A84440089844400ED847C000900E000E1
:10D6D000F4FF3A0083045200858F540006003400A2
:10D6E0008301420025002000110009008501D800B7
:10D6F0000003780089027800820F5200050039008B
:10D700000F0037008301E800828F510002003900CA
:10D710000B003700840178000C82410011000900E1
:10D720000282D800010278000A024200040242008C
:10D730006D027A000400E000D8FF3A00F1FF3700E4
:10D7400008044400878F520003003D00088446000F
:10D75000008CEB00050037000C00430011000900AD
:10D760000280D8008000FD0080367C004F06BE009D
:10D770004F05BE004F04BE0000000600F04A8800BE
:10D780000000060050252600F14A80000088B900FC
:10D790009261230000004100F04A8800000006006A
:10D7A000889FBE008A9FBE008C1F7800000578000D
:10D7B0000A007800BBFA0700800478000A007800AD
:10D7C000B8FA070080057800898444000004EB0063
:10D7D000060037004A06900009064600E9FF0700E8
:10D7E000000E78000804E8008984E8008B0F5400DC
:10D7F000F8FF39004F0678004F05BE004F04BE0009
:10D8000000000600889FBE008A1F78000004780090
:10D8100008007800A3FA0700800478000800780068
:10D82000A0FA070000057800080078009DFA0700BC
:10D83000480090000A054500898444006935780055
:10D840004F0578004F04BE0000000600889FBE0010
:10D850008A9FBE008C9FBE000004780008007800FC
:10D8600090FA070000057800080078008DFA07009C
:10D8700080047800080078008AFA070080064000DB
:10D8800048009000E0857E000800780085FA0700D7
:10D89000000678000800780082FA0700000278008D
:10D8A0004800900060807E000000E000030035002A
:10D8B000E3005600810F5000030036000800780096
:10D8C00080FA0700040037008C0278000A01BE00CD
:10D8D0000800BE0081FA07004F06BE004F05BE00DB
:10D8E0004F04BE0000000600889FBE008A9FBE0055
:10D8F0008C9FBE008E1F780000047800080078001E
:10D9000068FA0700800478000800780065FA0700CC
:10D91000000578000800780062FA070080064000E1
:10D9200048009000E0857E00080078005DFA07005E
:10D9300000067800080078005AFA0700000778000F
:10D94000C800900009814400E10179000901E80064
:10D9500002014100E10279000C81E900E1807E00D2
:10D960000100E00009003500630656008C8F50006E
:10D9700006003E008B805100810F570003003E00DF
:10D980000A0545008003EB000F003700080078000F
:10D990004CFA07000E003700C80190000B824200CD
:10D9A00007024200110009000282D800010278003B
:10D9B000048244000482E800040242006AB2790052
:10D9C0008703E8000A85E8008E8F5300F2FF3900D4
:10D9D0004F0778004F06BE004F05BE004F04BE0043
:10D9E00000000600889FBE008A9FBE008C9FBE007C
:10D9F00000047800080078002AFA07008004780004
:10DA00000800780027FA0700000578000800780071
:10DA100024FA07008006400048009000E0857E0060
:10DA2000080078001FFA0700000678000800780058
:10DA30001CFA0700800278004800900060807E0099
:10DA40000000E0000300350063005600808F5500A1
:10DA500003003600080078001AFA070004003700B7
:10DA60000C0278000A01BE000800BE0099FA070007
:10DA70004F06BE004F05BE004F04BE00000006006A
:10DA8000889FBE008A9FBE008C1F7800000478002B
:10DA90000800780003FA0700800478000800780086
:10DAA00000FA07000006780008007800FDF907007A
:10DAB000C80090000C06460061057E000000400092
:10DAC000E105780008007800F6F907000002780008
:10DAD0004800900060007E000000E0000300350078
:10DAE00063005200800F55000300360008007800E4
:10DAF000F4F90700030037000A01BE000800BE0069
:10DB000040FA07004F0678004F05BE004F04BE00E4
:10DB100000000600889FBE008A9FBE0000047800B7
:10DB200008007800DFF9070080047800080078001A
:10DB3000DCF907000005780008007800D9F9070033
:10DB40008005780008007800D6F907008002780088
:10DB50000B0278008001EB000A0178000800BE008B
:10DB60005CFA07004F05BE004F04BE00000006002F
:10DB7000889FBE008A9FBE000004780008007800DD
:10DB8000C8F907008004780008007800C5F907008C
:10DB90000005780008007800C2F9070080057800C9
:10DBA00008007800BFF90700800278004801900063
:10DBB000898044000B027800E28178000A01780035
:10DBC0000800BE0043FA07004F05BE004F04BE0028
:10DBD00000000600889FBE008A9FBE008C1F780050
:10DBE0000004780008007800AEF90700800578008E
:10DBF00008007800ABF907000006780008007800FC
:10DC0000A8F907000005780008007800A5F90700CA
:10DC1000800478008A027800090278008001EB0015
:10DC20000B0178008C00780008007800ABF9070041
:10DC30000A027800890178000001EB008B0078006F
:10DC400008007800EFF907004F0678004F05BE0086
:10DC50004F04BE0000000600889FBE008A9FBE00E1
:10DC60008C9FBE0000047800080078008DF9070042
:10DC700080047800080078008AF9070080067800A0
:10DC80000800780087F9070000067800080078008F
:10DC900084F9070080057800C800900009804400DE
:10DCA00000804000108515008C0278000B0278007F
:10DCB0008A017800090178008D007800080078005A
:10DCC00086F907000C0278000A01BE000800BE00B9
:10DCD000CCF907004F06BE004F05BE004F04BE0042
:10DCE00000000600F14380000100E0001200320055
:10DCF00084C8EC0084E8B700FF4F500004003400F3
:10DD0000E3806000F143880000CEB30084E8B700F0
:10DD10007E08E2000800320041882000914078002F
:10DD20008100FB0001F0A7008100EA00E0C0B30021
:10DD3000DAC5020000000000F043800000F0A700F8
:10DD40000000EA000000E9004F00DE008000EB0068
:10DD50000004E00005003200E182200091407800DC
:10DD60008180FB008100E900CF08DE002EE8B700CB
:10DD70000100E000040032008040EB00E0C0B3008E
:10DD8000DAC502000000000000000600881F7800CD
:10DD9000F1FB2200A046230065824000514178003B
:10DDA0000204E0000600320010417800E341410027
:10DDB0000348780002C2B30082CF51000100360050
:10DDC000024878000000E800848F5000F3FF3A001A
:10DDD000C04623001004E0000B00320008022000BF
:10DDE000C04623009040780008407800DAC5020061
:10DDF000000000000804E80040022000800F5400EA
:10DE0000F7FF3A001C003700A0462300904078003E
:10DE10000104E0000300320010C2B300DAC50200C2
:10DE200000000000B0462300904078000104E000AC
:10DE30000300320020C2B300DAC502000000000077
:10DE4000D0462300904078000104E0000300320037
:10DE500000C2B300DAC5020000000000E046230063
:10DE6000904078000104E0000300320030C2B300AB
:10DE7000DAC50200000000008000EB00A04623008D
:10DE80001004E00004003A000080E8009080FB00ED
:10DE90008100E900CF08DE000000EB000104E00093
:10DEA0000400320036C8BF000080FB000000E9001B
:10DEB0004F00DE0063832000814978000000E0000D
:10DEC000040032008040EB0010C2B300DAC502004B
:10DED000000000008000EB00B04623001004E000CA
:10DEE00004003A000000E8009080FB008100E90097
:10DEF000CF08DE000000EB000104E0000400320067
:10DF000035C8BF000080FB000000E9004F00DE00C4
:10DF100053832000814978000000E00004003200B3
:10DF20008040EB0020C2B300DAC502000000000010
:10DF30008000EB00D04623001004E00004003A000B
:10DF40000000E9009080FB008100E900CF08DE00BE
:10DF50000000EB000104E0000400320034C8BF0000
:10DF60000080FB000000E9004F00DE00438320003A
:10DF7000814978000000E000040032008040EB009E
:10DF800000C2B300DAC50200000000008000EB0010
:10DF9000E04623001004E00004003A000080E9009D
:10DFA0009080FB008100E900CF08DE000000EB005C
:10DFB0000104E0000400320033C8BF000080FB0011
:10DFC0000000E9004F00DE00338320008149780023
:10DFD0000000E000040032008040EB0030C2B300DB
:10DFE000DAC50200000000004F04780000000600BF
:10DFF000618A2000914078008180FB008100E90067
:10E00000CF08DE000000EB000104E0000400320055
:10E010003CC8BF000080FB000000E9004F00DE00AC
:10E02000C2832000014978000000E00004003200B3
:10E030008040EB00D0C1B300DAC502000000000050
:10E04000A648E20005003200A668EF0001C2B30056
:10E05000D0C1B300DAC502000000000000000600D5
:10E06000881F78008A48EC008AE8B700EA4F500021
:10E0700024003A008A68EF00619480005009200073
:10E08000808F500006003C008040EB0060C2B3006F
:10E09000DAC502000000000001C2B300160037001C
:10E0A00080112000808F50000600340001C2B300B0
:10E0B0006E404000DAC50200000000008040EB0026
:10E0C0000D003700A0F62F00010040004500DD00E4
:10E0D00022082000110009000200D8000044780046
:10E0E0008040780060C2B300DAC502000000000082
:10E0F00001C2B30088C0500070C2B300DAC502008C
:10E10000000000004F04780000000600889FBE0059
:10E110008464AB003C0032008648E2000E003A0006
:10E120008040EB0050C0B300DAC5020000000000E0
:10E130008040EB0060C0B300DAC5020000000000C0
:10E140008040EB0070C0B300DAC5020000000000A0
:10E1500010C0B30086E8B7007388200093417800B0
:10E16000100020000304E000010032000300FB0067
:10E1700072C0B300EA0F500004003C0022002000EF
:10E18000110009000200D8000041E800834041006E
:10E19000728820000149780040C6B30080CF50004B
:10E1A000120034008548EC0085E8B70011C0B300C8
:10E1B0007288200001497800E34F500001003A00C6
:10E1C0008568EF008548E20008003A008040EB00D7
:10E1D00070C0B300DAC50200000000008040EB0010
:10E1E00060C0B300DAC502000000000085C8BF00AF
:10E1F000654040007188200091407800DAC5020037
:10E2000000000000AF003700602721008080E80098
:10E210009100780010804000883E20000884B900FA
:10E22000A2F820001100090042CCD80000047800B8
:10E230008648E200260032008668EF005018200071
:10E24000800F54000A00360001C2B30050C0B30072
:10E25000DAC502000000000001C2B30060C0B300D4
:10E26000DAC502000000000001C2B300150037004B
:10E2700080162000800F54000600360001C2B30053
:10E2800050C0B300DAC502000000000001C2B300B4
:10E290000800370040152000800F54000C003600A5
:10E2A00001C2B30050C0B300DAC502000000000094
:10E2B0008040EB0060C0B300DAC50200000000003F
:10E2C0008040EB0070C0B300DAC50200000000001F
:10E2D00011C0B30050182000800F540003003E000E
:10E2E0008040EB000000EB000400370032C8BF00A4
:10E2F0000080FB000000E9004F00DE0022832000C8
:10E30000014978000000E0000C00320001C2B300B7
:10E3100050C0B300DAC502000000000001C2B30023
:10E3200060C0B300DAC502000000000001C2B30003
:10E3300070C0B300DAC502000000000070E92F00D1
:10E340000800400011C0B300F70F50000300360072
:10E350008040EB000000EB000400370031C8BF0034
:10E360000080FB000000E9004F00DE001283200067
:10E37000014978000000E0000C00320001C2B30047
:10E3800050C0B300DAC502000000000001C2B300B3
:10E3900060C0B300DAC50200000000008040EB005E
:10E3A00070C0B300DAC5020000000000B0EA2F0020
:10E3B0000800400011C0B300EE0F5000030036000B
:10E3C0008040EB000000EB000400370030C8BF00C5
:10E3D0000080FB000000E9004F00DE000283200007
:10E3E000014978000000E0000C00320001C2B300D7
:10E3F00050C0B300DAC50200000000008040EB000E
:10E4000060C0B300DAC50200000000008040EB00ED
:10E4100070C0B300DAC502000000000011C0B300F4
:10E4200040152000800F5400030036008040EB00B0
:10E430000000EB00040037002FC8BF000080FB0085
:10E440000000E9004F00DE00F28220000149780060
:10E450000000E000080032008040EB0060C0B30024
:10E46000DAC50200000000008040EB0070C0B3007D
:10E47000DAC502000000000040152000800F5400A3
:10E4800010003E008748EC0087E8B700E34F5000DB
:10E4900004003A0001C2B30050C0B300DAC5020064
:10E4A0000000000087C8BF00E54F500005003400A1
:10E4B0008040EB0050C0B300DAC50200000000004D
:10E4C0008768EF004F04BE000000060000FC220039
:10E4D0009080FB008100EA00CF08DE000000EB0026
:10E4E0000104E000040032003BC8BF000080FB00D4
:10E4F0000000E9004F00DE00B283200001497800EF
:10E500000000E000030032002000200000E10200D3
:10E510000000000010FC22009080FB008100EA0057
:10E52000CF08DE000000EB000104E0000400320030
:10E530003AC8BF000080FB000000E9004F00DE0089
:10E54000A2832000014978000000E00003003200AF
:10E550002000200000E102000000000020FC22005A
:10E560009080FB008100EA00CF08DE000000EB0095
:10E570000104E0000400320039C8BF000080FB0045
:10E580000000E9004F00DE0092832000014978007E
:10E590000000E000030032003000200000E1020033
:10E5A0000000000030FC22009080FB008100EA00A7
:10E5B000CF08DE000000EB000104E00004003200A0
:10E5C00038C8BF000080FB000000E9004F00DE00FB
:10E5D00082832000014978000000E000030032003F
:10E5E0002000200000E102000000000040FC2200AA
:10E5F0009080FB008100EA00CF08DE000000EB0005
:10E600000104E0000400320037C8BF000080FB00B6
:10E610000000E9004F00DE0072832000014978000D
:10E620000000E000030032002000200000E10200B2
:10E630000000000000000600E4874700889FBE003D
:10E640008A9FBE008C9FBE008E1F7800CC3C2300AA
:10E650006B232100C23B23006E0246008B01780031
:10E660008C00780053007800D10F100001003D00AD
:10E67000800878000000E00003003200920F1000D4
:10E6800001003400000978000281E800848F500006
:10E69000F4FF3A00AA3D2300C9262100E401450009
:10E6A000890078000A00780051017800D00F11002D
:10E6B00001003D0002087800830F5000FAFF3A0085
:10E6C000AD3B23000004EB005D0078005C07100008
:10E6D0005B00100001003B000000EB000102200085
:10E6E0000181B900110009004E19D8000007780017
:10E6F000C0262A0060417C008E40780002407800ED
:10E7000082BF9F00DAC50200000000000FB9970029
:10E71000E20F540004003A000240E8008E40780006
:10E72000DAC50200000000000804E800E70F54000A
:10E73000E5FF3A002B272A000004EB005A0178007D
:10E74000590078000000E00001003D000000EB00EF
:10E75000010220000182B90011000900422AD800FC
:10E76000804078005B407800DAC5020000000000BD
:10E770000804E800E20F5400F0FF3A004F07780069
:10E780004F06BE004F05BE004F04BE004F00B10053
:10E7900000000600889FBE0050948000F40F5000D7
:10E7A0003C003C0041948000309480000E630200E5
:10E7B0000000000022002000110009000200D80023
:10E7C000037D200003014000F1F92000C801200072
:10E7D000810F51001C003600027721000202400028
:10E7E000B8012000810F520017003600047122008A
:10E7F00004024000A8012000810F520012003600E0
:10E80000046B23000402400098012000810F520095
:10E810000D00360088012000F5D52600850F520036
:10E8200009003E00830150006C044400818F5100B8
:10E830000500360002005000F8012000810F500052
:10E8400001003E00660444005994800009F0A700CE
:10E850008904EA00F48414008984440001003B0028
:10E860008004EB00404480000000E000030035001D
:10E870008040EB00DAC5020000000000894078000B
:10E8800008407800DAC50200000000004844880013
:10E8900007003700404480000000E000030035001E
:10E8A0008040EB00DAC502000000000088A8EF00FD
:10E8B0004F04BE0000000600670060004800DD0055
:10E8C000F18F2F00F20580008280600081007000CF
:10E8D000F105880000000600114480000100E000FE
:10E8E00002003A008AC0A9009AC0A8000080700007
:10E8F00010448800000006008208B60000000600F0
:10E900008AC0A800000006000080EA008208B60065
:10E910001044880001003A009AC0A90000000600D7
:10E920001000FA00889FBE008A9FBE0090C8BF00FA
:10E93000E14F50004B023A00C2F402000000000018
:10E940000000E00004003A006CC302000000000078
:10E950000048A3002700320000002100EAFF070062
:10E960000001EB006000B800AEC70200000000002C
:10E970008043EB0007437800874278000742780025
:10E980008741780007417800874078000740780089
:10E99000BAC60200000000008043EB000743780085
:10E9A0008742780007427800874178000741780065
:10E9B00087407800074078005EC702000000000032
:10E9C000202721000008EB000080E8000008EB0091
:10E9D0006CC30200000000000058A30002003200D7
:10E9E000A6C4020000000000D45F02000000000086
:10E9F000370237008EC8BF00E14F500008003200D8
:10EA0000E24F5000090032000004E0000C003A0020
:10EA10000001EB00F100200000022000060037009A
:10EA20000001EB000102200002003700020220007A
:10EA30008000EB00F0002000AEC7020000000000E4
:10EA40008FC8BF00E14F40001D003A008B48EC002A
:10EA50008BE8B700FC4F50000A003A0007C2B30031
:10EA600007437800874278000742780087417800A2
:10EA70000741780087407800074078005EC70200B1
:10EA80000000000080C3B3008B48E300380036006C
:10EA90008B68EF008043EB000743780087427800E3
:10EAA0000742780087417800074178008740780066
:10EAB000074078005EC70200000000002C0037000D
:10EAC0009C540200000000009C5402000000000062
:10EAD0009C54020000000000000478008843780085
:10EAE000084378008842780008427800884178001E
:10EAF0000841780088407800084078005EC702002E
:10EB0000000000008EC8BF00E14F50000800320036
:10EB1000E24F50000C0032000004E0000F003A0009
:10EB2000C545DD00C55DDE006F44B9000300370058
:10EB30006F40B900C505DE004544DD004545DE00F7
:10EB40008044EB00050037006F40B900C505DE00CA
:10EB50004544DD00C544DE000045EB000981FB00B3
:10EB60008A80FB000B80FB00AEC7020000000000A3
:10EB70008FC8BF00750032004240A90003003C006E
:10EB8000E14F4000B3013A0005003700E14F50006B
:10EB9000C9003200E24F5000AE013A008C0137004C
:10EBA00000FC22009080FB008100EA00CF08DE001C
:10EBB0000000EB000104E000040032004AC8BF007E
:10EBC0000080FB000000E9004F00DE00A28420006E
:10EBD000014978000000E000010032008E68ED007D
:10EBE00030FC22009080FB008100EA00CF08DE00AC
:10EBF0000000EB000104E0000400320049C8BF003F
:10EC00000080FB000000E9004F00DE00928420003D
:10EC1000014978000000E000010032008E68EC003D
:10EC200010FC22009080FB008100EA00CF08DE008B
:10EC30000000EB000104E0000400320048C8BF00FF
:10EC40000080FB000000E9004F00DE00828420000D
:10EC5000014978000000E000010032008E68EC00FD
:10EC600040FC22009080FB008100EA00CF08DE001B
:10EC70000000EB000104E0000400320047C8BF00C0
:10EC80000080FB000000E9004F00DE0072842000DD
:10EC9000014978000000E000010032008E68ED00BC
:10ECA0008EC8BF0009003B006CC3020000000000DA
:10ECB0000008A3000200320020C0B30001003700AA
:10ECC00010C0B3008EE8B7000A003700E14F5000D3
:10ECD000040034006CC30200000000000008A30020
:10ECE000030032008EC8BF00E24F50000100340024
:10ECF0008E68EF0020FC22009080FB008100EA007B
:10ED0000CF08DE000000EB000104E0000400320048
:10ED100046C8BF000080FB000000E9004F00DE0095
:10ED200062842000014978000000E00049013200BF
:10ED3000E188200091407800F288200001497800A5
:10ED400010C0B30091E8B7004201370000FC220078
:10ED50009080FB008100EA00CF08DE000000EB009D
:10ED60000104E0000400320045C8BF000080FB0041
:10ED70000000E9004F00DE00538420008149780044
:10ED80000000E000030032008D68EC00DEBD0200F0
:10ED90000000000030FC22009080FB008100EA00AF
:10EDA000CF08DE000000EB000104E00004003200A8
:10EDB00044C8BF000080FB000000E9004F00DE00F7
:10EDC00043842000814978000000E0000300320005
:10EDD0008D68ED00DEBD0200000000008DC8BF00A0
:10EDE00002003B008D68EF0004003700E84F500040
:10EDF0000200340080C0B3008DE8B700D188200045
:10EE0000914078008100FB0051868900C0FF2F00EF
:10EE10000088B900E40040007A8057006A815700FA
:10EE2000012878000100E00001003D000008EB002F
:10EE3000E4804000820F5000F9FF3A008FEB97000A
:10EE40002FEB9700CFEA97006FEA97008FF19700BA
:10EE50002FF19700CFF097006FF09700BAC602002D
:10EE6000000000008000EB0020FC22001004E00005
:10EE70000500320011892000914078008180FB005C
:10EE80008100E900CF08DE000000EB000104E00093
:10EE90000400320043C8BF000080FB000000E9000E
:10EEA0004F00DE0033842000814978000000E0003C
:10EEB000E8003200B5003700909380000000E000C9
:10EEC0006400320040FC22009080FB008100EA00D8
:10EED000CF08DE000000EB000104E0000400320077
:10EEE00042C8BF000080FB000000E9004F00DE00C8
:10EEF00023842000814978000000E00003003200F4
:10EF00008C68EC00DEBD02000000000010FC220056
:10EF10009080FB008100EA00CF08DE000000EB00DB
:10EF20000104E0000400320041C8BF000080FB0083
:10EF30000000E9004F00DE001384200081497800C2
:10EF40000000E000030032008C68ED00DEBD02002E
:10EF500000000000C1882000914078000104E0001A
:10EF600018003500FFCF50000E0034007FC1500064
:10EF70008043EB000743780087427800074278001F
:10EF800087417800F1C1B30007407800BAC602009B
:10EF90000000000020C3B3008C48E30025003400CB
:10EFA000180037008043EB00074378008742780061
:10EFB00007427800874178000741780007407800D1
:10EFC0001A003700FFCF400010003D00F7C1B3002A
:10EFD00016CEB300014353008042EB000542780097
:10EFE000854178000541780085407800054078002B
:10EFF000BAC6020000000000E0CCB3008C48E30079
:10F000000C003D008CE8B7000A0037008143EA009D
:10F010000043EB0086427800064278008641780083
:10F02000064178008640780006407800BAC60200A3
:10F03000000000008CC8BF000000FB00A10D2300F1
:10F040000310200083084000030178008180E8005D
:10F050008008510000FC22009080FB008100EA0043
:10F06000CF08DE000000EB000104E00004003200E5
:10F0700040C8BF000080FB000000E9004F00DE0038
:10F0800002842000014978000000E0000D003200F9
:10F090002027210001F82F00108040009093880065
:10F0A0004127210002F82F009108410011E82F00AC
:10F0B000810F500003003D0000E82F00909388006E
:10F0C000A093880030FC22009080FB008100EA00C1
:10F0D000CF08DE000000EB000104E0000400320075
:10F0E0003FC8BF000080FB000000E9004F00DE00C9
:10F0F000F3832000814978000000E0000C0032001A
:10F1000020272100030820001080410090938800F0
:10F110004127210091884100F1172000810F500004
:10F12000030034000018200090938800A09388000A
:10F130008000EB0020FC22001004E00005003200FB
:10F1400011892000914078008180FB008100E90056
:10F15000CF08DE000000EB000104E00004003200F4
:10F160003EC8BF000080FB000000E9004F00DE0049
:10F17000E2832000014978000000E0003500320001
:10F18000909380000000E0000C003A008FE8EF0050
:10F190008043EB00074378008742780007427800FD
:10F1A0008741780007417800874078000740780061
:10F1B000BAC6020000000000260037002027210008
:10F1C0000008EB000080E8000008EB002100370099
:10F1D0006CC30200000000000058A30002003A00C7
:10F1E0009EC40200000000008000EB0020FC220012
:10F1F0001004E000050032001189200091407800E1
:10F200008180FB008100E900CF08DE000000EB00F8
:10F210000104E000040032003DC8BF000080FB0094
:10F220000000E9004F00DE00D28320000149780091
:10F230000000E000070032006CC302000000000084
:10F240000058A30002003200A6C402000000000023
:10F250008FE8EF0020FC22001004E0001C003A00C0
:10F260001A00370010FC22001004E00017003200E2
:10F27000630040001004E000140032009148EC00EC
:10F2800091E8B70041C6B300814F5000100036002E
:10F290008140E800814F500009003A0010C0B300DF
:10F2A00090E8B7000040200097FD07008FE8EF00CE
:10F2B000508681008DE8B700D08681008CE8B700C9
:10F2C00060C6B30091E8B700010037009168EF0015
:10F2D0004F05BE004F04BE000080FA00000006008B
:10F2E00002882000124178008288AB0016003200AC
:10F2F000A19480000100E0000B0032000080FB00C0
:10F30000810F5000030034004300DE00804F5100A5
:10F31000030039000204E000040032000240E9006A
:10F3200080E8B700010037008068EF000188200006
:10F3300091407800814F510003003200E0C1B300DA
:10F34000DAC502000000000000000600E18720008E
:10F350000000E00003003D006700600091087000BD
:10F36000000006000080EA0091086000000006002E
:10F370000200FA00F0BF9F006101B900E40F5100E4
:10F38000E08F590010003E000260010004003700C9
:10F390000500370006003700070037000800370077
:10F3A000110888000E003700610888000C00370043
:10F3B000710888000A003700D1088800080037006B
:10F3C000E1088800060037008F81E9004210200024
:10F3D000014D2000C0132A00D8FA020000000000EE
:10F3E0000080FA00000006000200FA00F0BF9F0053
:10F3F000EA0F500019003E00120020000010DD004E
:10F4000082412000020160000D003A0000017800F6
:10F410006220B20003003A000008A30015003A0081
:10F420000E003700E1806000C308DD008008800026
:10F430000030A10000807000800888000D003700B7
:10F44000E1806000C308DD00F00880000030A1000A
:10F4500000807000F0088800060037008F81E90006
:10F4600042102000A1462000C0132A00D8FA020052
:10F47000000000000080FA00000006000200FA0010
:10F48000F0BF9F006101B900EA0F5100E08F590001
:10F490002F003E00026001000A0037001000370014
:10F4A000160037001C003700220037002800370004
:10F4B00027003700260037002500370008003700F6
:10F4C00015003700E3806000C408DD00F0FC2F0069
:10F4D0000401B60000807000200888002200370078
:10F4E000E3806000C408DD00F0FC2F001001B600CE
:10F4F00000807000800888001B003700E3806000F7
:10F50000C408DD00F0FC2F001201B600008070007E
:10F510009008880014003700E3806000C408DD0014
:10F52000F0FC2F001E01B60000807000F00888007B
:10F530000D003700E3806000C408DD00F0FC2F0000
:10F540002001B60000807000000988000600370026
:10F550008F81E90042102000214A2000C0132A00B8
:10F56000D8FA0200000000000080FA000000060047
:10F570000200FA00F0BF9F00401ADE0005002000E4
:10F58000E90F500003003200EA0F500007003A0074
:10F5900003003700620888007408880009003700FB
:10F5A000D2088800E4088800060037008F81E9004F
:10F5B00042102000A14F2000C0132A00D8FA0200F8
:10F5C000000000000080FA0000000600E80F500074
:10F5D000020034000000D00071005000000006005E
:10F5E0008000780010002000E88F500001003C00EF
:10F5F0000000EB00000006000200FA00889FBE0039
:10F600008A1F7800C0BF9F0000047800EC0F5400F0
:10F6100006003600E881570042102000E115200066
:10F62000C0132A00D8FA0200000000000800780089
:10F63000E6FF070000057800A93923004250DD00ED
:10F6400000804400900078000110A1000100A0009B
:10F650000108780008007800E1FF07000000E000E2
:10F66000040032000A05E8004255DD008A844400A7
:10F670001900A0004F0578004F04BE000080FA007A
:10F6800000000600D1FF07004200DD000080E80016
:10F6900081392300610078006100600000000600ED
:10F6A0000200FA00889FBE00D0BF9F0001047800CE
:10F6B00080047800EC8F540004003600E681570087
:10F6C00042102000E11920000B00370009007800EB
:10F6D000BEFF07004200DD000080E8008139230002
:10F6E000610078000018A30006003A00E681570088
:10F6F00032102000211A2000C0132A00D8FA02007C
:10F70000000000006148B900EA0F5000E08F580087
:10F710002A003E00006001000A0037000F00370099
:10F7200014003700190037001E003700230037008F
:10F730002200370021003700200037000700370083
:10F74000120037004F44DD002008800000F0A100C7
:10F7500000007400200888001C0037004F44DD00C2
:10F760008008800000F0A10000007400800888007C
:10F77000160037004F44DD009008800000F0A10023
:10F780000000740090088800100037004F44DD002E
:10F79000F008800000F0A10000007400F00888006C
:10F7A0000A0037004F44DD000009800000F0A1008E
:10F7B000000074000009880004003700E68157004B
:10F7C00042102000511C2000CBFF37004F04BE0028
:10F7D0000080FA00000006008000EB00B0FF370058
:10F7E00011002000AEFF37000200FA00F0BF9F00BA
:10F7F000CF80DE00EA0F5000E08F580018003E0076
:10F80000006001000A0037000C0037000D003700CF
:10F810000F003700100037001100370010003700CC
:10F820000F0037000E0037000300370007003700D5
:10F83000020888001000370043088800320888005A
:10F840000D003700520888000B003700B30888000D
:10F85000A208880008003700C208880006003700A8
:10F860008F81E90042102000D11E2000C0132A0021
:10F87000D8FA0200000000000080FA000000060034
:10F880003800FA00889FBE008A9FBE008C1F780057
:10F89000B0AF9F00C2AF9F00D3AF9F00E1AF9F000A
:10F8A0006000B8006011B800F09F9F0081A79F0022
:10F8B00092A79F00A3A79F0060FC2F000080470035
:10F8C00081152A000700090031187800BFAC9700A5
:10F8D000EC8F54000500360063FD2F008F8141003E
:10F8E00042102000211020000C0037000900780091
:10F8F00036FF07004200DD000080E8008139230068
:10F90000610078000018A30007003A0063FD2F0093
:10F910008F8141003210200061102000C0132A00A6
:10F92000D8FA0200000000006FAC97000800E00069
:10F9300013003200E30F540011003200E60F5400B0
:10F940000F003200E90F54000D003200E10F4400B7
:10F950001D003200E20F44001B003200E30F4400A0
:10F9600019003200E40F440017003200C3FD2F00DD
:10F970008F81410052102000B1102000E7FF3700B6
:10F980004FA89700DFA897006011B8000005EB00B2
:10F9900006003700A4002000050020006033B800F6
:10F9A000A6040200000000000A05E8006902140035
:10F9B000840F5500F7FF3500F09F9F0081A79F003F
:10F9C00092A79F00A3A79F00E88F54007A003C00F5
:10F9D0008040EB000900780083FE07006FAE9700BF
:10F9E0000C00E000610035007F9C97008FA4970019
:10F9F0001FA59700AFA59700F8F9020000000000CE
:10FA00000002BE006033B8000440E10005C8E10018
:10FA100006D0E10007D8E100150039007F9C97006F
:10FA20008FA497001FA59700AFA59700F8F90200D3
:10FA3000000000006011B80004F02F00F50F200056
:10FA40006033B800A6040200000000000040E1009E
:10FA500001C8E10002D0E10003D8E10004003E004B
:10FA60002AFC2F000F0545000006EB0006003700BA
:10FA7000E3FB2F008F81410012102000D1112000E4
:10FA8000A6FF37000C06E8007F9A97008FA2970028
:10FA90001FA39700AFA39700F4AF9F0085B79F0007
:10FAA00096B79F00A7B79F00F8F90200000000007A
:10FAB0000004BE005A00BE006011B800B0B79F003D
:10FAC000C1B79F00D2B79F00E3B79F00F4FF2F009C
:10FAD000050020006033B800A6040200000000000A
:10FAE0000802BE006033B800A60402000000000057
:10FAF0007FAA97008FB297001FB39700AFB397000C
:10FB00000020E10001A8E10002B0E10003B8E1003B
:10FB1000DCFF3E007F9C97008FA497001FA59700F5
:10FB2000AFA59700F8F90200000000006011B800CE
:10FB30003FB29700CFB297005FB39700EFB3970043
:10FB4000A6040200000000000203BE000002BE0086
:10FB50000800BE000A01BE00C80502000000000047
:10FB60000205BE000004BE000C0037004FAC970039
:10FB7000DFAC9700E10F4400E08F5C000500360029
:10FB800083FD2F008F814100121020007112200090
:10FB900062FF37000C86EA006055B8008C007800E0
:10FBA0003FA8970035FE0700880078003FA897001F
:10FBB000EFFD07007600370011C0B30009007800A0
:10FBC00009FE07006FAD97000A00E00060003500F5
:10FBD0007F9C97008FA497001FA59700AFA5970063
:10FBE000F8F90200000000000002BE006033B80017
:10FBF0000440E10005C8E10006D0E10007D8E100BB
:10FC0000160039007F9C97008FA497001FA59700CE
:10FC1000AFA59700F8F90200000000006011B800DD
:10FC200004F02F00F5FF2F00F60F20000700200042
:10FC3000A6040200000000000040E10001C8E1004D
:10FC400002D0E10003D8E10004003E002BFC2F00AD
:10FC50008F8545000005EB0006003700E3FB2F0011
:10FC60008F81410012102000A11320002BFF3700CC
:10FC70000A05E8007F9897008FA097001FA19700C2
:10FC8000AFA19700B0B79F00C1B79F00D2B79F0048
:10FC9000E3B79F00F8F90200000000005B04BE001B
:10FCA0000801BE009A040200000000000002BE002D
:10FCB0006033B8003FB09700CFB097005FB19700B6
:10FCC000EFB19700C805020000000000F4FF2F000C
:10FCD000F5FF2F006033B8000400E1000588E10063
:10FCE0000690E1000798E100E1FF3E007F9A97004F
:10FCF0008FA297001FA39700AFA39700B4B79F00F0
:10FD0000C5B79F00D6B79F00E7B79F00F8F902007C
:10FD1000000000000002BE006033B8003FB0970052
:10FD2000CFB097005FB19700EFB19700C805020010
:10FD3000000000000802BE006033B800C8050200E1
:10FD4000000000000203BE000002BE0004003700F5
:10FD50000A85EA004FAA9700DFAA97006033B8002F
:10FD60008A0078003FA89700F4B79F0085BF9F00E6
:10FD700096BF9F00A7BF9F00C0FD07007FB29700FE
:10FD80008FBA97000401BE003FA89700F8FD070056
:10FD90006011B8003FA8970093FE07004F06780057
:10FDA0004F05BE004F04BE000080FA0000000600B0
:10FDB0000200FA00F0BF9F00CF80DE00EA0F500083
:10FDC000E08F58001F003E00006001000A0037006D
:10FDD0000B00370010003700110037001700370004
:10FDE00018003700170037001600370015003700DD
:10FDF000060037000C0037000008800001003700C3
:10FE0000300880008000EB001400370032088000CA
:10FE1000400880000600370050088000F9FF3700D6
:10FE2000A0088000F7FF3700A2088000B00880001B
:10FE3000800078000200780008003700C0088000C9
:10FE4000F0FF37008F81E90042102000512120008F
:10FE5000C0132A00D8FA0200000000000080FA0057
:10FE6000000006000400FA00E0BF9F00F1BF9F0001
:10FE7000E18F5000040036008F81E90062102000FD
:10FE8000912220003E0037006FB99700CF91DE002D
:10FE9000EA0F5100E08F590036003E000260010079
:10FEA0000A00370012003700190037002100370020
:10FEB000280037002F0037002E0037002D003700B4
:10FEC0002C0037000900370019003700E18060007E
:10FED00081804000200880000010A1000080700098
:10FEE0002008880005A1A9002800370013A1A90057
:10FEF000E180600081804000800880000010A10047
:10FF0000008070008008880011A1A9001F00370040
:10FF1000E180600081804000900880000010A10016
:10FF2000008070009008880013A1A9001700370016
:10FF300021A1A900E180600081804000F0088000DC
:10FF40000010A10000807000F00888001FA1A90027
:10FF50000E003700E18060008180400000098000D1
:10FF60000010A100008070000009880021A1A900F4
:10FF700006003700E48157004210200011262000BF
:10FF8000C0132A00D8FA0200000000000080FA0026
:10FF9000000006000200FA00F0BF9F006101B900F6
:10FFA000EA0F5100E08F59002F003E00026001006F
:10FFB0000A00370010003700160037001C00370019
:10FFC00022003700280037002700370026003700BE
:10FFD000250037000800370015003700E180600079
:10FFE000C608DD00200880000060A10000807000CD
:10FFF0002008880022003700E1806000C608DD008C
:020000040001F9
:10000000800880000060A1000080700080088800E7
:100010001B003700E1806000C608DD00900880000A
:100020000060A10000807000900888001400370074
:10003000E1806000C608DD00F00880000060A100DB
:1000400000807000F00888000D003700E18060003B
:10005000C608DD00000980000060A100008070007B
:1000600000098800060037008F81E9004210200057
:1000700041292000C0132A00D8FA02000000000025
:100080000080FA00000006000400FA00889FBE000D
:100090008A9FBE00A0BF9F0001047800B2BF9F00EE
:1000A00000057800EC0F550004003600EC81570085
:1000B00042102000812A200007003700BFBC9700B3
:1000C0000900E900E60F500006003600EA815700FB
:1000D00022002000912A2000C0132A00D8FA020032
:1000E000000000000A00780038FD07004200DD0033
:1000F0008139230088307800CFD5DE00EA0F550023
:10010000E08F5D0037003E000A6001000A00370002
:10011000120037001A00370021003700290037008D
:10012000300037002F0037002E0037002D00370039
:100130001300370023003700E7846400CC4CDD0057
:10014000F0FF2800A400B60000807400200588009D
:100150008460A9009460A80026003700E78464004A
:10016000CC4CDD00F0FF2800A600B6000080740033
:100170003005880084E0A90094E0A8001D00370045
:10018000E784640080FF2F00A800B60000807400A0
:10019000400588008500A9009500A80015003700DB
:1001A000E7846400CC4CDD00F0FF2800B000B6000E
:1001B00000807400800588008760A9009760A8000F
:1001C0000C003700E784640080FF2F00B200B60007
:1001D00000807400900588008780A9009780A8009F
:1001E00004003700EC81570042102000D12E20007F
:1001F000B9FF37004F05BE004F04BE000080FA0073
:10020000000006000200FA00F0BF9F00CF80DE0071
:10021000EA0F5000E08F58002A003E000060010005
:100220000A0037000F0037001400370019003700AC
:100230001E0037002300370022003700210037005E
:10024000200037000D00370018003700A0048000A0
:100250004300DE00610060009460A8008460A80094
:100260001E003700A00480004700DE00610060002F
:1002700094E0A80084E0A80018003700A0048000E3
:100280004800DE00610060009500A8008500A8001D
:1002900012003700B00480004B00DE0061006000F7
:1002A0009760A8008760A8000C003700B0048000A9
:1002B0004C00DE00610060009780A8008780A800E5
:1002C000060037008F81E90042102000F133200042
:1002D000C0132A00D8FA0200000000000080FA00D3
:1002E000000006000200FA00F0BF9F00CF80DE0091
:1002F000EA0F5000E08F58001E003E000060010031
:100300000A0037000C0037000E00370010003700DD
:1003100012003700170037001600370015003700AD
:1003200014003700070037000C003700200480005D
:100330004300DE000B003700200480004700DE0091
:1003400008003700200480004800DE000500370068
:10035000300480004B00DE000200370030048000D3
:100360004C00DE00610060000080FA000000060022
:10037000060037008F81E90042102000113720006D
:10038000C0132A00D8FA0200000000000200FA00A0
:10039000F0BF9F006101B900EA0F5100E08F5900E2
:1003A00038003E00026001000A00370011003700EB
:1003B0001A003700210037002800370031003700CD
:1003C000300037002F0037002E00370013003700B1
:1003D00022003700200480004300DE00610060003E
:1003E000E1806000C308DD00220480000230A1002B
:1003F00007003700200480004700DE006100600035
:10040000E1806000C708DD00220480000270A100C6
:100410000281700022048800200037002004800040
:100420004800DE0061006000E1806000C808DD0077
:10043000220480000280A100F5FF37003004800014
:100440004B00DE0061006000E1806000CB08DD0051
:100450003204800002B0A1000700370030048000A1
:100460004C00DE0061006000E1806000CC08DD002F
:100470003204800002C0A1000281700032048800B2
:10048000060037008F81E90042102000613B200008
:10049000C0132A00D8FA0200000000000080FA0011
:1004A000000006000200FA00F0BF9F00CF80DE00CF
:1004B000EA0F5000E08F58001B003E000060010072
:1004C0000A0037000C0037000E003700100037001C
:1004D00012003700140037001300370012003700F5
:1004E00011003700070037000C0037009460A900A6
:1004F0008460A9001200370094E0A90084E0A900FC
:100500000F0037009500A9008500A9000C003700F6
:100510009760A9008760A900090037009780A900AB
:100520008780A900060037008F81E9004210200073
:10053000913F2000C0132A00D8FA020000000000FA
:100540000080FA00000006000600FA00889FBE0046
:100550008A9FBE008C9FBE00F0B79F008106780086
:1005600000057800EC0F550004003600F2815700BA
:1005700042102000210C2000100037000A007800F3
:1005800082BF9F0093BF9F0010FC07000006780009
:100590004264DD000880E8008139230061007800B2
:1005A0000FB997009FB997000008A30006003A0012
:1005B000F281570022102000610C2000C0132A0095
:1005C000D8FA020000000000AB392300088445007F
:1005D000980478000910A0000900A100090C780017
:1005E0000A00780082BF9F0093BF9F00FCFB0700BA
:1005F0000FB997009FB997000000E0000600320095
:100600000C06E8004266DD008C8545001B00A10059
:100610001820A000020037000920A100090C780072
:100620007FB0970082BF9F0093BF9F009DFF070090
:100630008D0078000FB997009FB997007FB09700A1
:100640008FFC07008000EB007FB0970005FE0700DD
:100650008000EB007FB097004EFE07004F06BE0003
:100660004F05BE004F04BE000080FA0000000600E7
:100670000200FA00F0BF9F00CF80DE00EA0F5000BA
:10068000E08F58001B003E00006001000A003700A8
:100690000B0037000C0037000D0037000E0037004C
:1006A0001400370013003700120037001100370024
:1006B00003003700060037002108800007003700DC
:1006C0008108800005003700910880000300370092
:1006D000F10880000100370001098000C408DE0035
:1006E000E380600000042000E28F500007003A0021
:1006F0000D0037008F81E900421020009142200058
:10070000C0132A00D8FA02000000000000102000E8
:10071000E38F50000400320080002000E18F500081
:1007200001003200100020000080FA0000000600E6
:10073000AA24AB000D0032003082800010419000EE
:1007400001C8B300814F510007003A008182800048
:100750001141900041C8B300814F510002003A009E
:10076000E8C0400011409800AA24A9000008200019
:10077000502488000000060000C8B30001032100D7
:10078000914F10002E003A00C005210001CCB300AB
:10079000014878003103210091407800E2CF5000F9
:1007A00008003200E3CF500015003200E1CF5000C6
:1007B00022003A0000122100D0828800200120008F
:1007C0001A003700200321001080FB0000004000C9
:1007D000E11B2100E1007800D1828800D1828000F5
:1007E000E0052100A140900001487800D1828000FE
:1007F0000000E800B14090000148780000000600C9
:100800002103210022C0B300914F110009003E00D6
:100810001180FB0000004000011C2100E100780075
:10082000D1828800D08280001080FB00F082880096
:10083000000006000048EB00000006000048EB0046
:1008400000000600800321000048EB008000E80063
:100850008048EB000103210091407800FFC0600058
:100860008180FB00E18F50000D003200E28F5000CC
:100870000F0032000100E00025003A00E182800014
:100880000170A000E18288001004A00011848000A3
:10089000E18F50001E003A001014A0001C00370029
:1008A000E08280000070A000E0828800180037001D
:1008B000E08280000070A000E082880040032100F8
:1008C0001004E00006003500104078006F40600022
:1008D0000080FB0000004000A1042100050037005B
:1008E000104078006F4060000080FB000000400076
:1008F0000105210061007800104090000028A3004D
:100900000300320011C0B3008003210001487800C9
:10091000E08280000078A3000800320080032100FC
:10092000D0828800E08280000000A000E082880081
:1009300021C0B300E0052100014878000000060056
:10094000F182800080C0B300E78F50000B003E00B2
:10095000F082800011C0B3005650E2000500320062
:100960006105210091407800E1CF500003003A007A
:1009700021C0B3006205210001497800F2828000A5
:100980008080FB0081005100F1828800818280001C
:10099000804878008103210041838800E182800043
:1009A0000108A300070032000F003700D182800049
:1009B000428380003159780042838800D1828800C8
:1009C0000040E9000004E000F8FF3A0000000600E3
:1009D000D1828000428380003159780042838800B0
:1009E000D18288000040E9000004E000F8FF3A00EE
:1009F00000000600881F7800000521008182800029
:100A0000110478004E44DE00614464001024A2000A
:100A100000828000E80F500008003A002003210007
:100A20001080FB00B0248800000120009604E20042
:100A300001003A00400020000082880058D0BF002A
:100A4000E14F500011003A008103210080828000B4
:100A500011009800BAFF070061052100914078005D
:100A600080828000E2CF500002003A0041C8B3000B
:100A70000400370081CCB3000804E000010032001C
:100A800081C8B300114098001200370020062100F1
:100A90001004E0000E003D00E30040009181FB00E7
:100AA000640040001081FB004811DD0002817100EC
:100AB000050032009180FB001080FB004800DD0043
:100AC0000080700000000100200621001074A100C9
:100AD0005870EF004F047800000006000080FB0013
:100AE0000181FB0000004000000141004311DD00D6
:100AF000030021000301410012F0A1000104E00005
:100B000002003A00A1042100010037000105210084
:100B10008230780012E0A1006401410012E0A000E0
:100B2000000006008430EF000001EB008000EB00C5
:100B30004007200030F50200000000008284A90078
:100B40000001200000248800000006008284A80024
:100B5000000120005024880010002000208488001C
:100B60000001EB008000EB005007200030F504008E
:100B7000000000000200FA00881F78002003210016
:100B800011C0B30090CF10000F003A000080E900C0
:100B9000104078007F4060000B003A00E082800047
:100BA0000070A000E08288001003210032C0B30072
:100BB000904F110003003A001000200010848800BC
:100BC000010037008230EF00200321001004E00014
:100BD0009A003A000080E900104078007F406000F1
:100BE000E24F500095003A00400321001041780088
:100BF000EF4061009100320010417800EF40610049
:100C00008180FB00E28F50008C003C00010220003C
:100C100002828000810F510088003A00E18280004A
:100C20000170A000E18288001004E0000C00350093
:100C300010417800EF4061008180FB00818040001E
:100C4000A204210062817800E2BF9F00104078007A
:100C50006F4060000080FB00210721000B0037007F
:100C600010417800EF4061008180FB0081804000EE
:100C70000205210062817800E2BF9F0010407800E9
:100C80006F4060000080FB00E106210061447800B5
:100C90000808A30004003A004FF897000024A100C0
:100CA000C0FF9F0003003700CFF897000124A00089
:100CB000C1FF9F00400321001004E0000600350042
:100CC000104078006F4060000080FB000000400092
:100CD000A104210005003700104078006F4060003B
:100CE0000080FB0000004000010521006FB9970063
:100CF000823078001003210031C0B30090CF100083
:100D000017003A006FB897001000E0000F003D0098
:100D1000400321001004E000050035001040780079
:100D2000EF4060008180FB002207210004003700B3
:100D300010407800EF4060008180FB00E206210057
:100D400062C078000014A00000F178006FB897002E
:100D50001041900041C8B300814071003600370057
:100D60004FF997000224A200C2FF9F00EFB897003E
:100D7000114090001100E00008003D000074A10047
:100D80000064A00090409800220020005000200045
:100D900030F5020000000000020037000064A000EF
:100DA000904098004FF897000024A200C0FF9F00D9
:100DB0000818A30006003A006FB897000240280008
:100DC0001001610001002800810F510018003A0055
:100DD000400321001004E0000500350010407800B9
:100DE000EF4060008180FB002207210004003700F3
:100DF00010407800EF4060008180FB00E206210097
:100E000062C078000014A10000F17800EFB89700EC
:100E100011409000B043B2009040980022002000A2
:100E20005000200030F502000000000003003700F1
:100E300090409000B143B200114098004F047800F8
:100E40000080FA0000000600E08280000070A00030
:100E5000E0828800AC24EF00AE24EF000000EB003D
:100E6000010021004201DD00028140000009EB0089
:100E7000321178000000E800EC0F5000F8FF3A0053
:100E80009424A8004470EF009424A90068804000D6
:100E900080828800318288004182880020032100FE
:100EA00010417800210421008248780000012000D0
:100EB0004250E2000600320012002000210421000E
:100EC0001000200030F502000000000000022000A9
:100ED00000828800000006000003210001C6B30064
:100EE00010C060003C003A00100321001080FB009D
:100EF0008000EB00EB0F5000E08F580036003E0002
:100F0000006001001500370015003700320037007F
:100F10001300370030003700060037000B003700A1
:100F2000280037000B003700090037000D0037009C
:100F30001B003700E08280000070A000E082880083
:100F40008000200000828800000006000AFE3700B2
:100F5000BDFF3700200421000600370039FE3700AE
:100F600004FF3700400321009080FB004004210073
:100F700000804000D0828800E08280000000A00055
:100F8000E082880011C0B300E0052100014878002C
:100F9000E08280000070A000E0828800000006006F
:100FA000E08280000070A000E08288004003210001
:100FB0001080FB0041042100220321009270780080
:100FC000000006000001EB008000EB002000200084
:100FD00030F5020000000000000006009EC0A900DD
:100FE0008EA4EF008AA4EF00AA24EF00AC24EF0047
:100FF000AE24EF002000200030258800A824EF0058
:101000008644A900F009200080248800602488001C
:101010008804A800000021004800DE00C0248800E9
:101020000000EB00C200DD00020021008100410051
:101030008008EB00B11078000000E800EC0F5000D1
:10104000F8FF3A009424A8009624EF0094A4A90085
:101050009424A9000C003700800020005024880050
:10106000C00521000048EB00200621000048EB00ED
:101070000000E800904078000048EB000000E80025
:10108000904078000048EB008A64AB00F2FF3A0021
:1010900010002000C0838800D08388007C30EF00DF
:1010A0007E30EF008430EF00E20421008104210053
:1010B0000000EB008001EB000029EB008028EB0032
:1010C000E4062100037278002407210003727800EF
:1010D0000000E800E30F5000F6FF3A008000210016
:1010E00080828800D0002000502588000003210065
:1010F0001080880081C0B300000021000148780002
:1011000041C8B3000000E800014878004270EF00D9
:101110004030EF00000006007810E20023003A00A3
:1011200010002000C08388007A10E2001F003A00FF
:10113000D08388008105210091407800E2CF5000E3
:1011400006003A00808280000048EB0081CCB300AA
:101150008082800011409800000006008105210077
:1011600091407800E1CF500010003A008030EF004D
:1011700082C0B300318280008248780033828000D0
:10118000010321009101980044C8B30094419800E4
:1011900000848800408280000248780040828000FD
:1011A0001100980001C8B30011409800000006002B
:1011B0003082800090407800320621001282FB00CD
:1011C0000200E8009081FB00C819DD008301720075
:1011D0000182FB00830F5200020036009280FB0068
:1011E0001080FB00320621001282FB000200E800A2
:1011F0009081FB00C819DD00830172000182FB00B1
:10120000848151001242780003497800C819DE0039
:1012100010417800034878000000EB000E00370012
:10122000040621009482FB008401E8001381FB0086
:101230004811DD00028172008503210065597800A4
:1012400094427800024A78004811DE001342780088
:10125000824978000000E80080CF5000F0FF3E0097
:10126000300621001080FB00410621009180FB0028
:10127000C808DD0081007000408280000D0032004F
:1012800081C0B300014878004082800081032100C2
:10129000110098003182800011E8A30002003A009A
:1012A00081CCB3000100370081C8B3001140980021
:1012B0000000060081C0B300014878004082800031
:1012C000010321001100980041C8B30011409800AB
:1012D000510621009181FB000100E8001081FB0014
:1012E0004811DD0002817100050032009180FB0091
:1012F0001080FB004800DD0000807000000001004D
:10130000200621001074A1007610E20001003A00CE
:1013100081FF07000000060058D0BF00E24F5000D8
:1013200001003A00A2FF37005870EF008010E20081
:1013300009003A0081C0B300408280000148780073
:10134000408280000103210011009800C1C8B30051
:1013500011409800000006008030EF0000000600F9
:101360007C30EF007E30EF0058D0BF00E24F5000DD
:1013700008003A0081C0B300408280000148780034
:1013800040828000810321001100980081CCB300CD
:1013900014003700610321001181FB000100E80007
:1013A0009081FB00C819DD0083017100F28280008A
:1013B000828F5100050031009180FB001080FB00FE
:1013C0004800DD0000807000F08288005CFD0700AE
:1013D00081032100808280001100980081CCB3003D
:1013E00080828000114098000000060094A4A900AB
:1013F000E08280000078A30017003A002006210058
:101400001004E00008003D0020C0B30058F0B70011
:101410007E10E20001003A00D1FF07007A30EF00B1
:101420007830EF000000060081C0B30040828000E9
:1014300001487800408280000103210011009800DB
:10144000C1C8B30011409800E8C0500080828000FD
:101450001140980000000600010321001104E00083
:101460000A003D0010C0B30058F0B7007C10E20045
:1014700001003A00BAFF07007A30EF007830EF0041
:101480007610E2000F003A0023FF370020C0B300BF
:1014900058F0B70082C0B300408280000248780054
:1014A000408280001100980041C8B30011409800AC
:1014B0007A30EF007830EF007610E20001003A0059
:1014C00015FF0700000006005670EF007630EF00B1
:1014D0007C30EF007E30EF008030EF005870EF007E
:1014E0000005210010017800924090000174A100D5
:1014F000114198001024A200100178009240900041
:101500000174A100114198001024A20041828000C2
:10151000114090000074A10090409800C005210087
:101520000048EB000000EB00F0828800210621005B
:10153000804878008100E8001141780080487800F8
:101540008100E800114178008048780062FE0700C1
:101550000001EB008000EB003000200030F50200BD
:1015600000000000A1FF3700D0C2B30086F0B70032
:101570006CD0BF00B00FB2001A003A006CD0BF00B0
:10158000C00FB2000100210001004000308288003D
:10159000408288004850AA0002C023001001610068
:1015A00001402300810F51000D003A00010321008A
:1015B00001017800E8814000100290009458780002
:1015C000100290000402E80014009800838F50007D
:1015D000F9FF3A003082800012009800BAFF37000D
:1015E0004DFF37006CD0BF00B00FB200E80F5000C5
:1015F00001003A00FFFC070000000600889FBE00C3
:101600008A1F780000447800814478000985FB0037
:101610000A38A300030032008040EB000840780045
:101620002EFD07000A28A3000300320011C0B300FA
:101630000840780029FD07000884FB0008044400E6
:10164000A04A200009707C004F0578004F04BE00BE
:10165000000006000004E0000B003A0081C0B30067
:101660004082800001487800408280000103210010
:1016700011009800C1C8B30011409800E8C05000A4
:10168000808280000F0037008180FB000080FB001B
:1016900000004000008040004300DD000200210007
:1016A000820140001342900041C8B3000142720021
:1016B00094419800640040000200400010419000F6
:1016C0008140710011409800000006000082FB007C
:1016D0000104E0000300320004024200050521007D
:1016E0000200370004024200A504210065027A00CE
:1016F0008002EB000400E0001400320012029800A7
:10170000034A7800144190000244B200124298004B
:101710009441900082C8B30002C171001242980047
:101720000080FB000104E0000300320000004000E4
:10173000010521000200370000004000A104210043
:10174000010040001024A200840278000500780007
:101750000000060094A4AB00170032000080FB00DC
:101760000000400001052100610178001203BE0065
:1017700004042000060362008003EB000689BE001B
:10178000E10278001501BE000260A200828ABE005C
:10179000010140001224A2006101780092419000F2
:1017A0000344B2001341980061007800904090001B
:1017B00004C2680014409800000006009424EF0062
:1017C0008C24EF004030EF00000006004010E200E3
:1017D00010003A009424EF008C24EF002000200039
:1017E00030258800A824EF008644A900F0092000D5
:1017F00080248800602488009EC0A8000100370073
:101800009404A8009404AB00FDFF320010002000F7
:101810000082880000000600A0009000910078007F
:10182000818040001C0037000181400020029000B0
:1018300002024200940278004C29DE008001EB0095
:1018400062015100E0815900E90F5100E08F590019
:1018500011003E00026001000B0037000E0037004F
:101860000D00370008003700070037000A00370076
:101870000900370008003700010037000400370076
:101880000590A100050A78008180E8000300370078
:10189000E3804000010037008100E8001001900063
:1018A000828F5000E0FF390000000600E10F510078
:1018B0000600320003003900E20F510009003A002F
:1018C000060037000100EA00000006000100780071
:1018D00000F0A7000000EA00000006000180EA0016
:1018E0000000060011002000EABC02000000000019
:1018F00000000500881F780000047800611AB80015
:10190000F10F5200E08F5A0064003E0004600100B5
:1019100011003700120037001300370014003700A1
:1019200015003700160037001A0037002E00370068
:101930002F00370030003700310037003500370006
:101940003A0037003D0037004000370043003700C1
:1019500046003700490037000208DD005400370018
:101960000288DE00520037000100410050003700BD
:10197000028050004E0037000190B9004C00370043
:101980000200E00005003200110009008200D800CA
:10199000470037000200E0000F003A0000A02900D5
:1019A0000000E000040032008000EB000800780036
:1019B000009A020000000000230020007304980039
:1019C0007001440071002900080078001CD3020057
:1019D0000000000035003700110009008200D80027
:1019E0008000FD00320037000280700030003700B8
:1019F000010069002E003700010061002C00370053
:101A00008280680001F0A7008100EA008100E900FF
:101A1000040037008280680001F0A7008100EA001E
:101A20008100EA004F08DE0021003700100020008E
:101A3000828F50001E003C001C0037001000200068
:101A4000828F50001A003D0018003700100020005F
:101A5000828F50001600350014003700100020005F
:101A6000828F500012003400100037001000200058
:101A70000100E000040032000D0037000000EB0020
:101A80000100E0000A00320002F0A7000201EA00B3
:101A90000200EA004F00DE000500370021002000B0
:101AA00008007800EABC0200000000000000EB0023
:101AB0004F047800000006008000EB000108980049
:101AC0007100980021189800200190000109780009
:101AD00030019000020141004000900060070400C6
:101AE000000000002001900092017800100020000A
:101AF000090037000002400062027A00810F5200A4
:101B000004003A000000E800000040006200780095
:101B1000000006000080E800830F5000F5FF390048
:101B2000000005000600FA00889FBE008A9FBE00E4
:101B30000004780008089000A80090000000400011
:101B4000E1047800780090000008A30004003A0047
:101B50008100200008007800EABC020000000000BC
:101B60004C48DE008000EB00EE0F5000E08F580084
:101B700077013E00006001000E00370011003700C1
:101B80002100370038003700550037006E0037005D
:101B90008A003700BB003700CB003700E200370077
:101BA000EF003700250137003F01370044013700BF
:101BB00058013700780090000000A10070049800E0
:101BC00067013700C44CDD00C4CCDE0098089000EB
:101BD0008100E80058009000808F50000400390018
:101BE0004100200008007800EABC0200000000006C
:101BF000E8009000180890000000E800100C980021
:101C00000000400032003700980890008100E80092
:101C100058009000808F50000400390041002000DF
:101C200008007800EABC0200000000006801900093
:101C3000180890000000E800100C98000000400018
:101C4000880890008100E800A80190008180400091
:101C5000E380780001317800080890000080E800F7
:101C6000000C98003E013700F0FF200080846400E3
:101C7000980890008100E80058009000808F500084
:101C8000040039004100200008007800EABC02008E
:101C90000000000038009000808F540004003900DC
:101CA0006100200008007800EABC0200000000008B
:101CB000E8009000180890000000E800100C980060
:101CC000000040004801900089844400E2847C00C8
:101CD00089307800080890000000E800E0FF370035
:101CE000F0FF200080846400180890000000E000ED
:101CF00004003D005100200008007800EABC02000A
:101D00000000000038009000808F5400040039006B
:101D10006100200008007800EABC0200000000001A
:101D200018089000C800900089844400E8019000E1
:101D3000000140006301790082B07C000000E900EE
:101D4000100C9800E3FF3700180890000000E00036
:101D500004003D005100200008007800EABC0200A9
:101D600000000000880990000300E800A80090002F
:101D700000004000610178009808900081804000D8
:101D8000680090008100400011007800820F500030
:101D90000300390093BF9F00A2BF9F001E003700C1
:101DA000F2FF200082846400090040004801900096
:101DB00000004000E2087800A7FF370018089000F4
:101DC0000000E00004003C00510020000800780002
:101DD000EABC020000000000080990000200E800D0
:101DE000A800900000004000E1007800E8019000A9
:101DF000180890000002E9000402420063027A0021
:101E00000000400063007800810F5000130039008B
:101E100092BF9F00A1BF9F00B0BF9F002000200085
:101E200070049800630020006E8157006100290053
:101E3000080078001CD302000000000000A0290068
:101E40000000E000C60032008000EB0008007800CF
:101E5000009A020000000000C1003700F1FF2000DE
:101E60008184640009004000C80090000000400028
:101E700084307800180890000080E900100C980069
:101E800075FF3700180890000000E00004003D00D6
:101E90005100200008007800EABC020000000000A9
:101EA00009017800F20FB20018089000E8009000D5
:101EB00000004000E1007800080078007BFE070089
:101EC0009808900014003700180890000000E00007
:101ED00004003C005100200008007800EABC020029
:101EE0000000000068009000980890000181400008
:101EF0008100E900818040008981FB006001790058
:101F0000E0807800080078007AFE070098089000CA
:101F10008100E900110C9800680190008180400068
:101F200000B178006BFF3700C44CDD00C4CCDE008C
:101F3000880890008180440018009000808F500035
:101F4000040039007100200008007800EABC02009B
:101F50000000000008089000890440006B00370072
:101F6000180890000000E00004003C005100200030
:101F700008007800EABC0200000000006800900041
:101F800098089000018140008100E90081804000B4
:101F90008981FB0060017900E0807800080078000A
:101FA00054FE0700980890008180E900110C980009
:101FB000880890000000E000050032000930B200FF
:101FC0002A00200002302000828F540006003A00D0
:101FD000280190008101E800838141006285790039
:101FE0000000E000050032008180400028009000E1
:101FF000810040001190A000030037008180400064
:10200000810041001190A1008808900081004500E6
:1020100018009000808F50000400390071002000EB
:1020200008007800EABC02000000000008089000E8
:102030000A0540000A0C980049003700280090006B
:10204000880890000101E80002014100E0057900E4
:102050008180E80081804000608578004020200079
:10206000800F550004003600A10020000800780011
:10207000EABC0200000000008B854500480190008A
:102080000B014100F1FF2000818064008A014500BE
:10209000080078001CD3020000000000080890002F
:1020A00063004000EEFE3700F1FF200081806400F5
:1020B000080078006CBB02000000000005FF37003C
:1020C000F0FF200080846400980890008100E80000
:1020D00058009000808F500004003900410020001B
:1020E00008007800EABC020000000000E800900050
:1020F000180890000000E800100C98000000400054
:1021000000804000880890000108E800090C980051
:1021100013003700180890000000E00004003D00A4
:102120005100200008007800EABC02000000000016
:10213000180890006801900080004000E28078005C
:10214000010C98000000E900100C98000400370012
:102150003100200008007800EABC02000000000006
:102160004F05BE004F04BE000080FA0000000600CC
:102170000000FA00889FBE008A9FBE008C9FBE00B0
:1021800000047800810578000F0578000B007800C6
:102190006E0702000000000080067800638646009B
:1021A000658046000000A100808747008A0478000F
:1021B00000A029000000E000040032008B0078003D
:1021C00008007800009A02000000000020002000B3
:1021D0007004980008089000800C7800AD449800C6
:1021E000638044000D0178008B00780052070200E4
:1021F000000000008C01780009017800910029009E
:10220000080078001CD30200000000008A07780054
:102210004F06BE004F05BE004F04BE000080FA000E
:1022200000000600A0199000000178008000EB007B
:102230000A003700A20A90000281E800000A90001C
:10224000848F520004003A00F00090000110A000BA
:1022500071009800100005008100E800838F500095
:10226000F4FF390000000500889FBE000004BE0096
:10227000780090000020A000700498000900E000A1
:102280000D003200030037000800780025FE07002B
:102290008904E9007800900065006000E50F5000B7
:1022A00009003A000900E000F7FF3A000600370095
:1022B000080078001BFE07007800900065006000B1
:1022C000E50F5000FAFF3200780090000020A100D6
:1022D000700498004F04BE0000000600889FBE00F6
:1022E0000004BE0018009000808F540004003900E4
:1022F0009100200008007800EABC02000000000005
:10230000A81890000040EB00EF8F500006003E0040
:102310006A80400000004000093478008100E80035
:10232000211C980010C0B3004F04BE00000006003E
:10233000201A9000800178000001EB0012003700A5
:10234000A30A90008381E800818F52000D003A00BB
:102350008401E90023189800EA00410081804000D0
:1023600001004000040037000201E8000080E8009E
:102370009000780071B89F00830F5100FAFF390078
:10238000100005000201E800840F5100ECFF390045
:10239000000005008000EB002118980000000600F6
:1023A0000400FA0080089000E1BF9F00F000900058
:1023B000F1BF9F004300200064815700A100290065
:1023C0001CD30200000000000080FA00000006009C
:1023D000889FBE000004BE00780090000020A0008E
:1023E000700498000900E0001B003200070037006D
:1023F000080078008BFF07000000E0000E003A00A4
:1024000008007800C7FD07008904E9007800900003
:1024100065006000E50F500013003A000900E0007D
:10242000F3FF3A0010003700080078007DFF070036
:102430000000E00006003200780090000010A000CC
:102440007004980008007800D5FF070009003700E5
:1024500008007800B3FD0700780090006500600078
:10246000E50F5000F0FF3200780090000020A1003E
:10247000700498004F04BE0000000600F0019000B8
:102480000001EB000308A300090032000318A300B9
:1024900007003A00201990000200E000020032001C
:1024A000CBFF0700010037006FFF0700120020007C
:1024B0000200780000000600889FBE00000478003B
:1024C0000800780087FD0700800478000900E0001C
:1024D00013003200780090000008A30006003200CC
:1024E00070014400230020008100290008007800CA
:1024F0001CD3020000000000090C98000080EB00D3
:10250000100C9800780090000000A0007004980063
:102510000018A3000200320008007800A0FF0700A6
:10252000090078004F04BE00000006000600FA0013
:10253000889FBE008A9FBE000004780000002A0029
:10254000808F500004003A0040002000920F1000DD
:10255000AC003E00A800370010012A00808F500018
:1025600006003A005000200090BF9F00230020008A
:102570006E815700C1002900650037000300E000AC
:10258000A000320012007800980F50009D003A0021
:102590000285E8008305E900F2FF2500F3FF2F0024
:1025A00002804000E0804900EF0F5000E08F5800AB
:1025B00094003E00006001000F003700210037004A
:1025C000300037003B00370040003700450037003F
:1025D0003B003700450037005100370054003700FA
:1025E0005600370064003700770037007A00370064
:1025F0007D003700800037009A0478008B05E900E1
:102600008980450018009000808F5000040036003B
:102610007100200008007800EABC02000000000001
:10262000898444000000EB00040037000000E8004B
:10263000A8009000DAB07C008984E8008B0F50007D
:10264000FAFF39002000200070049800080078008C
:1026500071FC0700E0102C000000E00003003200D5
:10266000080078000EC10200000000008080EB002E
:102670000800780090FF07000000E00061003A00C9
:102680000F003700780090000010A100700498003F
:102690000800780042FF0700E0B129000000E000D8
:1026A00058003200080078001E9B02000000000065
:1026B00054003700780090000010A00070049800CB
:1026C0000800780036FF07004E00370078009000C1
:1026D0000008A3004B0032000800780011FD07003D
:1026E000F7FF370020002000F4FF37009A00780041
:1026F000A1BF9F0008007800F8FE07000080FB00E3
:10270000B0BF9F00430020006C815700B10029003A
:10271000080078001CD302000000000039003700D8
:102720009A0078000800780001FF070035003700A4
:102730000800780017FF0700320037009A0478007D
:102740001A0590008900450038009000808F5000E5
:10275000040036006100200008007800EABC020096
:10276000000000000A0178000800BE004AD3020001
:1027700000000000230037009A0478008B05E90070
:102780008980450038009000808F5000040036009A
:102790006100200008007800EABC02000000000090
:1027A000898444000000EB00040037000000E800CA
:1027B000C8009000DAB07C008984E8008B0F5000DC
:1027C000FAFF39000F003700080078007CBB0200D8
:1027D000000000000B0037000800780040BB02003A
:1027E00000000000070037000800780060BB02000E
:1027F0000000000003003700080078009ED30200AC
:10280000000000004F05BE004F04BE000080FA002B
:1028100000000600920078000100E000050035008D
:10282000B0FC070000F0A7000000EA008001E9000A
:102830001000370013002000F4FF2900848F50009F
:102840000D003600120190008001EB000402E80048
:10285000848F50000800320071024200848F5000C3
:10286000050032009001690003F0A7008301EA002F
:102870008301EA00CF19DE000300780000000600A3
:10288000627E2400F10F200012C860001241900007
:1028900012409800827E24009281600023409800BC
:1028A0001241900032409800A27E24009280600085
:1028B000414098001241900052409800917F2400BE
:1028C0009140780061409800A17F240091407800F9
:1028D00071409800B17F2400914078000148980031
:1028E000C17F24009140780011489800C17E2400E7
:1028F0009140780021489800D17E240091407800D2
:1029000031489800E17E24009140780041489800C9
:10291000F17E24009140780051489800017F240006
:102920009140780061489800117F24009140780020
:1029300071489800417F2400914078000150980030
:10294000517F24009140780011509800317F24007D
:102950009140780021509800717F240091407800C8
:1029600031509800817F24009140780041509800B8
:1029700000000600889FBE008A9FBE000004BE00C3
:102980000A4020000B0020000005450081854D0015
:102990000A0037000800BE006ECB020000000000F5
:1029A000F2FF2F00F30F2000820F5000838F58009A
:1029B00007003A0062044400E0844C008A0F54008F
:1029C0008B8F5C00F3FF39000000EB000100370043
:1029D000100020004F05BE004F04BE00000006009E
:1029E0000001EB00110221000001200018F9020093
:1029F0000000000081012000607E240024F9020014
:102A0000000000005CF9020000000000E17F2400EB
:102A10001100680000F0A7000000EA000000E900D3
:102A20004F00DE00000006002E00FA0023FD2F00FC
:102A30008F814100D2022000AECB020000000000D6
:102A40009FA897006380680000F0A7000000EA00DC
:102A50000000E9004F00DE000080FA0000000600E0
:102A60001600FA00889FBE008A9FBE000005BE00C7
:102A70007E044000E08448000A003700FE815700D1
:102A8000520120000800BE00AECB02000000000092
:102A90000FE897000008A3000A003A006E04440003
:102AA000E0844C0000402000010020000A004000AB
:102AB0008B804800800F5400818F5C00EFFF39004D
:102AC0006044B8000800BE004F05BE004F04BE00C1
:102AD0000080FA00000006001600FA00881F780047
:102AE0008A9FBE008C9FBE00000478000206BE00D4
:102AF00088017800D20220000C00BE00AECB02009C
:102B000000000000086890000040E800006C980099
:102B10007E054600E0854E00CA00370003FE2F0008
:102B20008F814100520120000A00BE00AECB02009E
:102B300000000000C86090006FE0970000C07000C7
:102B400040649800D86090007FE0970000C070005B
:102B500050649800E86090000FE8970000C0700093
:102B600060649800F86090001FE8970000C0700053
:102B700070649800CFF097008180FB00286190007E
:102B80000281FB00386090004800DD000000710009
:102B900000804000206498004800DE003064980007
:102BA000BFF097008180FB00086190000281FB006C
:102BB000186090004800DD000000710000804000B7
:102BC000006498004800DE0010649800AFF09700A1
:102BD0008180FB00685990000281FB0078589000CA
:102BE0004800DD000000710000804000605C98003B
:102BF0004800DE00705C98009FF097008180FB0029
:102C0000485990000281FB00585890004800DD00B0
:102C10000000710000804000405C98004800DE0029
:102C2000505C98008FF097008180FB00285990003D
:102C30000281FB00385890004800DD000000710060
:102C400000804000205C98004800DE00305C980066
:102C5000FFE897008180FB00085990000281FB008B
:102C6000185890004800DD0000007100008040000E
:102C7000005C98004800DE00105C9800EFE89700C8
:102C80008180FB00685190000281FB007850900029
:102C90004800DD0000007100008040006054980092
:102CA0004800DE0070549800DFE897008180FB0048
:102CB000485190000281FB00585090004800DD0010
:102CC0000000710000804000405498004800DE0081
:102CD00050549800CFE897008180FB002851900065
:102CE0000281FB00385090004800DD0000007100B8
:102CF00000804000205498004800DE0030549800C6
:102D0000BFE897008180FB00085190000281FB0022
:102D1000185090004800DD00000071000080400065
:102D2000005498004800DE00105498004849900074
:102D30000281FB00D8499000C819DD000300710032
:102D4000684990000281FB00F8499000C819DD0035
:102D5000830071002FB1970000004100E08048001F
:102D6000404C98004801DE00524C9800614C98009D
:102D70004808DE00704C9800084990000281FB0072
:102D800098499000C819DD0003007100284990009F
:102D90000281FB00B8499000C819DD008300710072
:102DA0001FB1970000004100E0804800004C9800EF
:102DB0004801DE00124C9800214C98004808DE00C3
:102DC000304C9800484190000281FB00D8419000AF
:102DD000C819DD0003007100684190000281FB000A
:102DE000F8419000C819DD00830071000FB1970011
:102DF00000004100E0804800404498004801DE00A7
:102E000052449800614498004808DE0070449800DD
:102E1000AFE897008180FB00284190000281FB0011
:102E2000384090004800DD00000071000080400044
:102E3000204498004800DE00304498006E054500AC
:102E4000E0854D0000402000010020000C00400003
:102E50008D804800800F5500818F5D002FFF390065
:102E60004F06BE004F05BE004F0478000080FA00F8
:102E7000000006004F03B000889FBE008A1F780044
:102E80008E1F78000004BE00E00F5100E08F590053
:102E900006003A000F0078006003B1001500090039
:102EA0000018EB000058EB0003003700A0FC2F00D7
:102EB0000F00400008FF070030002000D0A79F004F
:102EC0000800BE00ABFE07000000E0000300320077
:102ED0000800BE000CCC0200000000000005EB0062
:102EE000A1FC2F008F8040000A804000B040780095
:102EF000E1C79F006EFC2F000F074700306F78007E
:102F000010407800104798003FA19700CFA197008C
:102F10000800BE0046CC020000000000620444002D
:102F2000E0844C0063054500D0022000800F55006E
:102F3000EBFF3A004F0778004F0578004F04BE00C2
:102F40004F03B1000000060000C023001100200064
:102F5000B5FE07000000E00014003A000000240065
:102F600011002000B0FE07006011B8000000E00072
:102F7000080032000000240011002000B8FE070005
:102F8000E00F5000E08F580028003A0002002400B3
:102F90001300200000C0230011002000B5FF07002F
:102FA000E0C12300110020000000060000C0230043
:102FB00011002000AAFE0700E00F5000E08F58002B
:102FC0001A003A00000024001100200096FE0700BD
:102FD0000000E00008003A0002C0230013002000B7
:102FE0000000240011002000A2FF0700E0012400DF
:102FF0001100200000000600000024001100200045
:1030000097FE0700E00F5000E08F580007003A00DD
:10301000020024001300200000C023001100200043
:1030200094FF0700E0C1230011002000000006000B
:10303000FC874700881F78008A9FBE008C9FBE00D7
:103040008E1F78000004EB00B1938000F028200070
:10305000808F50002F003400BBFF07000006BE0029
:10306000E0FD2F000F00400005FE07000C05BE002C
:10307000E1FD2F008F80400008804000B0407800C4
:10308000A1DF9F00AEFD2F000F074700306F7800D3
:1030900010407800104798005FA99700EFA99700AB
:1030A0000A00BE0046CC0200000000006205450098
:1030B000E0854D0063044400F50F5400ECFF3A0036
:1030C0006E004600E0804E00020024001300200045
:1030D000820F5000838F580005003A0002C0230081
:1030E0001300200063FF07001800200009003700CC
:1030F000180020000440240015002000840F500018
:10310000858F580003003A0000C023001100200002
:1031100058FF0700080078004F0778004F06BE00F0
:103120004F05BE004F047800CF01B100000006003B
:10313000303F8200E10F400002003200617E240037
:103140008008E80040610200000000000000E0008C
:1031500006003D00707F240090407800E1CF4000E1
:103160000A0032000148E80008003700E80040008B
:10317000627E2400E2C07800E1CF4000030032000C
:103180008140E80068014100017178008464AB006F
:103190000F003200C2F40200000000000000E00056
:1031A00006003200403F8200E10F4000080032007C
:1031B000817E24008008E80000000600503F820065
:1031C000E10F400002003200A17E24008008E800E8
:1031D000000006000080FB00C300DE00927F240098
:1031E00002814000C308DD000100500011002000F2
:1031F0000008DD0012497000000006006105200093
:10320000810F50000B0039008100E800810F500051
:1032100004003600F0804000810F500005003A00A5
:103220000200370070C0B300EAFF370000C1B300EE
:10323000E8FF07000000060021062000810F500073
:1032400011003E008180E900810F50001D00310017
:10325000F1032000810F500007003E00E68050007F
:10326000810F500015003100A002B100E40F5000A2
:103270001C003E000F0037000005B100E50F5000B4
:1032800018003E000D00370051062000810F50004D
:1032900004003E008100E900810F50000D00310064
:1032A0000A00370061062000810F50000D003A002F
:1032B0000A003700F0C0B3000700370080C0B30039
:1032C00005003700E0C0B3000300370090C0B30032
:1032D0000100370010C1B300BEFF370000C1B300CA
:1032E000BCFF0700000006008000EB004002B100B8
:1032F0000180B100EF0F5000E08F58001F003E002A
:10330000006001000F0037000E0037000D0037008D
:103310000E0037000F0037000E0037000D00370099
:10332000080037000D0037000E0037000D00370091
:103330000E0037000D0037000C0037000F0037007B
:103340000C003700A0C0B30009003700D0C0B300A4
:1033500007003700C0C0B3000500370020C1B3002C
:1033600003003700B0C0B3000100370030C1B30024
:1033700098FF370070C1B30096FF070000000600F9
:10338000724980008349800061004100E08049006B
:10339000704988008149880002302A0023002000FB
:1033A000820F5000838F580007003A002E29EF004B
:1033B0003029EF00807F240090407800E1CF40006A
:1033C000010032000148E800000006000001EB00A7
:1033D000110221000001200018F902000000000085
:1033E00081012000607E240024F90200000000001A
:1033F0005CF9020000000000F03F8A0000000600B7
:1034000020C0B30073FF37002C09EC00604988002E
:1034100001A62E00810F500002003A002C29EF0077
:1034200043FF070000000600889FBE008A1F780047
:1034300040F12000B1788000910078004A0020001F
:103440008004EB0018002000908F500032003600FE
:10345000770037008800440081004000E0FF2F0023
:10346000110050008000EB00F00F5000E08F58007A
:1034700022003E0000600100100037000F003700FE
:103480000E0037000D0037000C0037000B0037002E
:103490000C003700190037000C0037000B00370014
:1034A0000C00370015003700100037000B00370004
:1034B0000C0037000F0037000E003700F0C0B300DB
:1034C0000D00370080C0B3000B003700E0C0B30030
:1034D0000900370000C1B3000700370010C1B30076
:1034E0000500370070C0B3000300370040C1B300CF
:1034F0000100370050C1B30036FF0700B0788000EC
:1035000060007D00808F540001003100800478004D
:103510000884E80064054500B0788000900F5400EE
:10352000CCFF39003F003700B1788000080044002C
:10353000610078004C01DE008001EB00ED0F5100CE
:10354000E08F590036003E00026001000D00370098
:10355000330037001D0037000D0037001000370022
:1035600013003700160037002D0037002C003700FD
:1035700018003700150037001A0037002500370003
:103580001E003700890F540025003900280037003D
:10359000F1FF20000100600027FF07002000370036
:1035A000F1FF20000100600014FF07001C0037003D
:1035B000F1FF2000010060001FFF0700030037003B
:1035C000F1FF2000010060000CFF07000884E80004
:1035D000140037004400DD004480DE000800400095
:1035E000080037000800E800000040006100780093
:1035F00011FF0700630444000A003700F1FF2000B8
:1036000001006000808F54000500310080047800C4
:1036100003003700F1FF20000100600032FF0700C7
:103620000804E80040F12000900F5400BEFF39006C
:103630004F0578004F04BE0000000600D07E240035
:1036400090407800E1CF4000010032000148E800DE
:1036500075FF3700E2FC07000000E00003003A00BD
:10366000607E24000C0009000018EB004027AB002E
:103670000300320010C0B300D6FE07004027A900A7
:10368000807F24001004E00004003A00313F8200F3
:10369000005A2000808F50000600360064FE0700AC
:1036A0000000E00003003200607E24000C000900EE
:1036B0000018EB00C07E240090407800E1CF40006D
:1036C000010032000148E800000006001C00FA007A
:1036D000881F78008A9FBE0000047800580190007F
:1036E000E801900008007800D04F020000000000C0
:1036F0000AC023001B0020000A00BE006ECB02009F
:103700000000000080B79F0091B79F00E3FD2F00ED
:103710008F8141003200200001FE2F008F80400089
:10372000080078005E4D0200000000007FA89700AE
:10373000E30F500025003A0062054500E0854D008A
:103740000040240011002000800F5500818F5D0093
:10375000E9FF3A007C80570049FC0700E3FD2F0099
:103760008F81410052012000FC8057000800780042
:103770005E4D020000000000607E24000C00090085
:103780000018EB0000C023001100200079FC0700A6
:103790000000E0000400320000C0230011002000FF
:1037A0000CCC0200000000000000240011002000EA
:1037B00070FC07000000E00004003200000024005C
:1037C000110020000CCC0200000000004F05BE00DC
:1037D0004F0478000080FA00000006009008900076
:1037E000E001900001814000630179008100E9005F
:1037F0001108980002007800000006000003BE00D7
:10380000530020000002EB000271220011000900A9
:103810000283D80001037800800278000500E000F0
:1038200004003A000400E00002003A00E10F5100F9
:1038300003003A0000C3B30080DB42001400200004
:10384000A5002000110009000581D80000017800C2
:103850008301E900EDFF3A00070078000000060050
:10386000E6FF0700E1C2B3000148780071C7B3006A
:1038700001687800F6C0500001687800F5C040008B
:10388000016878008040EB001140980000000600BD
:10389000889FBE008A1F7800800478004904900049
:1038A00009007800CDFF07000000400068047800A0
:1038B0004905900009007800C8FF0700000040009B
:1038C000EA007800EF0F5400080032000800E00022
:1038D0000600350070022000800F540003003C00F9
:1038E00008407800DAC50200000000004F057800AB
:1038F0004F04BE00000006000E00FA00881F78008A
:10390000F0805700050009008018EB008058EB009C
:1039100001C7B30081F79F0040049000AFFF07008C
:103920000000400068047800100020008474020049
:10393000000000005EE00200000000000000EB005C
:10394000E10F440004003200EF80570008007800C7
:10395000C3FF070070805700E6E00200000000008F
:103960004F0478000080FA00000006000E00FA0004
:10397000881F7800F0805700050009008018EB00D0
:103980008058EB0021C7B30081F79F0040049000EE
:1039900092FF07000000400068047800E10F440037
:1039A00003003A0062B30200000000000900370083
:1039B000100020008474020000000000EF80570017
:1039C00008007800A6FF07007080570006B30200C9
:1039D000000000004F0478000080FA00000006009C
:1039E0000E00FA00881F7800F080570005000900DB
:1039F0008018EB008058EB0021C7B30081F79F00CF
:103A00004004900075FF0700000040006804780043
:103A10001000200084740200000000005EE002003C
:103A2000000000000000EB00E10F44000400320041
:103A3000EF8057000800780089FF0700708057006A
:103A4000E6E00200000000004F0478000080FA0069
:103A500000000600F0874700889FBE008A1F78009C
:103A60008E1F78000004780076805700050009005A
:103A70000018EB000058EB007687570020C7B30012
:103A8000005F7800C80490000800780053FF07002A
:103A90000000400069057800080078004FFF07002B
:103AA000800478008E0078000A0078006CFF070020
:103AB00089844400480090008904400076805700C3
:103AC00088B3020000000000800C78004F077800E7
:103AD0004F0578004F04BE000F01B1000000060042
:103AE0000E00FA00881F7800F080570005000900DA
:103AF0008018EB008058EB0031C7B30081F79F00BE
:103B00004004900035FF0700000040006804780082
:103B10001000200084740200000000005EE002003B
:103B2000000000000800780000E102000000000032
:103B30000000E00006003200EF8057000800780027
:103B400047FF070070805700E6E002000000000019
:103B50004F0478000080FA0000000600E487470068
:103B6000889FBE008A9FBE008C9FBE008E1F78007B
:103B700080007800410490000100780081BF9F0020
:103B800016FF070000004000E80478008FB8970097
:103B9000410490000100780010FF07000000400081
:103BA000680478008FB89700410590000100780004
:103BB0000AFF0700000040006A0578008FB89700F0
:103BC000C10590000100780004FF070000004000DC
:103BD000EB0578008FB8970041069000010078004F
:103BE000FEFE0700000040006C0678008FB89700CA
:103BF000C106900001007800F8FE070000004000B8
:103C0000ED0678008FB8970041079000010078001A
:103C1000F2FE0700000040006E0778008FB89700A2
:103C2000410190000100780082BF9F00EBFE070079
:103C3000000040000FB99700E20378000010200058
:103C400087BF9F0084740200000000008FBB9700B4
:103C50000E4378008D4278000C4278008B4178004A
:103C60000A4178008840780009407800BAC602000E
:103C7000000000004F0778004F06BE004F05BE0051
:103C80004F04BE004F00B10000000600889FBE0038
:103C90008A9FBE00000578004A0490000A00780060
:103CA000CEFE07000000400068047800CA049000BF
:103CB0000A007800C9FE070000004000E90478000F
:103CC000CA0590000A007800C4FE0700000040000A
:103CD0006B01780089407800084078000AC702002C
:103CE000000000004F05BE004F04BE0000000600AB
:103CF000889FBE008A9FBE00000578004A0490009D
:103D00000A007800B5FE0700000040006804780053
:103D1000CA0490000A007800B0FE070000004000CE
:103D2000E9047800CA0590000A007800ABFE07009D
:103D3000000040006B01780089407800084078005E
:103D400026C70200000000004F05BE004F04BE0061
:103D500000000600889FBE008A9FBE000005780014
:103D60004A0490000A0078009CFE07000000400012
:103D700068047800CA0490000A00780097FE0700E3
:103D800000004000E9047800CA0590000A007800AD
:103D900092FE0700000040006B0178008940780027
:103DA0000840780042C70200000000004F05BE0036
:103DB0004F04BE0000000600889FBE008A9FBE0020
:103DC0008C1F780000047800C80490000800780078
:103DD00082FE070000004000E9057800C80490005A
:103DE000080078007DFE07000000400069057800AB
:103DF000C80490000800780078FE0700000040002A
:103E0000E9047800480690000800780073FE070077
:103E1000000040006C047800200020008474020040
:103E2000000000008B40780000C2B300DAC5020039
:103E3000000000008A40780030C2B300DAC50200FA
:103E4000000000008940780010C2B300DAC502000B
:103E5000000000008840780020C2B300DAC50200EC
:103E6000000000004F0678004F05BE004F04BE0062
:103E700000000600E4874700889FBE008A9FBE00BE
:103E80008C9FBE008E1F7800800078004104900057
:103E90000100780081BF9F0050FE07000000400035
:103EA000E80478008FB89700410490000100780082
:103EB0004AFE070000004000680478008FB89700B1
:103EC000410590000100780044FE0700000040001A
:103ED0006A0578008FB89700C1059000010078004E
:103EE0003EFE070000004000EB0578008FB8970009
:103EF000410690000100780038FE070000004000F5
:103F00006C0678008FB89700C10690000100780019
:103F100032FE070000004000ED0678008FB89700E1
:103F200041079000010078002CFE070000004000CF
:103F30006E0778008FB8970041019000010078006B
:103F400082BF9F0025FE0700000040000FB99700C8
:103F5000E20378004000200087BF9F0084740200C5
:103F6000000000008FBB97000E4378008D42780060
:103F70000C4278008B4178000A4178008840780034
:103F8000094078005EC70200000000004F0778007B
:103F90004F06BE004F05BE004F04BE004F00B100EB
:103FA00000000600889FBE008A1F78000004780089
:103FB000C80490000800780008FE070000004000D8
:103FC000E9047800480590000800780003FE070027
:103FD000000040006A047800400020008474020061
:103FE000000000008940780060C1B300DAC502001B
:103FF000000000008840780070C1B300DAC50200FC
:10400000000000004F0578004F04BE0000000600CD
:10401000881F780040049000F0FD07000000400079
:10402000680478000004200084740200000000008E
:1040300088407800D0C1B300DAC50200000000005B
:104040004F04780000000600881F780040049000AC
:10405000E2FD070000004000680478000001200035
:10406000847402000000000088407800E0C1B300C2
:10407000DAC50200000000004F04780000000600CE
:10408000889FBE008A1F780000047800C804900052
:1040900008007800D1FD070000004000E904780026
:1040A0004805900008007800CCFD070000004000A3
:1040B0006A047800002020008474020000000000E0
:1040C0008940780060C2B300DAC502000000000039
:1040D0008840780070C2B300DAC50200000000001A
:1040E0004F0578004F04BE0000000600889FBE0008
:1040F0008A1F780080047800490490000900780045
:10410000B6FD0700000040006804780049059000F3
:1041100009007800B1FD070000004000EA047800C3
:104120001000200084740200000000005EE0020025
:10413000000000000800BE0020E1020000000000B6
:104140004F0578004F04BE0000000600889FBE00A7
:1041500000047800C8049000080078009FFD070064
:104160000000400000804400000178008000EB0067
:104170000308200032824100F30F2000830F520019
:104180000500360001B0290008007800B890020050
:1041900000000000060037008100E800E30820006E
:1041A000838F5000F2FF3A00D2F6020000000000B8
:1041B0004F04BE0000000600881F780040049000F5
:1041C00086FD070000004000680078000000E00065
:1041D000030032007EB10200000000000200370040
:1041E00088B10200000000004F04780000000600C3
:1041F0000E00FA00889FBE008A1F78000004780035
:10420000C80490000800780074FD0700000040001A
:10421000690578000800780070FD070080047800C8
:1042200074805700050009000018EB000058EB00EF
:1042300050C7B300C0EF9F00E10F450008003A00EF
:104240000000EB00B6B4020000000000480090003F
:104250008984440089044000800CEB00140037007E
:10426000F38057000A00780064FD0700E1C2B30044
:104270000148780041C6B30001687800E3C05000EF
:1042800001687800F3C04000016878008040EB00CE
:10429000114098008984440048009000890440003F
:1042A00074805700B6B4020000000000800C780053
:1042B0004F0578004F04BE000080FA0000000600A1
:1042C000889FBE008A9FBE0080047800C9059000C8
:1042D0000900780041FD070000057800090078001A
:1042E0003EFD070000047800090078003BFD070050
:1042F00008044400C9009000088440008000400089
:104300000A0545000A8045008AB502000000000049
:10431000000CD1004F05BE004F04BE000000060097
:10432000889FBE008A9FBE0080047800C905900067
:104330000900780029FD07000005780009007800D1
:1043400026FD0700000478000900780023FD07001F
:1043500008044400C9009000088440008000400028
:104360000A0545000A80450044B50200000000002F
:10437000000CD1004F05BE004F04BE000000060037
:10438000889FBE008A1F780080047800490490004E
:104390000900780011FD0700000040006805780062
:1043A000090078000DFD070000004000490490005E
:1043B000000444006150B9000000400081804800C2
:1043C00004B5020000000000000C78004F057800E2
:1043D0004F04BE0000000600881F780040049000D3
:1043E000FEFC0700000040006800780082C3020065
:1043F00000000000C2C40200000000004F0478006A
:1044000000000600881F7800980E2000803E2000E3
:104410003CFA0200000000000804E900FBFF3A003B
:104420004F0478000000060001C2B30080C0B30052
:10443000DAC5020000000000F2FF07008040EB0038
:1044400080C0B300DAC502000000000001C2B30062
:1044500090C0B300DAC5020000000000E9FF0700C9
:104460008040EB0090C0B300DAC5020000000000FD
:1044700001C2B300A0C0B300DAC502000000000012
:10448000E0FF07008040EB00A0C0B300DAC50200E7
:104490000000000001C2B300B0C0B300DAC50200E2
:1044A00000000000D7FF07008040EB00B0C0B30061
:1044B000DAC502000000000001C2B300C0C0B300B2
:1044C000DAC5020000000000CEFF07008040EB00CC
:1044D000C0C0B300DAC502000000000001C2B30092
:1044E000D0C0B300DAC5020000000000C5FF07001D
:1044F0008040EB00D0C0B300DAC50200000000002D
:1045000001C2B30020C0B300DAC502000000000001
:10451000BCFF07008040EB0020C0B300DAC50200FA
:104520000000000001C2B30030C0B300DAC50200D1
:1045300000000000B3FF07008040EB0030C0B30074
:10454000DAC502000000000001C2B30040C0B300A1
:10455000DAC5020000000000AAFF07008040EB005F
:1045600040C0B300DAC504000000000001C2B3007F
:1045700020C2B300DAC5020000000000A1FF07005E
:104580008040EB0020C2B300DAC50200000000004A
:1045900001C2B30001407800DAC50200000000004B
:1045A00098FF07008040EB0000C2B300DAC50200AC
:1045B0000000000001C2B30030C2B300DAC502003F
:1045C000000000008FFF07008040EB0030C2B30006
:1045D000DAC502000000000001C2B30010C2B3003F
:1045E000DAC502000000000086FF07008040EB00F3
:1045F00010C2B300DAC504000000000001C2B3001D
:10460000C0C1B300DAC50200000000007DFF070052
:104610008040EB00C0C1B300DAC50200000000001A
:1046200001C2B30040C2B300DAC5020000000000BE
:1046300074FF07008040EB0040C2B300DAC50200FF
:104640000000000001C2B30050C2B300DAC502008E
:10465000000000006BFF07008040EB0050C2B30079
:10466000DAC502000000000001C2B300F0C1B300CF
:10467000DAC502000000000062FF07008040EB0086
:10468000F0C1B300DAC502000000000001C2B300AF
:1046900080C1B300DAC502000000000059FF070026
:1046A0008040EB0080C1B300DAC5020000000000CA
:1046B00001C2B30090C1B300DAC5020000000000DF
:1046C00050FF07008040EB0090C1B300DAC5020044
:1046D0000000000001C2B300A0C1B300DAC50200AF
:1046E0000000000047FF07008040EB00A0C1B300BE
:1046F000DAC502000000000001C2B300B0C1B3007F
:10470000DAC50200000000003EFF07008040EB0019
:10471000B0C1B300DAC504000000000001C2B3005C
:1047200000C1B300DAC502000000000035FF070039
:104730008040EB0000C1B300DAC5020000000000B9
:1047400001C2B30010C1B300DAC5020000000000CE
:104750002CFF07008040EB0010C1B300DAC5020057
:104760000000000001C2B30040C1B300DAC502007E
:104770000000000023FF07008040EB0040C1B300B1
:10478000DAC502000000000001C2B30050C1B3004E
:10479000DAC50200000000001AFF07008040EB00AD
:1047A00050C1B300DAC502000000000001C2B3002E
:1047B00020C1B300DAC502000000000011FF0700AD
:1047C0008040EB0020C1B300DAC502000000000009
:1047D00001C2B30030C1B300DAC50200000000001E
:1047E00008FF07008040EB0030C1B300DAC50400C9
:1047F000000000008040EB0050C0B300DAC50200AA
:1048000000000000C5FF070001C2B300D0C1B30023
:10481000DAC5020000000000FAFE07008040EB004D
:10482000D0C1B300DAC502000000000001C2B3002D
:10483000E0C1B300DAC5020000000000F1FE07008D
:104840008040EB00E0C1B300DAC5020000000000C8
:1048500001C2B30050C0B300DAC50200000000007E
:10486000E8FE07008040EB0050C0B300DAC502004C
:104870000000000001C2B30060C0B300DAC502004E
:1048800000000000DFFE07008040EB0060C0B300C6
:10489000DAC502000000000001C2B30070C0B3001E
:1048A000DAC5020000000000D6FE07008040EB00E1
:1048B00070C0B300DAC50200000000004FFF07001F
:1048C0002AFF070001C2B30060C2B300DAC50200CC
:1048D00000000000CBFE07008040EB0060C2B30088
:1048E000DAC502000000000001C2B30070C2B300CC
:1048F000DAC5020000000000C2FE07008040EB00A5
:1049000070C2B300DAC502000000000001C2B300AB
:104910000040EB00DAC5020000000000B9FE07000D
:104920008040EB0001407800DAC502000000000082
:1049300001C2B300E0C0B300DAC50200000000000D
:10494000B0FE07008040EB00E0C0B300DAC5020013
:104950000000000001C2B30010C0B300DAC50200BD
:1049600000000000A7FE07008040EB0010C0B3006D
:10497000DAC502000000000001C2B30060C1B3004C
:10498000DAC50200000000009EFE07008040EB0038
:1049900060C1B300DAC502000000000001C2B3002C
:1049A00070C1B300DAC502000000000095FE0700E8
:1049B0008040EB0070C1B300DAC5020000000000C7
:1049C00099FE37008BFF070001C2B30020C0B3007F
:1049D000DAC502000000000001C2B30000C1B3004C
:1049E000DAC502000000000001C2B30010C1B3002C
:1049F000DAC502000000000001C2B30040C1B300EC
:104A0000DAC502000000000001C2B30020C1B300FB
:104A1000DAC502000000000001C2B30030C1B300DB
:104A2000DAC502000000000001C2B3000040EB0044
:104A3000DAC502000000000001C2B30010C0B300DC
:104A4000DAC502000000000001C2B300E0C1B300FB
:104A5000DAC502000000000001C2B30070C2B3005A
:104A6000DAC502000000000001C2B30080C1B3003B
:104A7000DAC502000000000001C2B30090C1B3001B
:104A8000DAC502000000000001C2B300A0C1B300FB
:104A9000DAC502000000000001C2B300B0C1B300DB
:104AA000DAC502000000000001C2B300C0C1B300BB
:104AB000DAC502000000000001C2B30040C2B3002A
:104AC000DAC502000000000001C2B30050C2B3000A
:104AD000DAC502000000000001C2B300F0C1B3005B
:104AE000DAC502000000000001C2B300D0C1B3006B
:104AF000DAC502000000000001C2B30060C1B300CB
:104B0000DAC502000000000001C2B30070C1B300AA
:104B1000DAC502000000000001C2B30080C0B3008B
:104B2000DAC502000000000001C2B300D0C0B3002B
:104B3000DAC502000000000001C2B300E0C0B3000B
:104B4000DAC5020000000000008020006C74020042
:104B5000000000001000200086E8040000000000B3
:104B6000C028210072F32F0090004100A012200005
:104B7000808F500005003E003809A8008040EB00FF
:104B800063405000DAC502000000000060272100E9
:104B90008080E8009100780010804000813E200075
:104BA0000182B900A2F820001100090042AAD80031
:104BB00080007800C118B10010022000808F5000E2
